:020000040801F1
:100000004892002039010108C1430108C343010897
:10001000E9430108ED430108F14301080000000035
:10002000000000000000000000000000D5F50108FD
:10003000F54301080000000041F6010851F60108EF
:10004000530101085301010853010108D36F01084E
:10005000530101085301010853010108530101082C
:10006000530101085301010853010108530101081C
:10007000530101085301010853010108530101080C
:1000800053010108530101085301010853010108FC
:1000900053010108530101085301010853010108EC
:1000A00053010108530101085301010853010108DC
:1000B000835C010853010108530101085301010841
:1000C00053010108530101085301010853010108BC
:1000D000530101084B460108A15C01086154010865
:1000E00021710108636F01085301010853010108E0
:1000F000530101085301010853010108530101088C
:100100005D7401083580010853010108530101089D
:10011000530101085301010853010108530101086B
:1001200053010108DFF80CD00FF042FF00480047F0
:10013000D93F0108489200200648804706480047FA
:10014000FEE7FEE7FEE7FEE7FEE7FEE7FEE7FEE787
:10015000FEE7FEE76F42010825010108324901432D
:10016000324A1160704770B5002100230F22C47815
:100170001CB32E4C246804F4E064C4F5E064C4F3BA
:100180000721C1F10404E3B20A4144789C40E1B282
:100190008478144021430C07210E254C05786155C5
:1001A000047804F01F050124AC4005786D11AD0002
:1001B00005F1E025C5F8004109E0047804F01F05C9
:1001C0000124AC401B4D0678761145F8264070BDE1
:1001D000194A0A400243154B1B1F1A60704739B178
:1001E000124A121D12680243104B1B1D1A6006E0D2
:1001F0000E4A121D126882430C4B1B1D1A60704779
:10020000042808D14FF0E021096941F004014FF0C2
:10021000E022116107E04FF0E021096921F00401BB
:100220004FF0E022116170470000FA050CED00E08C
:1002300000E400E080E100E080FFFF1F10B504460D
:10024000FE48844207D10121401500F09FFE0021A5
:10025000601500F09BFE10BD30B502460020002363
:100260005068F74C20400D790C6844EA052420437F
:1002700050609068F34C2040D1E903542C438D68C2
:100280002C434D7944EA450420439060106B20F0E4
:10029000F8700C7D641EE4B2234340EA03501063FF
:1002A00030BD002101600171417181604FF04071EA
:1002B000C1600021016101210175704701460020E4
:1002C000E14A106820F440300A681043DE4A1060AA
:1002D000704700210160704721B1826842F001023D
:1002E000826003E0826822F001028260704721B1DF
:1002F000826842F00402826003E0826822F0040215
:10030000826070471AB143680B43436002E0436860
:100310008B43436070470A460021816821F0F00159
:100320001143816070470A4600214168C74B19405C
:100330001143416070478162C26270470A460021E2
:10034000416821F01F0111434160704730B1BE493F
:10035000096841F40001BC4A116005E0BA49096826
:1003600021F40001B84A11607047F0B504460D460B
:10037000002000211D2D11DDE06DA5F11E0606EB0C
:100380004607072606FA07F18843A5F11E0606EB85
:10039000460603FA06F10843E06534E0132D11DD4B
:1003A000E068A5F1140606EB4607072606FA07F1F2
:1003B0008843A5F1140606EB460603FA06F1084346
:1003C000E06020E0092D11DD2069A5F10A0606EBA9
:1003D0004607072606FA07F18843A5F10A0606EB49
:1003E000460603FA06F1084320610CE0606905EB5C
:1003F0004507072606FA07F1884305EB450603FA89
:1004000006F108436061072A0FDA206C561E06EBDE
:1004100086071F2606FA07F18843561E06EB860656
:1004200005FA06F1084320644AE00D2A0FDAE06B72
:10043000D61F06EB86071F2606FA07F18843D61F4C
:1004400006EB860605FA06F10843E06338E0132A56
:1004500011DAA06BA2F10D0606EB86071F2606FA3D
:1004600007F18843A2F10D0606EB860605FA06F1B0
:100470000843A06324E0192A11DA606BA2F1130685
:1004800006EB86071F2606FA07F18843A2F113063A
:1004900006EB860605FA06F10843606310E0206B60
:1004A000A2F1190606EB86071F2606FA07F1884314
:1004B000A2F1190606EB860605FA06F10843206349
:1004C000F0BD816841F080418160704701460020A5
:1004D0008A6802F080420AB1012000E000207047E3
:1004E00021B1826842F48062826003E0826822F473
:1004F00080628260704721B1826842F002028260AD
:1005000003E0826822F002028260704710B50A465A
:1005100000210023416821F46041531E41EA433128
:10052000416010BD21B1426842F40062426003E0C4
:10053000426822F40062426070470146886D80B2D2
:10054000704721B1826842F48072826003E0826861
:1005500022F480728260704721B1826842F4007296
:10056000826003E0826822F4007282607047F0B516
:10057000044615460020002200261D2911DDE06DED
:10058000A1F11E0707EB470C072707FA0CF290436F
:10059000A1F11E0707EB470703FA07F21043E065D6
:1005A00034E0132911DDE068A1F1140707EB470CD3
:1005B000072707FA0CF29043A1F1140707EB47074E
:1005C00003FA07F21043E06020E0092911DD2069F9
:1005D000A1F10A0707EB470C072707FA0CF2904333
:1005E000A1F10A0707EB470703FA07F2104320615E
:1005F0000CE0606901EB410C072707FA0CF290430D
:1006000001EB410703FA07F210436061606CC0F32D
:100610000156EF1C06F1010CA7EB0C0707EB870C4A
:100620001F2707FA0CF29043EF1C06F1010CA7EB11
:100630000C0707EB870701FA07F209E000240140E5
:10064000FFFEFFFCFDF7FFC004270140FFFD3FFF59
:1006500010436064F0BD10B50A4600210023416CD0
:1006600021F44011531E41EA0351416410BD08B505
:10067000002300930090009B0B440093009B1A60A2
:1006800008BD0A460021816821F470211143816070
:1006900070470A460021816821F4401111438160AE
:1006A0007047816841F480018160704701460020F5
:1006B0008A6802F480020AB1012000E0002070473D
:1006C00021B1426842F48062426003E0426822F451
:1006D00080624260704721B1426842F480524260B9
:1006E00003E0426822F480524260704708B5024637
:1006F00000200090009201F13000009B184400900F
:100700000098006880B208BD10B50B460021D9B230
:10071000012404FA01F11AB144680C43446002E078
:1007200044688C43446010BD0246002013680B40AF
:100730000BB1012000E000207047CA4302607047FF
:1007400070B502460020002300240B0A55680126DC
:100750008E4005EA060415681D4015B10CB1012054
:1007600000E0002070BD00220A12D34303607047EE
:10077000002044490860091D0860091D0860091D22
:1007800008606FF07F403F491431086070470021D6
:100790003C498279002A3AD00A46126803689A4393
:1007A0000B461A600A1D126803689A430B1D1A60F3
:1007B000027911440A6803681A430A60314A083210
:1007C000126803689A432F4B08331A601A1D126887
:1007D00003689A432B4B0C331A604279102A0ED1CE
:1007E0001A1F126803681A43264B08331A601A1D31
:1007F000126803681A43234B0C331A600DE0214939
:10080000427911440A6803681A430A6005E00279D4
:1008100011440A6803689A430A6070470021016026
:1008200001710C214171002181717047154910310E
:1008300009680143134A10321160704701460020D5
:10084000104A143212680A400AB1012000E0002068
:1008500070470C491431086070470146002000229F
:10086000084B1B6803EA0102064B14331B680B405C
:1008700013B10AB1012000E0002070470149143192
:10088000086070470004014010B504468548844262
:1008900008D10121084600F068FB0021012000F08A
:1008A00064FB52E08048844208D10121022000F01C
:1008B0005CFB0021022000F058FB46E07B488442AC
:1008C00008D10121042000F050FB0021042000F099
:1008D0004CFB3AE07648844208D10121082000F020
:1008E00044FB0021082000F040FB2EE071488442C8
:1008F00008D10121102000F038FB0021102000F069
:1009000034FB22E06C48844208D10121402000F0F1
:100910002CFB0021402000F028FB16E067488442B1
:1009200008D10121802000F020FB0021802000F070
:100930001CFB0AE06248844207D10121202000F01C
:1009400014FB0021202000F010FB10BDF0B50A467A
:1009500000210023002400BF3DE0012505FA01F33A
:10096000156805EA03049C4234D105684F0003264C
:10097000BE40B543056015794E00B5400668354365
:1009800005601579012D02D01579022D16D18568E3
:100990004F000326BE40B543856055794E00B540F3
:1009A000866835438560858801268E40B5438580FD
:1009B000858896798E40B6B235438580C5684F00EC
:1009C0000326BE40B543C560D5794E00B540C66824
:1009D0003543C560491C1029BFD3F0BD4FF6FF71E8
:1009E00001600021017141718171C171704708B5C9
:1009F0004FF480320092009A0A430092009AC2613A
:100A0000C161009AC261C2690092C269009208BDC8
:100A100002460020138A0B400BB1012000E00020A9
:100A200070470146088A704702460020938A0B40AF
:100A30000BB1012000E0002070470146888A704712
:100A400001837047418370470AB1018300E041830D
:100A5000704781827047828A4A4082827047F0B52F
:100A6000002300244D07ED0E02FA05F3CE1000F12D
:100A7000200555F826504E07F70E0F26BE40B54309
:100A8000CF1000F1200646F82750CE1000F12005C7
:100A900055F8265045EA0304CE1000F1200545F82C
:100AA0002640F0BD00000240000402400008024061
:100AB000000C02400010024000180240001C0240DE
:100AC0000014024010B50121080700F070FA00215F
:100AD0004FF0805000F06BFA10BD4D49086270472E
:100AE000014600204B4A106820F0E00008431060E7
:100AF000704747490861704708B500220092444A90
:100B0000A03202440092009A116008BD40498862F8
:100B100070473F4948627047014600203D4A1068CF
:100B200020F4C050084320F00C023A4B1A60704782
:100B300058B13849096841F00101364A116011463F
:100B4000096841F4804111600AE03249096821F4E2
:100B50008041304A11601146096821F0010111609D
:100B6000704710B5024600202A4B186820F0030099
:100B700010431860284B1B6823F00403264C2360A5
:100B8000012901D130BF00E020BF10BD10B50246E1
:100B90000020204B186820F00300104318601E4B03
:100BA0001B6843F004031C4C2360012901D130BFB2
:100BB00000E020BF184B1B6823F00403164C236091
:100BC00010BD1448006840F004001249086008464F
:100BD000006840F0020008600F48006840F0040020
:100BE0000D49086000BF00BF30BF704701460020BC
:100BF000084A52680A400AB1012000E0002070470C
:100C00000449096841EA8001024A11607047000006
:100C100000000E420070004010ED00E0F94800684E
:100C200040F48070F7490860F64808300068F649DB
:100C30000840F44908310860F2480068F349084068
:100C4000F04908600846006820F480200860ED48FC
:100C50000830006820F47D00EA490831086000206F
:100C6000091D086070470021E64A921C1170114668
:100C70000870704710B501460022002300204A1179
:100C8000012A02D1DF4C236802E0DE4C34342368B1
:100C900001F01F02012494401C400CB1012000E02F
:100CA000002010BD38B5002000900024002500BFB2
:100CB0003120FFF7DFFF05460098401C00900098A8
:100CC000B0F5A06F01D0002DF2D03120FFF7D2FF98
:100CD00008B1012400E00024204638BDC949C91DDF
:100CE0000870704701460020C64A121D106820F4A3
:100CF0006040084310607047C5490862704701466C
:100D00000020C04A121D106820F4F85040EA01206B
:100D100010607047BE49086070470021B94A3532FB
:100D20001170114608707047BA490860704710B5D5
:100D300041EA02030343B34C0A34237010BDB449A3
:100D400008667047B24908677047B2492C3108609D
:100D5000704740EA0102AB4B0B331A7070470146F3
:100D60000020A84A0832106820F0030008431060F1
:100D70007047A4480830006800F00C007047014636
:100D80000020A04A0832106820F0F00008431060EC
:100D90007047014600209B4A0832106820F4E0604A
:100DA00008431060704701460020964A08321068D8
:100DB00020F4605040EAC10010607047F0B5002197
:100DC000002200230026002400258E4F08373F68AC
:100DD00007F00C0131B1042912D0082913D00C29D5
:100DE00037D113E0874F3F1D3F68C7F342356F1C73
:100DF0004FF0010C0CFA07FC4FEACC37076036E0E5
:100E0000854F076033E0854F076030E07D4F08373E
:100E10003F6807F470127B4F08373F6807F44003C0
:100E20007F4F07EB92473A78012707EB9353754FB3
:100E300008373F6807F480362EB9774F5743B7FB22
:100E4000F3F7076004E0754F5743B7FBF3F707600C
:100E50000DE06C4F3F1D3F68C7F342356F1C4FF0EC
:100E6000010C0CFA07FC4FEACC37076000BF00BF4B
:100E7000644F08373F6807F0F0010909694F7C5C4F
:100E80000768E74047605F4F08373F6807F4E06155
:100E9000090A644F7C5C4768E7408760594F083710
:100EA0003F6807F46051C90A5E4F7C5C4768E740C1
:100EB000C760F0BD002100F44032B2F5403F08D1D8
:100EC000504A116821F0C04100F0C04211434D4A20
:100ED00011604C4A3432126822F44032494B3433A8
:100EE0001A601A46126800F440331A43454B3433F3
:100EF0001A607047474958310860704745495C316E
:100F00000860704739B13F4A1C32126802433D4BBA
:100F10001C331A6006E03B4A1C3212688243394B8C
:100F20001C331A60704739B1364A203212680243C6
:100F3000344B20331A6006E0324A20321268824372
:100F4000304B20331A60704739B12E4A2432126870
:100F500002432C4B24331A6006E02A4A24321268DA
:100F60008243284B24331A60704739B1254A103226
:100F700012680243234B10331A6006E0214A1032F4
:100F8000126882431F4B10331A60704739B11D4AF3
:100F90001432126802431B4B14331A6006E0194ADC
:100FA000143212688243174B14331A60704739B1F8
:100FB000144A183212680243124B18331A6006E0C2
:100FC000104A1832126882430E4B18331A60704769
:100FD00039B10C4A2832126802430A4B28331A608E
:100FE00006E0084A283212688243064B28331A600A
:100FF0007047C9B1034A2C3212680243014B2C33AB
:101000001A6016E0003802400CC0FF88FEFFFEEEBA
:1010100000004742800647420024F40000127A0094
:1010200050620020596200201F4A126882431E4B02
:101030001A60704739B11C4A121D126802431A4BDC
:101040001B1D1A6006E0184A121D12688243164BD7
:101050001B1D1A60704739B1134A1F3A12780243B8
:10106000114B1F3B1A7006E00F4A1F3A1278824359
:101070000D4B1F3B1A7070470B480830006840F05A
:101080008070094908310860704701460020064A0F
:10109000203A12680A400AB1012000E0002070479F
:1010A00001491E39087070472C38024008B50022EB
:1010B000009200200021CA22F94B1A6053221A60C4
:1010C000F74A183A126822F0A002F54B183B1A6052
:1010D00000BFF34A183A126802F02001009A521C2D
:1010E0000092009AB2F5004F01D00029F1D0EC4AED
:1010F000183A126802F020020AB1012000E0002034
:10110000FF22E74B1A6008BD08B5002200920020BC
:101110000021E34A183A126802F04002E2B9421E86
:10112000DF4B183B1A6000BFDD4A183A126802F024
:101130004001009A521C0092009AB2F5005F01D063
:101140000029F1D0D64A183A126802F040020AB1DA
:10115000012002E0002000E0012008BD38B5002099
:10116000009000240025CA20CD4908605320086063
:10117000FFF7CAFF00B952E00020C94924390860CE
:1011800042F20110091D0860081D006800F0070008
:10119000091D086000BFC2481838006800F0040448
:1011A0000098401C00900098B0F5005F01D0002C22
:1011B000F1D0BB481838006800F0040008B90025D9
:1011C0002DE0B7481C3800680020B5491C3908607C
:1011D0004FF6FF70B24910390860B248091F086025
:1011E0000020AF490C390860091D0860091D08601E
:1011F000AB4908310860AA4918310860A849203174
:101200000860091D0860A64918390860A4491C3106
:101210000860FFF74BFF08B9002500E00125FF201B
:101220009F490860284638BD9D481838006820F05E
:1012300080009B4918390860704730B50446002586
:10124000CA209749086053200860FFF75DFF00B986
:101250001DE093481C38006820F0400090491C397C
:10126000086008460068216808438D491C390860F9
:101270008B491439A068086008460068A18840EAD4
:101280000140874914390860FFF7CEFF0125FF2090
:1012900083490860284630BD002101607F214160FC
:1012A000FF218160704718B1FF217D4A116004E081
:1012B000CA217B4A116053211160704730B5044642
:1012C0000025CA207649086053200860FFF71CFFFC
:1012D00000B914E044B172481C38006840F01000B6
:1012E0006F491C39086007E06D481C38006820F021
:1012F00010006B491C390860FFF796FF0125FF209D
:1013000067490860284630BDCA21654A11605321EB
:10131000116040B162491C39096841F02001604AFE
:101320001C3A116007E05E491C39096801F0DF01D1
:101330005B4A1C3A1160FF21594A1160704701460F
:10134000002204E0501CC2B2A1F10A00C1B20A2975
:10135000F8DA100741EA10607047014600BF08093B
:1013600000EB8000420001F00F001044C0B2704753
:101370002DE9F04105460C460026002755B948489E
:101380001C38006800F0400000B102E00020E0706E
:1013900000BF0EE042481C38006800F0400020B159
:1013A0002078FFF7DAFF064602E00020E07000BF79
:1013B00000BF55B120780004617840EA0120A1788F
:1013C0000843E17840EA014611E02078FFF7B7FFD3
:1013D0004FEA00486078FFF7B2FF48EA0028A0789B
:1013E000FFF7ADFF48EA0008E07848EA0046CA2067
:1013F0002B49086053200860FFF786FE08B90027D4
:1014000014E029483040264924390860FFF70CFFD2
:1014100023481C38006800F0200030B9FFF746FE72
:1014200008B9002702E0012700E00127FF201C493E
:1014300008603846BDE8F0810021C170017041703C
:101440008170704770B506460C4600251448243854
:101450000068154900EA0105C5F305402070C5F391
:101460000620607005F07F00A07005F48000000C7D
:10147000E0705EB92078FFF770FF20706078FFF7AA
:101480006CFF6070A078FFF768FFA07070BD00204F
:101490000349091D0868024920390968704700009E
:1014A00024280040FF007F007F7F7F002DE9F0416E
:1014B00005460C46002600274DB9607800F0100064
:1014C000102804D1607820F010000A30607005B94F
:1014D00008E06078FFF741FF0646A078FFF73DFF80
:1014E000064600BF55B1E0780004617840EA01206B
:1014F000A1780843217840EA413611E0E078FFF70F
:101500001EFF4FEA00486078FFF719FF48EA0028FD
:10151000A078FFF714FF48EA0008207848EA403630
:10152000CA20FE49086053200860FFF7EDFD08B9A6
:10153000002714E0FA483040F84920390860FFF7E6
:1015400073FEF6481C38006800F0200030B9FFF741
:10155000ADFD08B9002702E0012700E00127FF20C8
:10156000EE4908603846BDE8F081012101708170C4
:1015700041700021C170704770B506460C460025C9
:10158000E64820380068E64900EA0105280CE070CA
:10159000C5F30420607005F03F00A070C5F3423031
:1015A00020705EB9E078FFF7D8FEE0706078FFF752
:1015B000D4FE6070A078FFF7D0FEA07070BD2DE95A
:1015C000F04105460E46144600276DB9D3481C3835
:1015D000006800F0400000B102E00020E07000BFB1
:1015E000A06800B91AE019E0CC481C38006800F087
:1015F000400020B12078FFF7B0FE074602E000204F
:10160000E07000BFA06820B9207BFFF7A6FE074668
:1016100004E0207BFFF7A1FE074600BF95B12078CC
:101620000004617840EA0120A1780843E17840EAAB
:101630000140217B40EA0160A1680843616840EAFB
:1016400001071BE02078FFF77AFE4FEA0048607838
:10165000FFF775FE48EA0028A078FFF770FE48EA19
:101660000008E07848EA0048207BFFF768FE48EA77
:101670000060A1680843616840EA0107CA20A749E1
:10168000086053200860B6F5807F03D1A34808386E
:10169000076002E0A148001F0760FF209F49086023
:1016A000BDE8F0810021C1700170417081708160DE
:1016B000012101730021416070472DE9F041064688
:1016C0000F4614460025B7F5807F03D193480838AC
:1016D000056802E09148001F0568C5F305402070C9
:1016E000C5F30620607005F07F00A07005F480004F
:1016F000000CE070C5F30560207305F08040A06029
:1017000005F0803060607EB92078FFF726FE2070FB
:101710006078FFF722FE6070A078FFF71EFEA070D1
:10172000207BFFF71AFE2073BDE8F08138B5024632
:101730000024009400230020CA24784D2C605324F8
:101740002C6041B1754C1C3C24681443734D1C3D06
:101750002C6001201EE0714C1C3C246894436F4DAA
:101760001C3D2C6000BF6D4C183C246804EA122319
:10177000009C641C0094009CB4F5005F01D0002B19
:10178000F1D0664C183C246804EA12240CB90020FD
:1017900000E00120FF24614D2C6038BD30B50023EE
:1017A000CA245E4D2C6053242C6041EA0203B0F53C
:1017B000807F03D1594C2034236002E0574C2434FD
:1017C0002360FF24554D2C6030BD01460020B1F54B
:1017D000807F05D1514A20321268C2F30E0004E026
:1017E0004E4A24321268C2F30E007047CA214B4A97
:1017F00011605321116049491C39096821F0070122
:10180000464A1C3A11601146096801431160FF21E4
:10181000424A11607047CA21404A11605321116049
:101820003E4910390860FF21116070473B4810386D
:10183000006880B2704718B501460023009300226B
:101840000020CA23354C23605323236049B1334B16
:101850001C3B1B6843F48063304C1C3C236001201C
:101860001FE02E4B1C3B1B6823F480632B4C1C3C5D
:10187000236000BF294B183B1B6803F00402009B48
:101880005B1C0093009BB3F5005F01D0002AF1D0F0
:10189000224B183B1B6803F004030BB9002000E047
:1018A0000120FF231D4C236018BDCA221B4B1A6068
:1018B00053221A60194A1C3A126822F48022174BEC
:1018C0001C3B1A601A46126840EA01031A43134B84
:1018D0001C3B1A60FF22114B1A6070470F481C38DE
:1018E000006800F480207047CA220C4B1A60532213
:1018F0001A600A4A1C3A126822F4E002074B1C3BA9
:101900001A601A46126840EA01031A43034B1C3B53
:101910001A60FF22014B1A60704700002428004023
:101920003FFFFF0070B504460D460026CA20FE4961
:10193000086053200860FFF7E7FB00B907E044EABE
:101940000500F9490C390860FFF76EFC0126FF20FD
:10195000F5490860304670BD30B504460025CA2000
:10196000F149086053200860FFF7CEFB00B914E08E
:1019700044B1ED481C38006840F08000EA491C3949
:10198000086007E0E8481C38006820F08000E6495D
:101990001C390860FFF748FC0125FF20E249086078
:1019A000284630BDCA21E04A11605321116040B180
:1019B000DD491C39096841F40001DB4A1C3A116019
:1019C00007E0D9491C39096821F40001D64A1C3ABC
:1019D0001160FF21D44A11607047CA21D24A1160B8
:1019E00053211160D0491C39096821F40021CE4AE5
:1019F0001C3A11601146096801431160FF21CA4A6F
:101A00001160704770B5034600200024CA25C64EF9
:101A1000356053253560C44D183D2D6805F480357B
:101A200055B100E0641CC04D183D2D6805F48035AB
:101A300015B1B4F5805FF5D1BB4D183D2D6805F4A7
:101A400080353DB943EA01051543B74E1836356078
:101A5000012000E00020FF25B34E356070BD10B5B9
:101A60000A460021B04B1C3B1B6840F6080423EAE1
:101A700004011AB140F40063194300E00143CA2392
:101A8000A94C236053232360A74B1C3B1960FF2301
:101A9000236010BD2DE9F04180460C461546002616
:101AA0000027A1480C300068A04900EA01069E48C2
:101AB000103000689E4900EA0107C6F30540207017
:101AC000C6F30620607006F07F00A07006F4800068
:101AD000000CE0700020E870C7F30420687007F085
:101AE0003F00A870C7F342302870B8F1000F17D13B
:101AF0002078FFF732FC20706078FFF72EFC6070D2
:101B0000A078FFF72AFCA0706878FFF726FC6870C1
:101B1000A878FFF722FCA8702878FFF71EFC287031
:101B2000BDE8F081804814300068704741B97E4AB2
:101B30001C32126822EA40027B4B1C331A6007E019
:101B4000794A1C32126842EA4002774B1C331A6011
:101B5000704739B1744A1C3212680243724B1C330D
:101B60001A6006E0704A1C32126882436E4B1C33C6
:101B70001A6070476C491C31096821F4C0516A4AE7
:101B80001C321160114609680143116070476649B3
:101B90001C31096821F4E061634A1C32116011466E
:101BA00009680143116070475F491C31096821F4DD
:101BB000C0415D4A1C321160114609680143116041
:101BC000704740B158491C31096841F08001564ABC
:101BD0001C32116007E054491C31096821F0800172
:101BE000514A1C321160704740B14F491C3109689D
:101BF00021F400414C4A1C32116007E04A491C3173
:101C0000096841F40041484A1C321160704708B528
:101C100000220092444A2C320092009A02EB800289
:101C20000092009A116008BD08B50146002000909E
:101C30003D482C300090009800EB81000090009807
:101C4000006808BD38491C31096821F48021364AF2
:101C50001C32116011460968014311607047F0B5EC
:101C600004460D4600270026CA202F49086053204D
:101C700008602D481838006800F0080050B100E0F6
:101C8000761C29481838006800F0080010B1B6F535
:101C9000005FF5D124481838006800F0080098B9B2
:101CA00021481C38006800F0100058B945EA0400CB
:101CB0001D4908310860FFF7F9F908B9002704E069
:101CC000012702E0002700E00027FF2016490860F6
:101CD0003846F0BDCA22144B1A6053221A6091B1E3
:101CE000114A1C3A126820F004031A430E4B1C3BA5
:101CF0001A600D4A1C32126800F004031A430A4BA2
:101D00001C331A6018E0084A1C3A126820F00403D9
:101D10009A43054B1C3B1A60034A1C32126800F0C0
:101D200004039A43004B05E0242800407F7F7F0096
:101D30003FFFFF001C331A60FF222A4B1A607047D6
:101D400010B5014600200022264B183B1B68264C8C
:101D500003EA040202EA01030BB1012000E00020C3
:101D600010BDC0F3100141F080011E4A183A1268FC
:101D700002F0800262EA01011A4A183A11607047C3
:101D800030B50146002000220023164C1C34246884
:101D900004F00402134C1C3C24680C408D0C21FA06
:101DA00005F502EAD53544EA05030E4C183C2468D3
:101DB00004EA11121BB194B20CB1012000E0002022
:101DC00030BD002101098AB242F08002054B183B68
:101DD0001B6803F0800363EA0202024B183B1A609F
:101DE00070470000242800407FFF010010B5044622
:101DF000BA48844208D101218014FFF7C7F80021B6
:101E0000A014FFF7C3F816E0B548844208D10121B9
:101E10000014FFF7CCF800212014FFF7C8F80AE0FF
:101E2000B048844207D10121C013FFF7C0F8002158
:101E3000E013FFF7BCF810BD10B50022028802F4D1
:101E400041520B884C8823438C882343CC882343FE
:101E50000C8923434C8923438C892343CC89234316
:101E60001A430280838B4FF2FF74234083830B8AD3
:101E7000038210BD2DE9FF5F05460C464FF00009B7
:101E800002274FF000084FF0010B0026B246A88B46
:101E90004FF240010840A88302202884B5F81C9026
:101EA000A068022801D100BF33E0A08810B94FF02C
:101EB000010B01E04FF0020B6846FEF77FFFDDF8F3
:101EC00000A0E088B0F5007F0AD14FEA1A2000EBAD
:101ED00080004000A168B0FBF1F0401D86B20BE02D
:101EE0004FEA4B10BAFBF0F000EB80004000A16815
:101EF000B0FBF1F0401D86B20A20B6FBF0F606F00A
:101F00000108A6EB0800C0F34F074FF6FF7000EA88
:101F10000828022F01DBFF2F02DD02274FF0000807
:101F2000E08840EA080038432884A088A189084353
:101F3000618808432188084340F4006040EA0909A9
:101F4000A5F81C90BDE8FF9F0021018041808180A1
:101F5000C180018141818181C18107210182704756
:101F60000021018041808180C180022181600021A7
:101F70008181704721B1028842F04002028004E072
:101F800002884FF6BF731A400280704721B1828BDE
:101F900042F48062828304E0828B4FF6FF331A4062
:101FA0008283704702884FF2FF731A4002800288D2
:101FB0000A4302807047B1F5804F04D1028842F491
:101FC0008042028004E002884BF6FF731A400280D0
:101FD00070474FF6FF62914204D0028842F480724B
:101FE000028004E002884FF6FF631A4002807047C7
:101FF00021B1828842F00402828004E082884FF698
:10200000FB731A408280704701468889704781813E
:10201000704721B1028842F40052028004E0028835
:102020004DF6FF731A4002807047018841F48051D9
:102030000180704702460020012901D0108B00E08A
:10204000908A70470146088A70471AB183880B430B
:10205000838002E083888B438380704730B50024FF
:1020600000230C110125A540ABB21AB185881D4390
:10207000858002E085889D43858030BD0246002032
:1020800013890B400BB1012000E000207047CA43C8
:1020900002817047F0B5024600200024002300258D
:1020A00001F00F070126BE40B4B20B1101269E407D
:1020B000B3B2968806EA03051689264016B10DB11B
:1020C000012000E00020F0BD10B5002201F00F0457
:1020D0000123A3409AB2D343038110BD00300140D5
:1020E00000380040003C004010B501210846FEF7D2
:1020F0004DFF00210120FEF749FF10BD0020B2492D
:102100000860091D0860091D0860091D0860091D97
:102110000860091D0860091D08607047AB49086028
:102120007047AA48006800F44070704730B1A74972
:10213000496841F00101A54A516005E0A349496899
:1021400021F00101A14A5160704730B500228B0790
:102150001C0F0F2303FA04F29C4B08338C1053F826
:1021600024309343994C08348D1044F8253023468D
:102170008C1053F824308C07240F00FA04F4234306
:10218000924C08348D1044F8253030BD01460020B3
:102190008D4A106820F440300843106070470246B2
:1021A0000020894B1868104302F48023B3F5802F78
:1021B00002D120F00F00084302F40023B3F5002FF2
:1021C00003D120F0F00040EA011002F48013B3F5CF
:1021D000801F03D120F4706040EA012002F4001354
:1021E000B3F5001F03D120F4704040EA0130764B74
:1021F0001860704739B1744A121F12680243724B5B
:102200001B1F1A6006E0704A121F126882436E4B51
:102210001B1F1A60704739B16B4A121F1268824344
:10222000694B1B1F1A6006E0674A121F12680243BF
:10223000654B1B1F1A60704710B50022C20F20F0BB
:10224000004081B13AB1604B1B1D1B6803435E4CDB
:10225000241D236017E05C4B08331B6803435A4C72
:10226000083423600FE03AB1574B1B1D1B688343B2
:10227000554C241D236006E0534B08331B688343F1
:10228000514C0834236010BD40B14F49091D096805
:1022900041F000414C4A121D116007E04A49091DF6
:1022A000096821F00041484A121D1160704710B5BD
:1022B000012810D13AB1444B0C331B688B43424C7C
:1022C0000C3423607FE0404B0C331B680B433E4CC7
:1022D0000C34236077E0022813D14AB13A4B0C3317
:1022E0001B68CC4303EA0443374C0C3423606AE098
:1022F000354B0C331B6843EA0143334C0C342360E9
:1023000061E0032810D13AB12F4B10331B688B4387
:102310002D4C1034236056E02B4B10331B680B43BD
:10232000294C103423604EE0042813D14AB1264BC7
:1023300010331B68CC4303EA0443234C103423605E
:1023400041E0214B10331B6843EA01431E4C10341B
:10235000236038E0052810D13AB11B4B14331B68B9
:102360008B43194C143423602DE0174B14331B6836
:102370000B43154C1434236025E0062813D14AB1D1
:10238000114B14331B68CC4303EA04430E4C143442
:10239000236018E00C4B14331B6843EA01430A4CDA
:1023A000143423600FE03AB1074B18331B688B439A
:1023B000054C1834236006E0034B18331B680B43AD
:1023C000014C1834236010BD047C00400000014023
:1023D00010B50446B4F1804F08D101210846FEF73C
:1023E000E6FD00210120FEF7E2FD5EE0FB488442AD
:1023F00008D101210220FEF7DAFD00210220FEF7BC
:10240000D6FD52E0F648844208D101210420FEF7AF
:10241000CEFD00210420FEF7CAFD46E0F1488442CB
:1024200008D101210820FEF7C2FD00210820FEF797
:10243000BEFD3AE0EC48844208D101211020FEF7AD
:10244000B6FD00211020FEF7B2FD2EE0E7488442E1
:1024500008D101212020FEF7AAFD00212020FEF74F
:10246000A6FD22E0E248844208D101210420FEF7C3
:102470008DFD00210420FEF789FD16E0DD48844231
:1024800008D101210820FEF781FD00210820FEF778
:102490007DFD0AE0D848844207D101211020FEF7D3
:1024A00075FD00211020FEF771FD10BD002202888D
:1024B000B0F1804F08D0C94B984205D0C84B984224
:1024C00002D0C84B984204D14FF68F731A404B8804
:1024D0001A43C54B984207D0C44B984204D04FF6DC
:1024E000FF431A400B891A4302804B68C3620B8872
:1024F00003850123838270474FF0FF314160002143
:1025000001800181418070470185828270470A46BF
:10251000002101884FF68F731940114301807047E5
:1025200041627047C16270470146486A7047014680
:10253000088D704721B1028842F00202028004E057
:1025400002884FF6FD731A400280704721B102885D
:1025500042F00402028004E002884FF6FB731A4046
:102560000280704721B1028842F08002028004E0BC
:1025700002884FF67F731A400280704702884FF638
:10258000F7731A40028002880A430280704702886B
:102590004FF6FF431A40028002880A4302807047C8
:1025A00021B1028842F00102028004E002884FF665
:1025B000FE731A400280704730B500230022048C5D
:1025C0004FF6FE752C400484028C038B4FF68F74FB
:1025D0002340AC1E23400C8823436C1E22400C89F0
:1025E00022434C8822434C6844630383028430BDF9
:1025F00030B500230022048C4FF6EF752C40048484
:10260000028C038B48F6FF7423400C884FF6FF754D
:1026100005EA042423434FF6DF7422400C8905EABF
:10262000041422434C8805EA041422434C68846352
:102630000383028430BD30B500230022048C4FF6A2
:10264000FF652C400484028C838B4FF68F742340EB
:102650000C8823434FF6FF5422400C894FF6FF7538
:1026600005EA042422434C8805EA042422434C68EA
:10267000C4638383028430BD30B500230022048C00
:102680004EF6FF752C400484028C838B48F6FF7451
:1026900023400C884FF6FF7505EA042423434DF6CA
:1026A000FF7422400C8905EA043422434C8805EA71
:1026B000043422434C6804648383028430BD0021C7
:1026C0000180418041600181704770B50346002060
:1026D00000241846183001258D40ACB21D8CA5434E
:1026E0001D8409B1082909D100EB6100056825F0B6
:1026F000700505600568154305600EE00D1FC5F304
:102700004E052844056825F4E045056005684FF648
:10271000FF7606EA02263543056070BD41637047C7
:1027200081637047C1637047016470470A460021A6
:10273000018B4FF68F7319401143018370470A468E
:102740000021018B48F6FF7319404FF6FF7303EA2F
:1027500002231943018370470A460021818B4FF6FB
:102760008F7319401143818370470A460021818B82
:1027700048F6FF7319404FF6FF7303EA022319432B
:10278000818370470A460021018B4FF6F773194089
:102790001143018370470A460021018B4FF2FF73FA
:1027A00019404FF6FF7303EA022319430183704770
:1027B0000A460021818B4FF6F7731940114381833C
:1027C00070470A460021818B4FF2FF7319404FF684
:1027D000FF7303EA0223194381837047000400401A
:1027E00000080040000C00400010004000140040B1
:1027F00000080140000C0140001001400A46002181
:10280000018B4FF6FB7319401143018370470A4651
:102810000021018B4FF6FF3319404FF6FF7303EA97
:1028200002231943018370470A460021818B4FF62A
:10283000FB7319401143818370470A460021818B45
:102840004FF6FF3319404FF6FF7303EA0223194393
:10285000818370470A460021018B4FF67F73194030
:102860001143018370470A460021018BC1F30E0119
:102870004FF6FF7303EA02231943018370470A46A8
:102880000021818B4FF67F7319401143818370477C
:102890000A460021818BC1F30E014FF6FF7303EA54
:1028A00002231943818370470A460021018C4FF6A9
:1028B000FD7319401143018470470A460021018CC1
:1028C0004FF6DF7319404FF6FF7303EA0213194303
:1028D000018470470A460021018C4FF6FF531940CE
:1028E0004FF6FF7303EA02231943018470470A4637
:1028F0000021018C4DF6FF7319404FF6FF7303EA78
:10290000023319430184704702894FF6F7731A4066
:10291000028102890A430281704730B500230124F5
:102920008C40A3B2048C9C430484048C02FA01F50D
:10293000ADB22C43048430BD828B4FF2FF331A407A
:102940008283828B4FF6FF7303EA01231A4382834B
:102950007047F0B50C461546002100220026078C72
:102960004EF6FF7C07EA0C070784818B028C4FF63A
:10297000FF7707EA043640F6FF4739404FF6FF7706
:1029800007EA052739434FF6FF7707EA033739434C
:1029900045F6FF773A4046F480573A4381830284F4
:1029A000F0BD828B4FF6F3731A408283828B0A4309
:1029B00082837047F0B50C461546002100220026A0
:1029C000078C4FF6FF6C07EA0C070784818B028C9B
:1029D0004FF6FF7707EA04264FF60C7739404FF69B
:1029E000FF7707EA03172F4339434FF2FF573A4067
:1029F00046F480773A4381830284F0BD028B4FF224
:102A0000FF331A400283028B4FF6FF7303EA012360
:102A10001A4302837047F0B50C4615460021002288
:102A20000026078C4FF6EF7C07EA0C070784018B22
:102A3000028C4FF6FF7707EA041640F6FF4739404D
:102A40004FF6FF7707EA033739434FF6FF7707EA78
:102A5000052739434FF65F773A4046F010073A436F
:102A600001830284F0BD028B4FF6F3731A40028398
:102A7000028B0A4302837047F0B50C4615460021CD
:102A80000022068C4FF6FE773E400684018B028CB6
:102A90004FF60C7631407E1C06EA03162E43314376
:102AA0004FF6F576324044F001063243018302844A
:102AB000F0BD70B505460C46208850B92389A28820
:102AC00061882846FFF7D8FFE1882846FFF7CBFF4B
:102AD00025E0208804280AD12389A2886188284615
:102AE000FFF799FFE1882846FFF788FF17E0208865
:102AF00008280AD12389A28861882846FFF75AFF4F
:102B0000E1882846FFF74DFF09E02389A288618804
:102B10002846FFF71EFFE1882846FFF70DFF70BD2E
:102B2000002101804180012181800021C18001813B
:102B300070472DE9F04105460C46002601276088C4
:102B400008B9022600E00026A088012801D102274A
:102B500000E001272088A0B92389A288618828463F
:102B6000FFF78AFFE1882846FFF77DFF23893A4671
:102B700031462846FFF74FFFE1882846FFF73EFF22
:102B800013E02389A28861882846FFF744FFE18883
:102B90002846FFF733FF23893A4631462846FFF798
:102BA0006BFFE1882846FFF75EFFBDE8F081014634
:102BB000486B70470146886B70470146C86B704789
:102BC0000146086C70471AB183890B43838102E088
:102BD00083898B438381704781827047024600203E
:102BE000138A0B400BB1012000E000207047CA435C
:102BF0000282704730B50246002000230024158A67
:102C000005EA0103958905EA010413B10CB101201D
:102C100000E0002030BDCA430282704741EA02034F
:102C2000A0F8483070471AB183890B43838102E0D2
:102C300083898B438381704721B1828842F00802E7
:102C4000828004E082884FF6F7731A4082807047D2
:102C500001894FF6F8721140018170470A46002140
:102C600001894FF68F73194011430181704730B5C8
:102C700004460D4629462046FFF7F0FF208940F024
:102C80000700208130BD2DE9F04104460D4616466F
:102C90001F46602D06D13B46012231462046FFF7F4
:102CA000BAFE05E03B46012231462046FFF7E4FE2E
:102CB00029462046FFF7D2FF208940F007002081F7
:102CC000BDE8F08130B50C4600210189C9B24FF64C
:102CD000FF7505EA0325154325432943018130BDCE
:102CE0002DE9F04105460E46174698460024434616
:102CF0003A4631462846FFF7E5FF2C894FF6F87033
:102D0000044044F007044FF68F70044044F0700410
:102D10002C81BDE8F081F0B504460D4616461F46ED
:102D20003B46324629462046FFF7CCFF208940F437
:102D300080402081F0BD82884FF68F731A408280D8
:102D400082880A438280704702894FF6F8731A40DE
:102D5000028102890A430281704702894FF67F731C
:102D60001A40028102890A4302817047F0B50C467D
:102D700015461E460021002200230189028B038C88
:102D80004FF6F877394021434FF6FC473A4040F27E
:102D900001173A434FF6DD773B404FF6FF7707EADE
:102DA00006172F433B43018102830384F0BD21B109
:102DB000828842F08002828004E082884FF67F732E
:102DC0001A408280704730F8502F02EA1142028088
:102DD00002888BB21A4320F85029704710B5044678
:102DE000F748844209D101218803FEF7CFF800217A
:102DF0004FF48040FEF7CAF832E0F248844209D12D
:102E000001214804FEF7D3F800214FF40030FEF70B
:102E1000CEF825E0EC48844209D101218804FEF770
:102E2000C6F800214FF48020FEF7C1F818E0E7480B
:102E3000844209D10121C804FEF7B9F800214FF4FA
:102E40000020FEF7B4F80BE0E148844208D10121EC
:102E50000805FEF7ACF800214FF48010FEF7A7F844
:102E600010BD2DE9FF4705460E460024A14600BFD0
:102E7000A046B08900B100BF2C8A24F44054F088E9
:102E800004432C82AC8941F20C608443B0883189C0
:102E90000843718908430443AC81AC8A24F440742C
:102EA000B0890443AC826846FDF788FFC448854278
:102EB00002D1DDF80C9001E0DDF80890A88900F45B
:102EC000004040B109EBC90000EB0910316849002E
:102ED000B0FBF1F707E009EBC90000EB091031681E
:102EE0008900B0FBF1F76420B7FBF0F00401200982
:102EF000642101FB1078A88900F4004040B1322021
:102F000000EBC800B0FBF1F000F00700044308E05C
:102F1000322000EB08106421B0FBF1F000F00F004C
:102F200004432C81BDE8FF874FF416510160002156
:102F30008180C18001810C21418100218181704704
:102F400010B502460020108A20F470600B884C886F
:102F500023438C882343CC8823431843108210BD1D
:102F60000021018041808180C180704721B1828928
:102F700042F40052828104E082894DF6FF731A40C8
:102F800082817047028B02F47F420283028B0A43E4
:102F90000283704721B1828942F40042828103E0BA
:102FA0008289C2F30E028281704721B1828A42F483
:102FB0000062828204E0828A4FF2FF731A408282AA
:102FC0007047C1F308028280704701468888C0F3C9
:102FD00008007047028A4FF6F0731A400282028A94
:102FE0000A430282704721B1828942F00202828143
:102FF00004E082894FF6FD731A408281704782890E
:103000004FF2FF731A40828182890A43828170479E
:10301000028A4FF6DF731A400282028A0A43028252
:10302000704721B1028A42F48042028204E0028A9F
:103030004BF6FF731A4002827047818941F001010B
:103040008181704721B1828A42F00802828204E0C5
:10305000828A4FF6F7731A4082827047028BD2B28F
:103060000283028B42EA01220283704721B1828AE5
:1030700042F02002828204E0828A4FF6DF731A4017
:103080008282704721B1828A42F01002828204E07B
:10309000828A4FF6EF731A4082827047828A4FF617
:1030A000FB731A408282828A0A438282704721B16E
:1030B000828A42F00202828204E0828A4FF6FD7325
:1030C0001A40828270471AB1838A0B43838202E0DE
:1030D000838A8B4383827047F0B503460024002621
:1030E0000025002040F66A17B94200D100BF1846FB
:1030F000C1F3421401F01F06012707FA06F5012C5F
:1031000001D10C3004E0022C01D1103000E0143069
:103110001AB107682F43076002E00768AF430760F2
:10312000F0BD02460020B1F5007F00D100BF13883A
:103130000B400BB1012000E00020704701F4007249
:10314000B2F5007F00D100BFCA430280704770B55E
:103150000246002400230025002040F66A16B142F2
:1031600000D100BFC1F3421501F01F03012606FA8A
:1031700003F3012D02D19689334006E0022D02D1DE
:10318000168A334001E0968A33400C12012606FA73
:1031900004F41688344013B10CB1012000E0002083
:1031A00070BD10B50022002340F66A14A14200D180
:1031B00000BF0A1201249440A3B2DC43048010BD76
:1031C000003801400044004000480040004C0040EE
:1031D000005000404FF4FA700DF08EF8AAE0FD4860
:1031E00000680DF0EBFE401C38B9FB48007820F079
:1031F0000100401CF849087005E0F748007820F00D
:103200000100F5490870F54800680DF0D7FE401C34
:1032100038B9F148007820F00400001DEE4908702C
:1032200005E0ED48007820F00400EB490870EC4818
:1032300000680DF0C3FE401C38B9E748007820F064
:1032400008000830E449087005E0E348007820F001
:103250000800E1490870E0480078C0F3C003DE4888
:10326000007800F00102DC480078C0F38001DDA0A6
:1032700004F017FF4FF40051DD48FDF7C9FB08B912
:10328000012000E00020DB49097881F001010840BD
:10329000D1490978D04A1278C2F380021140CE4A4F
:1032A0001278C2F3C0021140D24A1278C2F38002EF
:1032B00082F0010211400840002838D0CE4890F832
:1032C0007A00312807D10020FEF7B5FA00214FF42B
:1032D0008070FEF72BFAC14800680DF06FFE0446BF
:1032E0002146C6A004F0DDFEBA4800680DF066FE77
:1032F00004462146C7A004F0D4FE4FF40050FDF769
:10330000BDFA4FF48040FEF75CFD4FF48010FDF7EE
:10331000B5FA4FF40050FEF754FD4FF48050FEF71D
:1033200050FD4FF40030FDF7A9FAFDF74AFC3220BA
:103330000CF0E2FF53E7F2B000200A900B900C90E3
:103340000D900690079008900990F0E01021B64883
:10335000FDF776FB4FF47A700CF0CEFFB34800789F
:1033600020F040004030B14908700AA906A803F0D7
:1033700014FBAE480078C0F38000C0B94FF0FF31B5
:10338000AB4800680DF0B2FDAA49AB4803F005FB5D
:103390000AF080FB01F02BFC01219548FDF750FB62
:1033A0000BF0B6FF01F02FFC0BF061FC05E04FF0D5
:1033B000FF319F4800680DF099FD0AAA9FA19D4822
:1033C0000EF050FC06AA9DA19B480EF04BFC05F0A8
:1033D000E5FD9648007800F0010040B94FF0FF315C
:1033E000974800680DF082FD09F0CCFA05E04FF037
:1033F000FF31934800680DF079FD924800680CF0A9
:103400009FFF00F0200000283BD040218D4800683D
:103410000CF0C0FF8CA004F044FE42F210730122B5
:103420008021884800680CF0DBFF8CA004F039FE96
:1034300004AA05A98FA005F004FE8F480CF054F9EA
:1034400004468E48C078DDE90412CDE901210090E0
:103450008A490B784A798849081989A10EF002FC3B
:1034600005F036FB8BA004F01CFE40217548006877
:103470000CF054FF4FF48071724800680CF08AFF22
:1034800023E040216F4800680CF084FF04AA05A9DE
:1034900078A005F0D6FD78480CF026F90446774868
:1034A000C078DDE90412CDE90121009073490B7861
:1034B0004A797149081972A10EF0D4FB05F008FB96
:1034C0004021604800680CF029FF6B480CF00CF9B3
:1034D000851C69482B4674A275A100900EA80EF0B9
:1034E000C1FB4FF0FF31754800680DF05BF80EA886
:1034F0000CF0FAF8054600232A460EA9184609F0F2
:10350000BBFF6E4800680DF071F84D4800680DF083
:1035100029FD474800680DF025FD4448007820F05B
:10352000400042490870664800680DF06BFD0DE7E9
:1035300000252DE14FF0FF313D4800680DF0D6FC2D
:103540000CF070FF5F4908603848007820F00400F4
:10355000001D364908703749374803F01EFA0AF053
:1035600099FA01F044FB01212148FDF769FA0BF0BB
:10357000CFFE01F048FB0BF07AFB05F00FFD314860
:1035800000680CF0DDFE00F02000002821D0402172
:103590002C4800680CF0FEFE4BA004F082FD42F2C5
:1035A000107301228021274800680CF019FF4AA0FF
:1035B00004F077FD04F029FF4CA004F072FD4021D7
:1035C000204800680CF0AAFE4FF480711D48006886
:1035D00094E096E08C6200207862002098620020DF
:1035E0008862002025642C25642C25640D0A0000C7
:1035F00000080240026300206E65002050726F6375
:10360000736565315F7374617475733A25640D0A6F
:1036100000000000424332355F7374617475733A81
:1036200025640D0A000000000000024071620020C5
:10363000A4620020EC630020FB63002025730000DF
:10364000A8620020AC6200207465737420737472E9
:103650006F6520776169740D0A00000074657374EA
:10366000205446206461746120656E747279310D56
:103670000A00000030000000E06D00201B63002005
:103680002C25642C25642C25642C256C642C256C3D
:103690006400000074657374207374726F65206633
:1036A000696E6973680D0A005075622C0000000095
:1036B000257325642C25732C2A000000B862002095
:1036C000A0620020806200207374726F65207761B1
:1036D00069740D0A00000000544620646174612082
:1036E000656E747279310D0A000000007374726F98
:1036F000652066696E6973680D0A00000CF04AFE69
:1037000011E0F9A004F0CDFC4021FC4800680CF069
:1037100041FE04F07AFE4021F84800680CF0FEFDFE
:10372000F7A004F0BEFCFAA004F0BBFCFE48006861
:103730000DF018FCFD48007820F00400FB490870EB
:10374000FB4800680DF05EFCFAA004F0AAFCF84803
:1037500000680DF057FC04460AE02146FCA004F086
:10376000A0FCF34800680DF04DFC0446681CC5B28F
:103770000CB1012000E000200A2D01DA012100E057
:10378000002108400028E8D14FF47A700CF0B4FD15
:10379000D0E60024F44B01225102D84800680CF016
:1037A0001FFE41E00220F1490870002500241BE0C3
:1037B0004FF0FF31EE4800680CF0F4FE09F099FE7E
:1037C0000546022D06D1002400230B22E9A118464C
:1037D00009F052FEE64800680CF008FF4EF6602043
:1037E0000CF08AFD601CC4B2042CE1DB0020DF4930
:1037F000087008460078022812D00821BF480068E7
:103800000CF0C8FD4FF40071BC4800680CF086FD58
:10381000DB4800680DF0F6FBDA4800680DF0F2FBBB
:1038200005200CF069FD00BFBCE72AE0B348006842
:103830000CF086FD00F40070A0B9D34A02F10A0131
:10384000A1F11E000AF088F80121D048FDF7F8F830
:103850001021CF48FDF7F4F84FF40071A748006835
:103860000CF098FD4FF0FF31C14800680CF09AFE53
:1038700003F065FEBE4800680CF0B8FE14200CF0A2
:103880003BFDD3E700240025C1E04FF0FF31C148E4
:1038900000680DF02BFB0CF0C5FDBF490860A34884
:1038A000007820F00100401CA04908700020BB49AE
:1038B0000871BBA004F0F5FB002412E009F062F8E7
:1038C000B648C078012808D1062409F057F9AE4956
:1038D0001E39A1F1140009F092F9601CC4B2601CF9
:1038E000C4B2052CEADB02F0F7F8B1A00EF0AAF999
:1038F0004FF4FA7000F0A5FDB149B2A004F0D1FB7D
:1039000020217E4800680CF045FD7C4800680CF0E2
:1039100017FD00F0400018B140F6B8300CF0ECFC98
:103920009E48C078012839D10024002508E0601C99
:10393000C4B2052000F085FDA4A005F021F90546DC
:103940001E2D01D8012000E00020322C01DA0121D7
:1039500000E0002108400028E9D11E2D1BD929468E
:103960009CA004F09EFB2A46002198A005F033F9A4
:1039700000240EE04FF47A700CF0BEFC9AA190483F
:103980000BF096FE18B102F0AFF902F0A5F8601C3A
:10399000C4B20A2CEEDB95A004F083FB202157482B
:1039A00000680CF0BBFC08F0E7FF6048007820F0EE
:1039B00001005E49087093A004F073FB0024754871
:1039C00000680DF0CFFA954800680DF01BFB064625
:1039D00093A004F066FB0AE031469CA004F061FB72
:1039E0008E4800680DF00EFB0646601CC4B20EB196
:1039F000012000E000200A2C01DA012100E0002172
:103A000008400028E8D14FF4FA700CF075FC3CE750
:103A100065E29448007800F0010000282FD0434868
:103A2000007800F0010190A004F03BFB7B480068A7
:103A30000DF0C4FA0446214691A004F032FB601C4C
:103A400020B13A48007800F0010050B992A004F08B
:103A500028FB974A0021AFF2D3100DF0C1FA6F494D
:103A6000086094A004F01DFB7E48007820F001005F
:103A70007C49087002F00BF8064603F0BFF879485D
:103A80000078C0F34000E8B1294800680DF096FACC
:103A9000044621468BA004F004FB601C50B990A0A2
:103AA00004F0FFFA954A0021AFF27B500DF098FA2E
:103AB0001F4908606B48007820F0020069490870CF
:103AC00003F016FB67480078C0F38000002809D097
:103AD0008BA004F0E6FA164800680DF06FFA044671
:103AE00021461BE151E100005446206461746120CD
:103AF000656E747279320D0A00000000AC6200201D
:103B0000544620646174612071756974320D0A0035
:103B10005465726D696E6174652050726F63736570
:103B200065310D0A00000000A462002071620020CF
:103B3000986200205465726D696E617465205072E0
:103B40006F6373656531206661696C0D0A00000062
:103B500050524F315F5468726561645F7374617471
:103B600075733A25640D0A00400D03006E62002053
:103B7000B86200204865617274626561742C2A0025
:103B80008862002090620020A065002000080240AA
:103B900000000240A86200207C6200201B6300201D
:103BA000424332355F53746172740D0A00000000A5
:103BB00041542B434750414444523F0D0A000000FA
:103BC000EC65002049503A25730D0A004243323516
:103BD00000000000424332355F7478745F73697A85
:103BE000653A256C640D0A007061720042433235FB
:103BF0002E7478742073656E642066696E697368CC
:103C00000D0A00005465726D696E6174652054611F
:103C1000736B424332350D0A000000008C620020B5
:103C20005465726D696E617465205461736B4243B3
:103C300032352E2E2E2E2E2E2E2E2E2E2E2E2E2E99
:103C40002E206661696C0D0A000000004243323587
:103C50005F5468726561645F7374617475733A254B
:103C6000640D0A00026300205441534B52554E53D9
:103C7000532E424332355F52554E3A25640D0A00A9
:103C80005468726561645F5374617375735F6263D6
:103C900032353A25640D0A00555345525F5461731D
:103CA0006B5F424332352063726561740D0A000018
:103CB00014330208636F6E66696720416C61726D30
:103CC000410D0A0050524F5353315F546872656181
:103CD000645F5374617375733A25640D0A000000C4
:103CE000555345525461736B5F50726F63657373C4
:103CF000312063726561740D0A000000F032020821
:103D0000555345525461736B5F50726F63657373A3
:103D1000312073746172740D0A000000AFF25C0010
:103D200004F0BFF9601C20B1CD480078C0F38000DA
:103D300058B9AFF2540004F0B4F9CA4A0021AFF602
:103D40000F000DF04DF9C8490860C848007820F010
:103D50000400C649087005B9012501F08FFE461E12
:103D6000304602F090FE02F079FEC5EB051100EB43
:103D70008100BF49086008460068BE49884204D9EE
:103D8000BB480068401ABA490860BB480078C82898
:103D90000AD1B648007820F00800B4490870B7A0EE
:103DA00004F07FF901F0AAFDB34800781E2801DB7A
:103DB000012000E00020B5490978084328B3B44841
:103DC00000680DF0FBF80446601C90B9B1A004F047
:103DD00068F9B54A0021AFF2AD500DF001F9B349D1
:103DE0000860B34A0021AFF255600DF0F9F8A84918
:103DF00008609E48007820F008009C490870002068
:103E0000A2490870ABA004F04CF998480078C0F3C0
:103E1000001068B39548007820F0100093490870AE
:103E2000A84890F87A00312808D103F0FBF88C48B4
:103E3000007820F002008A49087019E08A4800687A
:103E40000DF0BCF80446601C38B9864A0021AFF674
:103E50001F100DF0C5F88449086001F00FFE461EE2
:103E6000304602F010FE01F012FE064602F0C6FED9
:103E70007E480078C0F34010A0B17B4800680DF088
:103E80009DF80446601C38B9764A0021AFF65F10F1
:103E90000DF0A6F8744908607448007820F02000FE
:103EA0007249087071480078C0F38010A0B186484C
:103EB00000680DF083F80446601C38B9834A00217D
:103EC000AFF68D300DF08CF87F49086067480078B8
:103ED00020F04000654908700A200CF00DFA98E5C2
:103EE00010B50122774956316E2001F02DFB78483C
:103EF0000CF06AFB7749086077480CF065FB77495E
:103F0000086077480CF060FB76490860764A00212B
:103F1000AFF203500DF064F874490860744A002150
:103F2000AFF64F500DF05CF87249086010BD0026E6
:103F3000FFF7D6FF4FE00CF075FA6F490968441A95
:103F40000CF070FA6D490968451A701CC6B20A2E49
:103F500005DB2A4621466AA004F0A3F80026714832
:103F60000078022801D10024002501F087FD00EB34
:103F70004001C1EBC0106C4901EBC000A04201D26E
:103F8000012000E0002067490978022901D00121C1
:103F900000E00021084008B100F050F801F077FD82
:103FA00000EB4001C1EBC010604901EBC000A8422A
:103FB00001D2012000E000205A490978022901D0ED
:103FC000012100E00021084008B100F037F84FF46B
:103FD0007A700CF091F9AEE755485649086000F048
:103FE00072F900F069FB0CF031FA53480CF0C0F99B
:103FF0005249086052480CF0BBF9524908605248D7
:104000000CF0B6F951490860514A012108460CF0FC
:1040100097FF50490860504A012108460CF090FF74
:104020004E4908604E4A0021AFF2FD000CF0D8FF67
:104030004C4908600CF020FA00BFFEE7BFF34F8F39
:104040003C48001D006800F4E06047490843001D3B
:104050003849091D0860BFF34F8F00BFFEE700001D
:1040600071620020F0320208986200200263002092
:10407000746200208051010003630020574B5550AB
:104080005F50494E5F3130530D0A00007A620020C4
:1040900088620020437265617465205769666920F3
:1040A0005461736B0D0A00003032020890620020E8
:1040B000E8310208574B55505F50494E5F33530D5E
:1040C0000A0000006E650020A0620020783202081D
:1040D00038330208B862002048330208BC6200206E
:1040E00058330208C0620020CC3202089C620020D3
:1040F0005432020884620020806200207C6200202A
:104100006D65615F6964765F69646C313A25640D41
:104110000A7075625F6964765F69646C313A256420
:104120000D0A00006E620020400D030000DD6D00EE
:104130000000010808ED00E09C320208AC6200209B
:10414000AC320208B0620020BC320208B462002027
:1041500068330208A462002078330208A8620020B5
:104160000C320208946200200000FA050CB5002011
:10417000019000908748006840F4803085490860CD
:1041800000BF8448006800F4003000900198401C93
:104190000190009818B90198B0F5A06FF1D17D4851
:1041A000006800F4003010B10120009001E0002010
:1041B00000900098012859D17748006840F0040029
:1041C000754908600846006840F00200086008462B
:1041D000006840F0010008606E482430006840F03C
:1041E00080506C4924310860C8146C49086000BFD5
:1041F0006A48406800F010000028F9D1654808308E
:10420000006864490831086008460068086008468C
:10421000006808600846006820F47D0008600846D1
:10422000006840F49A0008605A48006840F08070C6
:104230005849086000BF5748006800F00070002827
:10424000F9D054480830006820F003005149083183
:1042500008600846006840F00300086000BF4D4851
:104260000830006800F00C000C28F8D10CBD10B527
:104270004848006840F48070464908604548083066
:1042800000684749084043490831086041480068D0
:10429000444908403F4908600846006820F48020EF
:1042A00008603C480830006820F47D003949083136
:1042B00008600020091D0860FFF758FF4FF00060FC
:1042C0003949086010BD70B500220020002100248B
:1042D0000023304D08352D6805F00C0232B1042A58
:1042E00010D0082A12D00C2A39D113E0294D2D1DE7
:1042F0002D68C5F342335D1C0126AE40F5032B4EFD
:10430000356038E02A4D294E356034E0294D274E7E
:10431000356030E01F4D08352D6805F470101D4DD7
:1043200008352D6805F44001234D05EB90452878AC
:10433000012505EB9151174D08352D6805F48034A2
:1043400034B91B4D4543B5FBF1F5184E356005E01A
:10435000184D4543B5FBF1F5144E35600BE00D4D9E
:104360002D1D2D68C5F342335D1C0126AE40F503BB
:104370000E4E356000BF00BF064D08352D68C5F3F1
:1043800003150E4E725D094D2D68D540074E356000
:1043900070BD000000380240003C02400070004048
:1043A0000CC0FF88FEFFFEEE08ED00E0C4620020B6
:1043B0000024F40000127A00C8620020D1620020BC
:1043C000704710E000BFBFF34F8F0B48006800F448
:1043D000E0600A490843001D07490860BFF34F8F9A
:1043E00000BF00BFFEE7EDE700BFFEE700BFFEE74E
:1043F00000BFFEE7704700000CED00E00000FA058A
:104400001A48006840F08070184908600020184978
:1044100048600846006840F001000860704730B509
:10442000134C63680021134C2468134DB4FBF5F45E
:1044300004FB00F202E00E4C6468E11A9142FAD3E8
:1044400030BD10B504464FF47A7104FB01F0FFF75C
:10445000E6FF10BD10B500210246054C636802E07E
:10446000034C6468E11A9142FAD310BDFCED00E000
:10447000001000E0C462002040420F0070B5044606
:104480000D4629462046FEF79CFD00BF40212046F0
:10449000FEF747FE0028F9D070BD70B505460C4602
:1044A00004E021782846FFF7E9FF641C2078002803
:1044B000F7D170BD70B504460D4640217748FEF730
:1044C0003DFEE1B27548FEF77CFD00BF80217348D8
:1044D000FEF727FE0028F9D0204670BD1CB500214C
:1044E0006F48FEF743FD6E48FEF778FC012102207D
:1044F000FCF708FDC020009001208DF8040000208A
:104500008DF8060001208DF8070000208DF80500C9
:1045100069466448FCF71AFA40216248FCF790FAB1
:1045200080216048FCF78CFA1CBD10B588B00446A9
:10453000FFF7D4FF01205C49087001218003FCF7DC
:10454000F2FC01210846FCF7DDFC5548FEF746FC6D
:104550004FF4C060029002208DF80C008DF80D0021
:1045600000208DF80E0001208DF80F0002A94F48A1
:10457000FCF7ECF94FF48060029002A94B48FCF77D
:10458000E5F9072209214948FCF769FA07220A21BF
:104590004648FCF764FA04940020ADF81400ADF826
:1045A0001600ADF81800ADF81C000C20ADF81A008C
:1045B00004A93B48FEF755FC012240F2255138483A
:1045C000FEF78AFD25208DF8040003208DF80500F4
:1045D00000208DF8060001208DF8070001A8FBF7E8
:1045E000C2FD01212E48FEF7C1FC40212C48FEF7F8
:1045F000A5FD08B010BD1CB500212948FEF7B6FC8A
:104600002748FEF7EBFB01210846FCF77BFC4FF443
:10461000C060009001208DF8040000208DF8060095
:1046200001208DF8070000208DF8050069461F481D
:10463000FCF78CF94FF400711C48FCF701FA4FF4B9
:1046400080611A48FCF7FCF91CBD10B516480078CB
:1046500018BB40F225511248FEF779FDE8B1104829
:10466000FEF7B3FCC4B204F07F041148008800F4E4
:10467000004090B90E480088642808DA0C48018888
:104680000088401C0A4A10800A48445405E0084843
:10469000008840F400400649088010BD00440040F6
:1046A00000380140000402406D620020000002401A
:1046B000066300204468002010B5A8B08048006858
:1046C00027900020249025902690219022902390DE
:1046D0004FF44070FBF742FD62B6FFF791FE01F028
:1046E00084FA4FF4165003F021FC02F0AAFB0446B2
:1046F000012227A9BC2000F027FF9DF89C1071A083
:1047000003F0CFFC9DF89C00312828D17248007836
:1047100020F00100704908700846007820F002007F
:1047200008700846007820F00800087008460078F5
:1047300020F0200008700846007820F010001030AB
:1047400008700846007820F004000870002430202B
:104750008DF89C00012227A9BC2000F01EFF02F06A
:10476000D8F900F08DFA10215C48FCF769F94FF494
:10477000165001F0BBF94FF4165000F017FE4FF43D
:10478000E13002F0EFFD00F071F90AF04DFE01207A
:10479000FCF736FA012252498C2000F0D5FE01A820
:1047A00000F093FF7E2201A94E480AF05DFF4EA063
:1047B00003F077FC4A480078012854D001F09EF8B5
:1047C00001220021B42000F04EFF4EA003F069FC4E
:1047D00001A800F07AFF7E2201A942480AF044FFB6
:1047E000404952A003F05DFC3E49143153A003F050
:1047F00058FC3C49323155A003F053FC39493C3157
:1048000058A003F04EFC37491E315CA003F049FC70
:10481000344950315FA003F044FC3249563163A063
:1048200003F03FFC2F495B3164A003F03AFC2D49B3
:10483000613166A003F035FC2A496B3168A003F0B2
:1048400030FC28497A316CA003F02BFC012224496A
:104850008C2000F079FE224801786CA003F021FC46
:104860006FA003F01EFCD4B902F0BFF90AF05AFEA3
:1048700008F0A8FB022273A1AA2000F08EFE08F027
:104880007BF84FF4FA70FFF7DCFD21A924A802F0B1
:1048900084F824AA21A96CA003F003FC01E001F034
:1048A000E3FF21466CA003F0FCFB21A924A802F041
:1048B00074F824AA21A964A003F0F3FB28B010BD6A
:1048C000883302086961705F666C61672069733ABA
:1048D00025780D0A0000000002630020000002405D
:1048E000E46200206E65002045717569706D656E2B
:1048F000742053746172742E2E2E2E2E2E2E2E2E78
:104900002E0D0A007265616420496E69745F44610E
:1049100074615F45717569706D656E742E2E2E2EF3
:104920002E2E2E2E2E2E0D0A000000004263323550
:104930005F49703A25730D0A00000000426332356A
:104940005F506F72743A25730D0A0000455350385A
:104950003236365F41505F506F7274733A25730D73
:104960000A000000455350383236365F41505F50E0
:104970005744733A25730D0A000000004553503820
:104980003236365F41505F53534944733A25730DB5
:104990000A0000004D6561737572655F496E74654C
:1049A0007276616C3A25730D0A0000005075625FE3
:1049B0004D6F64653A25730D0A0000005075625F03
:1049C00054696D653A25730D0A00000045717569DB
:1049D000706D656E745F49443A25730D0A000000DE
:1049E0006170706F696E746D656E745F74696D650A
:1049F0003A25730D0A0000006D6561737572655F7D
:104A00006D6F64653A25730D0A0000005061725F96
:104A100073746F72655F666C61673A25640D0A0096
:104A20007265616420496E69745F446174615F45B9
:104A3000717569706D656E7420656E642121212128
:104A4000210D0A00323000005254432069733A2588
:104A5000732025730D0A000073746172745F7761AF
:104A600079206973203A25640D0A000000B589B0E9
:104A70000120FCF74FF900BF2120FCF7FBF80028CC
:104A8000FAD001210420FCF73DFA202007900320F2
:104A90008DF8200000208DF8230007A96948FBF756
:104AA00055FF01214802FCF73EFA00208DF808006E
:104AB0008DF8090004900590019001208DF81800F0
:104AC00001A96148FBF7C8FB0120FBF73FFC01216E
:104AD0005D48FBF701FC5D4800885D49088009B02E
:104AE00000BD10B5044601215A48FBF7A9FF072372
:104AF000012221465448FBF738FC5348FBF7E1FC00
:104B000000BF02215048FBF70FFE0028F9D04E48A5
:104B1000FBF713FD10BD2DE9F047044601214D4878
:104B2000FBF78EFF1120FFF7DCFF4B490880204682
:104B3000FFF7D7FF0746484800880BF047F8804644
:104B4000434800880BF042F8814644490AF046FE8B
:104B5000064641460AF074FE4149086038460BF0AB
:104B600035F880463F490AF06BFE06463C4801682E
:104B700030460AF033FE05462846BDE8F0872DE9A9
:104B8000F34F83B00C464FF00009CA4611E003987A
:104B9000FFF7A7FF06460BF019F8054649460AF04D
:104BA000C5FD81460A20FFF74CFC0AF1010000F028
:104BB000FF0AA245EBDB20460BF008F80146019006
:104BC00048460AF03DFE274902900AF039FE834626
:104BD0000BF031F80746244A244B0AF016FF05462D
:104BE0000BF03CF88146484605B0BDE8F08F10B5A3
:104BF00001211848FBF724FF10BD10B5012115480D
:104C0000FBF720FF10BD70B50A210F20FFF7B7FF9B
:104C100006464FF4FA70FFF714FC0A210F20FFF745
:104C2000AEFF0646124930460AF0D8FD0646304629
:104C30000BF001F8044622460B460EA10F480DF07A
:104C400011F870BD0008024000240140F800F81F70
:104C5000F462002000040240F662002000004040A0
:104C6000F862002000F07F45CDCCCCCCCCCC0A4003
:104C700066668640252E33662C000000F26F002009
:104C80001CB501210720FCF73DF941F223000090FB
:104C900001208DF8040000208DF8060001208DF819
:104CA000070000208DF8050069462748FBF74EFEF7
:104CB00041F61010009001208DF8040000208DF8BE
:104CC000060001208DF8070000208DF805006946D8
:104CD0001E48FBF73BFE012000908DF804000020E9
:104CE0008DF8060001208DF8070000208DF80500E2
:104CF00069461748FBF72AFE01211348FBF7A2FE7D
:104D00004FF480511048FBF79DFE02210E48FBF73F
:104D100099FE4FF480510D48FBF794FE10210B488B
:104D2000FBF790FE01210A48FBF78CFE4FF400616F
:104D30000648FBF787FE20210348FBF783FE4FF46C
:104D40004870FFF77EFB1CBD0004024000000240DB
:104D50000008024000B587B001210620FCF7D2F818
:104D600001208DF8180000208DF81A0001208DF820
:104D70001B0002208DF819004020059005A9494824
:104D8000FBF7E4FD40214748FBF75AFE02208DF86F
:104D9000180000208DF81A0002208DF819004FF439
:104DA0006040059005A94048FBF7D0FD4FF46041F5
:104DB0003D48FBF745FE05220D213B48FBF74FFE22
:104DC00005220E213848FBF74AFE05220F213648FE
:104DD000FBF745FE01218803FCF7B6F80020ADF88B
:104DE00000004FF48270ADF802000020ADF804001E
:104DF000ADF80600ADF808004FF40070ADF80A00F9
:104E00001020ADF80C000020ADF80E000720ADF822
:104E1000100069462548FDF70FF801212348FDF7EA
:104E2000A9F807B000BD00F00700204909884FF637
:104E3000C77211401D4A11801146098841EAC0011C
:104E400011801146098841F04001118070470246E7
:104E5000002107E0481C81B24FF6FE70814201DB61
:104E60000020704711480830008800F00200002838
:104E7000F0D00E480C300280002107E0481C81B2BF
:104E80004FF6FE70814201DB0020EAE70748083058
:104E9000008800F001000028F0D004480C300088A1
:104EA000C0B2DEE7000802400004024000380040C3
:104EB00010B504462046FFF7CAFF10BD10B53820D4
:104EC000FFF7B1FF10BD10B50020FFF7ACFF10BD1C
:104ED00010B5FFF73FFFFFF7F6FF10BD10B54021FB
:104EE000FC48FBF7ADFDFF20FFF7E2FF10BD10B55A
:104EF000002400BFFF20FFF7DBFFFF2801D10020C7
:104F000010BD641C6FF07F408442F3D30120F7E7AB
:104F100010B54021EF48FBF795FDFFF7E8FF08B912
:104F2000002010BDFFF7DAFF0120FAE770B5054653
:104F30004FF6FF7401E0601E84B2FF20FFF7B8FF58
:104F4000A84201D0002CF6D10CB9FF2070BD002082
:104F5000FCE770B504460D46FE20FFF7E7FF08B1F9
:104F6000012070BD04E0FF20FFF771FF2070641C7A
:104F7000281EA5F101018DB2F5D1FF20FFF798FFA2
:104F8000FF20FFF795FF0020EBE770B506460D46C2
:104F9000FFF7ADFF08B1012070BD2846FFF788FF7D
:104FA000FD2D19D0002404E0305DFFF750FF601C98
:104FB00084B2B4F5007FF7DBFF20FFF779FFFF2015
:104FC000FFF776FFFF20FFF773FF044604F01F0092
:104FD000052801D00220DFE70020DDE72DE9F041C0
:104FE00005460C4617464FF00008FFF777FFFFF71E
:104FF0008FFF10B1FF20BDE8F08145F04000FFF7C2
:1050000057FF200EFFF754FFC4F30740FFF750FF90
:10501000C4F30720FFF74CFFE0B2FFF749FF384623
:10502000FFF746FF0C2D02D1FF20FFF741FF4FF0A5
:105030001F0800BFFF20FFF73BFF064606F0800079
:1050400030B1B8F10000A8F1010101F0FF08F1D181
:105050003046D0E770B50546012200210A20FFF74F
:10506000BDFF044624B910212846FFF772FF04460D
:10507000FFF734FF0CB1012070BD0020FCE770B5D4
:105080000546012200210920FFF7A8FF044624B9A4
:1050900010212846FFF75DFF0446FFF71FFF0CB104
:1050A000012070BD0020FCE77FB56846FFF7E7FFF1
:1050B00010B1002004B070BD9DF8000000F0C000E9
:1050C000402809D19DF809009DF8081000EB012047
:1050D000401C84B2A50220E09DF8050000F00F00FE
:1050E0009DF80A1000EBD1109DF8091001F00301A2
:1050F00000EB4100861C9DF8080080119DF8071008
:1051000000EB81009DF8061001F0030100EB812007
:10511000441CA6F1090004FA00F52846CAE7F8B5D0
:10512000FFF7D6FEFFF7CAFE002504E0FF20FFF7D9
:10513000BFFE681C85B20A2DF8DB142600BF95223D
:1051400000210846FFF74AFF0446012C04D0301E18
:10515000A6F101018EB2F2D100205F490870012C46
:105160004AD187224FF4D5710820FFF737FF012875
:1051700047D1002506E0FF20FFF79AFE0DF8050055
:10518000681C85B2042DF6DB9DF80200012879D158
:105190009DF80300AA2875D14FF6FE7600BF0122C4
:1051A00000213720FFF71AFF012291072920FFF77E
:1051B00015FF044624B1301EA6F101018EB2EED1D6
:1051C000002E5FD0012200213A20FFF707FF0028C0
:1051D00058D1002506E0FF20FFF76AFE0DF8050014
:1051E000681C85B2042DF6DB9DF8000000F040003D
:1051F00018B106203849087044E004203649087088
:1052000040E0012200213720FFF7E8FE01220021C3
:105210002920FFF7E3FE0446012C17DC02202E496B
:1052200008704FF6FE7600BF012200213720FFF7FD
:10523000D5FE012200212920FFF7D0FE0446BCB193
:10524000301EA6F101018EB2EED111E001202249FB
:1052500008704FF6FE7600BF012200211046FFF7CE
:10526000BDFE044624B1301EA6F101018EB2F3D179
:105270002EB1012251021020FFF7B0FE10B1002024
:1052800015490870FFF72AFEFFF71DFE1248007847
:1052900008B10020F8BD0CB12046FBE7AA20F9E7D1
:1052A0002DE9F04106460F4615460B4800780628C2
:1052B00000D07F02012D11D1012239461120FFF7C4
:1052C0008DFE044624BB69023046FFF742FE0446C9
:1052D0001EE0000000080240FC6200200122394666
:1052E0001220FFF77BFE044600BF4FF400713046EA
:1052F000FFF72FFE044606F50076681EC0B2051EB5
:1053000001D0002CF1D0012200210C20FFF766FE15
:10531000FFF7E4FD2046BDE8F0812DE9F0410646A7
:105320000F46154620480078062800D07F02012D40
:105330000CD1012239461820FFF750FE04466CBB01
:10534000FE213046FFF721FE044627E0164800788C
:10535000012809D0012200213720FFF73FFE01225A
:1053600029461720FFF73AFE012239461920FFF798
:1053700035FE044694B900BFFC213046FFF705FE18
:10538000044606F50076681EC0B2051E01D0002C4A
:10539000F2D0FD210020FFF7F8FD0446FFF79EFD47
:1053A0002046BDE8F0810000FC62002010B588B006
:1053B000044601218804FBF7C7FD01210220FBF709
:1053C000A1FD5B48FDF70AFD4FF44060029002200A
:1053D0008DF80C008DF80D0000208DF80E000120D6
:1053E0008DF80F0002A95348FBF7B0FA07220A21F3
:1053F0005048FBF734FB07220B214E48FBF72FFBED
:1054000004940020ADF81400ADF81600ADF81800B3
:10541000ADF81C000C20ADF81A0004A94448FDF7B3
:1054200020FD01214248FDF7A1FD012240F2255156
:105430003F48FDF751FE27208DF8040002208DF82B
:10544000050000208DF8060001208DF8070001A856
:10545000FAF789FE40213648FDF770FE08B010BD0E
:1054600010B540F225513248FDF771FE00283AD0C0
:105470002F48FDF7AAFDC4B2242C02D100202E49EA
:1054800008802D490888411C2B4A11802B490C5457
:105490000846007824281FD1084600794D281BD1E2
:1054A00008464079432817D10A2C15D150212448A9
:1054B0000AF0F3F820480288204921480AF0D4F87D
:1054C00001201F4981F8A00000201B4908804FF4EB
:1054D00080711A480AF0E1F817480088FF2802DBBB
:1054E00000201549088010BD0FB438B505A80090FC
:1054F0001448009A04990CF0C9FB00200090114850
:105500000AF0F2F885B200240DE000BF40210848FF
:10551000FDF707FE0028F9D00A48015D0448FDF7B1
:1055200050FD601C84B2AC42EFDB38BC5DF814FB6C
:105530000048004000040240FE6200200A6400208F
:105540004E7800200A65002030B5FD4C031903E0B9
:1055500013F8014B01F8014B141EA2F10105AAB288
:10556000F6D130BD30B5F64C031903E01C8821F8A4
:10557000024B0833141EA2F10105AAB2F6D130BDC8
:1055800030B5EF4C031902E01C6810C11033141E33
:10559000A2F10105AAB2F7D130BD30B5E84C03192C
:1055A000E84CE94D2C60E94C2C6000BFE64C083C0F
:1055B000246804F00104002CF8D1E34C083C246872
:1055C00044F48074E04D083D2C600BE011F8014B71
:1055D00003F8014B00BFDC4C0C34246804F00104D8
:1055E000002CF8D1141EA2F10105AAB2EED1D64CBE
:1055F000083C246844F00104D34D083D2C6030BDC4
:1056000030B5CF4C0319CF4CCF4D2C60CF4C2C6014
:1056100000BFCD4C083C246804F00104002CF8D1F4
:10562000C94C083C246844F48074C74D083D2C6084
:105630000BE031F8024B1C60083300BFC24C0C3445
:10564000246804F00104002CF8D1141EA2F1010515
:10565000AAB2EED1BC4C083C246844F00104BA4D17
:10566000083D2C6030BD30B5B54C0319B54CB64D76
:105670002C60B64C2C6000BFB34C083C246804F08E
:105680000104002CF8D1B04C083C246844F4807428
:10569000AD4D083D2C600AE010C91C60103300BFFE
:1056A000A94C0C34246804F00104002CF8D1141E19
:1056B000A2F10105AAB2EFD1A34C083C246844F042
:1056C0000104A14D083D2C6030BD10B5A0B00446CA
:1056D0008021684609F0E1FF142269460020FFF7A7
:1056E00033FF0A2205A91420FFF72EFF0A220DF12D
:1056F00032011E20FFF728FF14220FA93C20FFF7DC
:1057000023FF14220DF11E012820FFF71DFF0622A2
:1057100014A96420FFF718FF05220DF156016E2031
:10572000FFF712FF06220DF15B017820FFF70CFF57
:105730000A220DF161018220FFF706FF0F220DF111
:105740006B019620FFF700FF02220DF17A01A620DF
:10575000FFF7FAFE01221FA9B920FFF7F5FE01228B
:105760000DF17D01BA20FFF7EFFE7E22694620464B
:1057700009F07AFF20B010BD18B500200090002479
:1057800000BF05E0A0B201226946FFF706FF641CD6
:10579000BA2CF7DB18BD0FB410B5FFF7EDFF02A868
:1057A00009F0A2FF84B2224602A90020FFF7F5FE0D
:1057B00007A809F099FF84B2224607A91420FFF731
:1057C000ECFE0DF13A0009F08FFF84B222460DF194
:1057D0003A011E20FFF7E1FE11A809F085FF84B20F
:1057E000224611A93C20FFF7D8FE0DF1260009F052
:1057F0007BFF84B222460DF126012820FFF7CDFE63
:1058000016A809F071FF84B2224616A96420FFF79A
:10581000C4FE0DF15E0009F067FF84B222460DF16F
:105820005E016E20FFF7B9FE0DF1630009F05CFF29
:1058300084B222460DF163017820FFF7AEFE0DF130
:10584000690009F051FF84B222460DF169018220FE
:10585000FFF7A3FE0F220DF173019620FFF79DFEC7
:1058600001220DF18201A620FFF797FE012221A956
:10587000B920FFF792FE01220DF18501B920FFF753
:105880008CFE012232498C20FFF787FE10BC5DF8A8
:1058900014FB10B514212F4809F0FFFE2D480021FC
:1058A0004161816181833230016041600181142155
:1058B0000A3009F0F2FE142126481E3009F0EDFEF0
:1058C000244800210165A0F8541056300160017190
:1058D000401D01608180801D0160416001810F21B8
:1058E0000A3009F0DAFE1B480021A0F87A100020E7
:1058F000184981F87C0081F87D0010BD00B5BDB06D
:10590000FFF7C7FF14A219A112480CF0ABF918A2B7
:1059100016A1104814300CF0A5F917A213A10D48D8
:1059200032300CF09FF916A210A10A483C300CF05E
:1059300099F916A20DA107481E300CF093F92BE03F
:1059400000000808EFCDAB890C3C024005040302BF
:10595000E46200206E650020223231392E32333865
:105960002E3234302E35382200000000257300001E
:10597000393032320000000038303830000000008A
:105980003838383838383838000000006C696361BE
:10599000776966690000000042A2AFF23001434817
:1059A0000CF060F942A2AFF23C014048801D0CF0BF
:1059B00059F940A2AFF24C013C480B300CF052F9BF
:1059C0003DA2AFF25801394811300CF04BF93CA21E
:1059D000AFF2680135481B300CF044F93CA2AFF23D
:1059E000740132482A300CF03DF900202F4950391B
:1059F00081F87C0081F87D006E221031684609F044
:105A000033FE7E22294950391DA809F02DFE1DA81C
:105A10000FC8FFF7C0FE01202E49087001228C201C
:105A2000FFF7BBFD3DB000BD2DE9F0410546002666
:105A3000284609F059FE87B2082F02DD0020BDE894
:105A4000F081002416E0285D30280FDB285D39281E
:105A50000CDC002C05DD06EB86004FF6FF7101EA39
:105A60004006285D3038304486B201E00020E6E789
:105A7000601C84B2BC42E6DB3046E0E710B50B4860
:105A8000FFF7D2FF0446C4EB0410800010BD10B530
:105A900006480B30FFF7C8FF0446C4EB0410800033
:105AA00010BD00003030303031000000BE650020F5
:105AB0003030000035000000313233340000000087
:105AC0003230323230333135303030303030000027
:105AD00030000000E462002010B50020FE4908807C
:105AE0004FF49671FD4809F0D8FD10BD10B588B08F
:105AF000044601214804FBF727FA01210846FBF779
:105B000001FAF748FDF76AF90C20029002208DF89F
:105B10000C008DF80D0000208DF80E0001208DF88E
:105B20000F0002A9EF48FAF711FF07220221ED4802
:105B3000FAF795FF07220321EA48FAF790FF049449
:105B40000020ADF81400ADF81600ADF81800ADF85F
:105B50001C000C20ADF81A0004A9E148FDF781F9FA
:105B60000121DF48FDF702FA012240F22551DC480D
:105B7000FDF7B2FA26208DF8040003208DF8050009
:105B800000208DF8060001208DF8070001A8FAF723
:105B9000EAFA4021D248FDF7D1FA08B010BD0FB49F
:105BA00038B5FFF799FF05A80090CF48009A0499EF
:105BB0000CF06CF800200090CB4809F095FD85B200
:105BC00000240DE000BF4021C548FDF7AAFA0028D7
:105BD000F9D0C548015DC248FDF7F3F9601C84B2F5
:105BE000AC42EFDB38BC5DF814FB1FB50121084661
:105BF000FBF7AAF940F2E730029040F67F40ADF89B
:105C000004000120ADF80C000020ADF8060001A949
:105C10004FF08040FCF74AFC012211469007FCF748
:105C2000D2FF01218807FCF7F6FF00214FF08040EA
:105C3000FCF7B6FC1C208DF8000001208DF8010057
:105C400000208DF8020001208DF803006846FAF765
:105C50008AFA01218807FCF7A3FC1FBD10B5044692
:105C60004CB100214FF08040FCF75AFC012188071D
:105C7000FCF796FC04E000214FF08040FCF790FC1C
:105C800010BD10B501218807FCF7B4FF38B1012120
:105C90008807FCF7C0FF01F04CFA9449087010BD6A
:105CA00010B540F225518E48FDF751FAD8B18C4815
:105CB000FDF78BF9C4B28848008800F4004090B921
:105CC00085480088B0F5957F07DC83490888411C2A
:105CD000814A118081490C5405E07F48008840F4D6
:105CE00000407D49088010BD2DE9F047FCB000263A
:105CF000B046602164A809F0D0FC7D48006863903C
:105D00000020609061905D905E905F901DA8FFF70D
:105D1000DCFC80221DA93DA809F0A6FC75A16F48F6
:105D200009F0C6FC90B1FFF7E9FD012274498C200F
:105D3000FFF70AFC7248007820B172A10D2006F02E
:105D4000DCFF03E073A10D2006F0D7FF75A16348C7
:105D500009F0AEFC00287DD07449604809F0A8FC29
:105D600010B14FF0010901E04FF000096F491139FE
:105D70005A4809F09DFC08B1012000E0002009EA22
:105D800000096A490A31554809F092FC08B101201E
:105D900000E0002009EA0009644919314F4809F080
:105DA00087FC08B1012000E0002009EA00095F49F2
:105DB000891F4A4809F07CFC08B1012000E000205E
:105DC00009EA0009B9F1000F0AD0002057496139EA
:105DD00081F87C0001220021B920FFF7DEFB09E0F9
:105DE00001205249613981F87C0001227C31B920BF
:105DF000FFF7D3FB642163A809F04FFC0026B1E054
:105E000036B948A1354809F053FC0446A41DA7E063
:105E1000641C47A1204609F04BFC051E49D0012E09
:105E200006D0022E0ED0032E2AD0042E3FD133E00E
:105E30003E4800210160416001812A1B214609F092
:105E400013FC00BF394861380021016580F8541007
:105E50002A1B00E0DFE02146503009F005FC334802
:105E60001138FFF7E1FD80463048613800210165B7
:105E700080F8541042462FA150300BF0F3FE17E08B
:105E80000F212A480A3009F008FC2A1B214627481E
:105E90000A3009F0E9FB0BE024486138002180F862
:105EA0007A102A1B21467A3009F0DEFB00E000BFA1
:105EB00000BF2C46042E53D1641C1FA1204609F0BC
:105EC000F7FB05461948801F0021016081802A1BCD
:105ED000214609F0C9FB31E000630020EC65002099
:105EE0000044004000000240186700207962002052
:105EF0008C330208706172772D7273740000000099
:105F0000E4620020706172772D7273742C4F4B2CF9
:105F10002A000000706172772D7273742C666169BB
:105F20006C2C2A00706172772D310000CF65002043
:105F30002C000000256400002C2A0000F948FFF71F
:105F400073FD8046B8F1010F01DA4FF00108F54802
:105F50000021016081804246AFF228010BF082FEF1
:105F6000701CC6B2052EFFF64BAFEE480B38FFF79C
:105F70005BFD012805DAECA2EDA1EA480B380BF035
:105F800071FE6E22E7494B39684609F06DFB7E22AF
:105F9000E4495B391DA809F067FB1DA80FC8FFF78E
:105FA000FAFBE4A10B2006F0A8FEDE49891D0DF2E4
:105FB000551009F0A0FBC8B9DA490B3951A809F00E
:105FC0009AFB98B9D74910310DF25F1009F093FB95
:105FD00060B9D4491F310DF5B77009F08CFB28B9B1
:105FE000D0490DF24F1009F086FB48B10120CD4990
:105FF0005B3981F87C0001227C31B920FFF7CDFAB2
:10600000C8485B3890F87A00312802D101F00AF8CC
:1060100001E001F06DF8CAA1CB4809F049FB10B1CD
:106020004FF0010901E04FF00009C8A1C64809F08E
:106030003FFB08B1012000E0002009EA0009B9F1A6
:10604000000F75D0B7495B39BF4809F031FB10B17B
:106050004FF0010901E04FF00009B2494739BA4851
:1060600009F026FB08B1012000E0002009EA000940
:10607000AC493D39B44809F01BFB08B1012000E0F0
:10608000002009EA0009A7491F39AF4809F010FBB1
:1060900008B1012000E0002009EA0009A1492939DE
:1060A000A94809F005FB08B1012000E0002009EA39
:1060B0000009B9F1000F0AD000209A495B3981F834
:1060C0007C0001220021B920FFF767FA09E00120D6
:1060D00094495B3981F87C0001227C31B920FFF7BB
:1060E0005CFA00264FE036B995A1974809F0E0FA2E
:1060F0000446A41D45E0641CAFF2CC11204609F013
:10610000D7FA051E3CD0012E06D0022E11D0032E48
:106110001BD0042E32D124E0142182485B3809F0D0
:10612000BCFA2A1B21467F485B3809F09DFA26E01D
:106130006FE07C485B3800214161816181832A1BCB
:106140002146143009F090FA19E0142175483D38C1
:1061500009F0A3FA2A1B214672483D3809F084FA57
:106160000DE070485B380021C1630164A0F8441061
:106170002A1B21463C3009F077FA00E000BF00BF3F
:106180002C46701CC6B2052EADDB66485B38D4F8D1
:106190000110C0F832106E2200F11001684609F0BB
:1061A00063FA7E225F495B391DA809F05DFA1DA8DC
:1061B0000FC8FFF7F0FA66A10B2006F09EFD5949C3
:1061C0005B393DA809F097FAC8B95649473942A842
:1061D00009F091FA98B953493D390DF5897009F0E4
:1061E0008AFA60B94F491F394CA809F084FA30B9CE
:1061F0004C4929390DF5937009F07DFA48B1012019
:1062000048495B3981F87C0001227C31B920FFF7D5
:10621000C4F952A14C4809F04BFA20B351A14A48A5
:1062200009F046FA041E19D051480078C0F3001056
:106230004F490978C1F38001084320B14DA10B20DB
:1062400006F05BFD0AE04E48007820F02000203088
:106250004B49087047A10B2006F04FFD49A13A4871
:1062600009F026FA04464AA1374809F021FA041E2B
:1062700056D0642163A809F010FAE41D0D222146CE
:1062800063A809F0F1F99DF8910130389DF890115B
:10629000303901EB810100EB41000C2801DD0121C7
:1062A00000E000219DF8930130389DF89221303AAA
:1062B00002EB820200EB42001F2801DD012000E01A
:1062C000002008439DF8951130399DF89421303A0B
:1062D00002EB820201EB4201172901DD012100E0FE
:1062E000002108439DF8971130399DF89621303AE6
:1062F00002EB820201EB42013B2901DD012100E0BA
:10630000002108439DF8991130399DF89821303AC1
:1063100002EB820201EB42013B293DDD01213CE021
:1063200004E10000C9650020303030303100000049
:1063300025730000706172772D312C4F4B2C2A0091
:10634000706172772D320000EC65002022000000A1
:10635000706172772D322C4F4B2C2A00706172774E
:106360002D330000706172772D332C310000000056
:1063700071620020706172772D332C4F4B2C2A00F4
:1063800002630020706172772D332C300000000012
:10639000706172772D3400000021084320B1C2A142
:1063A0000D2006F0AAFCC1E09DF8990130389DF857
:1063B0009811303901EB810100EB41019DF8970103
:1063C00030389DF89621303A02EB820200EB420011
:1063D000CDE900019DF895C1ACF1300C9DF8949188
:1063E000A9F1300909EB89090CEB49039DF893C128
:1063F000ACF1300C9DF89291A9F1300909EB8909B3
:106400000CEB49029DF891C1ACF1300C9DF89091D4
:10641000A9F1300909EB89090CEB49019DF88FC1FD
:10642000ACF1300C9DF88E91A9F1300909EB890986
:106430000CEB490000F025FA9DF8990130389DF8E1
:106440009811303901EB810100EB4100C1B29DF898
:10645000970130389DF89621303A02EB820200EB2A
:106460004200C0B2CDE900019DF895C1ACF1300CFD
:106470009DF89491A9F1300909EB89090CEB490CBD
:106480000CF0FF039DF893C1ACF1300C9DF8929194
:10649000A9F1300909EB89090CEB490C0CF0FF025A
:1064A0009DF891C1ACF1300C9DF89091A9F13009A3
:1064B00009EB89090CEB490C0CF0FF019DF88FC129
:1064C000ACF1300C9DF88E91A9F1300909EB8909E6
:1064D0000CEB490C0CF0FF0008F0D8FF022263A976
:1064E000AA20FFF75AF87448006800F4807020B1C1
:1064F000FFF7CDFA814600F081FB6F48006800F499
:10650000007030B1FFF7BAFAA0F10109484600F077
:10651000BAFA6AA10B2006F0F0FB01206A4981F863
:106520007C0001220021B920FFF737F867A16948F4
:1065300009F0BEF8041E19D0AFF20C61204609F034
:10654000B7F80446641CA51C2978207808F0B6FC2E
:10655000287808F0EBFC074627B95FA10B2006F06E
:10656000CCFB03E05FA10D2006F0C7FB61A15948F9
:1065700009F09EF8041E2AD0642163A809F08DF862
:106580001DA8FFF7A2F87E221DA94F4809F06CF85C
:106590004D485B30FFF748FA81464B485030FFF7D3
:1065A00043FA824648487A30A0F10F015346A0F1E1
:1065B0001902CDE90109009150A163A80BF052FB2B
:1065C00063A809F091F8814663A906F096FB51A1F2
:1065D000404809F06DF800B3642163A809F05DF844
:1065E0005DA960A800F0D9F93748323000F10A02FD
:1065F000A0F11401A0F11E03CDE90031CDE9022084
:10660000143B44A245A163A80BF02CFB63A809F03E
:106610006BF8814663A906F070FB45A12D4809F08F
:1066200047F8D8B1642163A809F037F85DA960A8DC
:1066300000F0B3F9022262A9AA20FEF785FF60A844
:106640005DAB62AA3CA1009063A80BF00BFB63A8B2
:1066500009F04AF8814663A906F04FFB3BA11D48AB
:1066600009F026F8041E1CD0642163A809F015F86F
:106670001DA8FFF72AF87E221DA9134808F0F4FF91
:1066800011486130FFF7D0F981464A4631A163A82D
:106690000BF0E8FA63A809F027F8814663A906F031
:1066A0002CFB7CB0BDE8F087706172772D342C66CE
:1066B00061696C2C2A000000082800407061727724
:1066C0002D342C4F4B2C2A006E65002070617277A0
:1066D0002D350000EC650020706172772D352C4F50
:1066E0004B2C2A00706172772D352C6661696C2CF9
:1066F0002A000000706172722D31000070617272A8
:106700002D312C25732C25642C25732C25732C25D9
:10671000642C2A00706172722D32000025732C25C2
:10672000732C25732C25732C25732C25732C2A0090
:10673000706172722D340000706172722D342C25DC
:106740007325732025732C2A00000000706172727B
:106750002D733F00706172722D362C25642C2A0037
:1067600000B585B001210420FAF7CCFB00208DF89C
:1067700004008DF806004FF40050009002208DF8C0
:1067800007006946FE48FAF7E1F800220D21FC48AF
:10679000FAF765F94FF48010FAF770F84FF48010AB
:1067A000029001208DF80E0000208DF80C000820CA
:1067B0008DF80D0002A8F9F7EAFF03208DF810000C
:1067C00001208DF8130000208DF811008DF81200C3
:1067D00004A8F9F7C8FC4FF40030FAF74FF84FF46B
:1067E0000030029000208DF80C0008208DF80D007C
:1067F00001208DF80E0002A8F9F7C9FF29208DF8B5
:10680000100000208DF811008DF8120001208DF885
:10681000130004A8F9F7A7FC05B000BD0EB50121CF
:106820000807FAF791FB0120FAF757F90120FAF768
:1068300074FA00BF4920FAF71DFA0028FAD04FF485
:106840008030FAF737FB0120FAF754FBFAF72EFCF9
:106850007F20019000200090FF2002906846FAF708
:10686000ECFCFFF77DFF0EBD10B501210807FAF71C
:106870006BFB0120FAF731F9FAF718FCFFF770FF0C
:1068800010BD2DE9FC4704460D4616461F46DDE9BE
:106890000A89F8B28DF8040008F0FF008DF80500B1
:1068A00009F0FF008DF8060000208DF8070001A90F
:1068B000FAF75EFDE0B28DF80300E8B28DF8010052
:1068C000F0B28DF8020001208DF80000694600202A
:1068D000FAF7ECFD43F2F2210020FBF798F9BDE84E
:1068E000FC872DE9FC47A74890F8CA00F0B3A548FB
:1068F00090F8CC003038A34991F8CB10303901EB37
:10690000810100EB41049F4890F8CE0030389D494A
:1069100091F8CD10303901EB810100EB4105994828
:1069200090F8D0003038974991F8CF10303901EB0A
:10693000810100EB4106934890F8A300303891495B
:1069400091F8A210303901EB810100EB410000F118
:1069500008078C4890F8A50030388A4991F8A410AF
:10696000303901EB810100EB410800E013E085487C
:1069700090F8A7003038834991F8A610303901EB20
:10698000810100EB41093B46324629462046CDE9CC
:106990000089FFF776FFBDE8FC877CB504460D460D
:1069A00001A90020FAF74EFD69460020FAF7E4FD40
:1069B0009DF803000A2190FBF1F0303028709DF81B
:1069C000030090FBF1F201FB1200303068709DF87B
:1069D000010090FBF1F03030A8709DF8010090FBB1
:1069E000F1F201FB12003030E8709DF8020090FBDC
:1069F000F1F0303028719DF8020090FBF1F201FBBC
:106A00001200303068719DF8040090FBF1F03030D6
:106A100020709DF8040090FBF1F201FB1200303071
:106A200060709DF8050090FBF1F03030A0709DF88B
:106A3000050090FBF1F201FB12003030E0709DF890
:106A4000060090FBF1F0303020719DF8060090FBBD
:106A5000F1F201FB1200303060717CBD38B569463F
:106A60000020FAF7EFFC9DF800004FF46161484305
:106A70009DF80110C1EB011100EB81009DF802109F
:106A80004418204638BD3EB504464FF48010F9F74F
:106A9000F5FE4FF48010009001208DF806000020D4
:106AA0008DF8040008208DF805006846F9F76FFEA0
:106AB00003208DF8080001208DF80B0000208DF8D0
:106AC00009008DF80A0002A8F9F74DFB0020FAF73B
:106AD000B2FE4FF48060FBF744F9B4F5803F06D373
:106AE0000620FAF783FEA4F57F44FF3C02E0042071
:106AF000FAF77CFE2046FAF78EFE4FF48040FBF753
:106B000060F901218803FBF7E5F80120FAF793FE0D
:106B10003EBD00B585B001210420FAF7F3F900204D
:106B20008DF804004FF40050009002208DF807000B
:106B300069461348F9F70AFF00220D211048F9F7BA
:106B40008EFF01210846FAF7EEF90D210220FBF72E
:106B5000FCFA4FF40050F9F791FE4FF40050029008
:106B600001208DF80E0000208DF80C0008208DF813
:106B70000D0002A8F9F70BFE28208DF8100003E0A5
:106B8000000802404E78002001208DF813000020FC
:106B90008DF811008DF8120004A8F9F7E4FA01212C
:106BA0000420F9F7A9FF05B000BD014601F5FA6020
:106BB00081B2CA1701EB92729210A1EB820292B9D4
:106BC000642091FBF0F200FB121050B94FF4C87032
:106BD00091FBF0F200FB121008B901207047002071
:106BE000FCE70120FAE70020F8E710B5FFF7B8FD51
:106BF000FFF714FE0120FAF703F810BD30B589B095
:106C000004464FF40030F9F739FE4FF40030069097
:106C100000208DF81C0008208DF81D0001208DF843
:106C20001E0006A8F9F7B3FD29208DF820000020EA
:106C30008DF821008DF8220001208DF8230008A88E
:106C4000F9F791FA4FF48070FBF78BF84FF480500E
:106C5000FBF7B7F800214FF48070FAF767FD05A93C
:106C60000020FAF7EFFB04A90020FAF785FC9DF855
:106C70001100401EFE490D5C9DF81100022805D14F
:106C80009DF81300FFF791FF00B96D1C9DF81400EB
:106C90004FF4616148439DF81510C1EB011100EB01
:106CA00081009DF8161001449DF8120040F2A322C5
:106CB000504301EBC0100444D001B4FBF0F0A842F3
:106CC00007D9D001B4FBF0F0451BE8B28DF80C00F9
:106CD00005E0E848B4FBF0F0C0B28DF80C000020ED
:106CE000029001908DF80300E248B4FBF0F100FB44
:106CF00011404FF46161B0FBF1F0C0B28DF80000BB
:106D0000DC48B4FBF0F100FB11404FF46161B0FBD3
:106D1000F1F201FB12003C21B0FBF1F0C0B28DF8A2
:106D20000100D448B4FBF0F100FB11404FF4616165
:106D3000B0FBF1F201FB12003C21B0FBF1F201FBD0
:106D400012008DF802006A464FF480710020FAF7B5
:106D500036FC01210803FAF7BDFF01210802FAF70A
:106D6000E5FC09B030BD2DE9F04387B08046894687
:106D700014461D46DDE90E674FF40030F9F77EFD3D
:106D80004FF40030049000208DF8140008208DF896
:106D9000150001208DF8160004A8F9F7F8FC292049
:106DA0008DF8180000208DF819008DF81A000120C8
:106DB0008DF81B0006A8F9F7D6F94FF40070FAF722
:106DC000D0FF4FF40050FAF7FCFF00214FF40070A1
:106DD000FAF7ACFCE0B28DF80C00002002900190B4
:106DE0008DF80300E8B28DF80000F0B28DF80100D4
:106DF000F8B28DF802006A464FF400710020FAF7ED
:106E0000DEFB01214803FAF765FF01214802FAF78A
:106E10008DFC07B0BDE8F08310B5002410E04FF4FE
:106E200000519548F9F7F4FD40B1601CC4B21E2032
:106E3000FDF707FB642C03DB012010BD0020FCE7FD
:106E4000EDE710B54FF48050FAF79AFF70B14FF4A8
:106E50000030F9F713FD4FF48050FAF7B2FF87487E
:106E6000007820F00100401C844908704FF4005065
:106E7000FAF786FF70B14FF40030F9F7FFFC4FF4DA
:106E80000050FAF79EFF7D48007820F00200801C39
:106E90007A4908704FF48040FAF772FF70B14FF4EE
:106EA0008010F9F7EBFC4FF48040FAF78AFF734843
:106EB000007820F00400001D704908704FF4005164
:106EC0006D48F9F7A5FD88B1FFF7A6FF6C4908707A
:106ED0000846007830B16948007820F00800083092
:106EE000664908704FF40050F9F7C8FC6348007811
:106EF00000F0010061490978C1F3400108435F498E
:106F00000978C1F3800108435C490978C1F3C001E5
:106F10000843D8B15948007800F0010008B10120B9
:106F200010BD56480078C0F3400008B10220F7E7D2
:106F300052480078C0F3800008B10320F0E74F48C2
:106F40000078C0F3C00050B10420E9E74B48007856
:106F500020F010001030494908700020E0E70020C0
:106F6000DEE710B54FF48050FAF70AFFB8B14FF4DE
:106F70008050FAF726FF4148007820F00100401CBD
:106F80003E49087000214FF48070FAF7CFFB3DA016
:106F900001F087F8FEF77BFD0446FFF72FFE4FF464
:106FA0000050FAF7EDFE78B14FF40050FAF709FF00
:106FB00000214FF40050FAF7B9FB3048007820F078
:106FC0000200801C2D4908704FF40030F9F756FC80
:106FD00010BD10B54FF48040FAF7D2FE08B34FF45D
:106FE0008040FAF7EEFE0020FAF725FC4FF48010FF
:106FF000F9F744FC2148007820F00400001D1F49E7
:10700000087023A001F04DF824480078C0F38001F7
:1070100023A001F046F8FEF731FD441E2046FFF79D
:1070200032FD10BD1CB500214FF48070FAF77EFBD5
:107030000020FAF700FC1F4890F8720030381D4914
:1070400091F87110303901EB810100EB41011948D1
:1070500090F870003038174A92F86F20303A02EBFF
:10706000820200EB4200CDE90001124824E000005A
:1070700090330208805101000008024002630020A2
:107080007A620020616C61726D412068700D0A00A7
:107090005755542068700D0A0000000071620020EE
:1070A0007775745F50524F53315F52554E3A256495
:1070B0000D0A00006E65002090F86E0030384C49D3
:1070C00091F86D10303901EB810100EB4103484824
:1070D00090F86C003038464991F86B10303901EB6C
:1070E000810100EB41020B211420FFF73CFE1CBD87
:1070F00010B54048007820F00100401C3D49087060
:107100000846007820F00400001D087000214FF4AC
:107110000070FAF70BFB3020354981F87A0010BD7A
:1071200010B54FF40050F9F7A9FB33A000F0B9FFF8
:1071300010BD10B500243448007820B1012818D0C3
:10714000022850D133E04FF400513048F9F760FC89
:1071500018B101202C49087002E000202A4908706B
:1071600000202B490870084600782A49087000243E
:107170003AE04FF400512548F9F74AFC98B1244809
:107180000078401C224908700846007821490870A0
:107190001F480078C82809DBC8201D490870022054
:1071A0001949087002E00220174908701CE04FF4EA
:1071B00000511648F9F72CFCA0B9002012490870BC
:1071C000134800780A2800DD032411480078642859
:1071D00000DD04240E4801780FA000F062FF0020BB
:1071E0000B49087000E000BF00BF204610BD000042
:1071F0006E6500200263002057414B4555503220F8
:107200006973204850000000046300200008024019
:10721000056300200363002054696D65436E743A72
:1072200025640D0A0000000010B588B00446002057
:107230004649087001218803F9F775FE01210220F3
:10724000F9F760FE4248FBF7C9FDC020029002201A
:107250008DF80C008DF80D0000208DF80E00012037
:107260008DF80F0002A93B48F9F770FB07220621B1
:107270003848F9F7F4FB072211463648F9F7EFFBD7
:1072800004940020ADF81400ADF816004FF48060AF
:10729000ADF818000020ADF81C000C20ADF81A0065
:1072A00004A92B48FBF7DDFD01212948FBF75EFE11
:1072B000012240F225512648FBF70EFF25208DF8CC
:1072C000040003208DF805008DF8060001208DF8DC
:1072D000070001A8F8F747FF40211D48FBF72EFFE4
:1072E00008B010BD10B564211B4808F0D6F9002085
:1072F0001A49088010BD10B56421194808F0CDF96D
:1073000010BD0FB438B505A800901548009A04992F
:107310000AF0BCFC00200090114808F0E5F985B2A5
:1073200000240DE000BF40210948FBF7FAFE0028C9
:10733000F9D00B48015D0648FBF743FE601C84B2A0
:10734000AC42EFDB38BC5DF814FB00006D6200203E
:107350000038014000040240446800200663002019
:10736000A868002010B588B004460121C804F9F7C8
:10737000EBFD01210420F9F7C5FDFE48FBF72EFDCA
:107380004FF44060029002208DF80C008DF80D0043
:1073900000208DF80E0001208DF80F0002A9F6489C
:1073A000F9F7D4FA4FF40060029002A9F248F9F715
:1073B000CDFA08220B21F048F9F751FB08220A21E7
:1073C000ED48F9F74CFB04940020ADF81400ADF83B
:1073D0001600ADF81800ADF81C000C20ADF81A002E
:1073E00004A9E448FBF73DFD0121E248FBF7BEFD9F
:1073F00030208DF8040005208DF8050000208DF860
:10740000060001208DF8070001A8F8F7ACFE012264
:1074100040F22551D748FBF75FFE4021D548FBF7E6
:107420008DFE012240F22441D248FBF755FE08B000
:1074300010BD10B5D148B0F8C80020F40040CF49C5
:10744000A1F8C8000846B0F8C8006FF30E00A1F814
:10745000C800C821C94808F020F910BD10B540F295
:107460002551C448FBF773FE20B3C248FBF7ADFDBE
:10747000C4B2C248B0F8C800C0F30E00C7280FDA83
:10748000BE49B1F8C810C1F30E00411CBB4AB2F8A6
:10749000C82061F30E02B949A1F8C8200C5409E0D4
:1074A000B648B0F8C80020F4004000F50040B349E9
:1074B000A1F8C8000821AF48FBF749FE30B1AD483C
:1074C000FBF783FD0821AB48FBF738FE40F224416F
:1074D000A848FBF73CFE68B1A848B0F8C80020F403
:1074E000004000F50040A549A1F8C800A148FBF7FD
:1074F0006CFDC4B210BD0FB438B505A80090A0480B
:10750000009A04990AF0C2FB002000909C4808F001
:10751000EBF885B200240DE000BF40219548FBF751
:1075200000FE0028F9D09648015D9248FBF749FD1E
:10753000601C84B2AC42EFDB38BC5DF814FB2DE973
:10754000F047E2B00026B04600205F9060905C906B
:107550005D905E901CA8FEF7B8F880221CA93CA89C
:1075600008F082F88548B0F8C8000121B1EBD03F9F
:1075700071D184A1814808F09BF8B0B1FEF7BEF943
:10758000012283498C20FDF7DFFF8148007830B16C
:1075900000230D227FA1184605F06EFF05E00023B1
:1075A0000F2280A1184605F067FF82A1734808F0FA
:1075B0007FF800287ED06421804808F06EF800260D
:1075C00080E036B97BA16D4808F072F80446A41D2E
:1075D00076E0641C7AA1204608F06AF8051E48D0BF
:1075E000012E06D0022E0ED0032E28D0042E3ED11E
:1075F00032E0744800210160416001812A1B21466C
:1076000008F032F800BF6F4861380021016580F84A
:1076100054102A1B2146503008F026F869481138CA
:10762000FEF702FA8046674861380021016580F85C
:107630005410424664A150300AF014FB18E00F21A8
:1076400060480A3008F029F82A1B21465D480A30B4
:1076500008F00AF80CE0FDE35A486138002180F890
:107660007A102A1B21467A3007F0FEFF00E000BFA7
:1076700000BF2C46042E23D1641C54A1204608F0E0
:1076800017F805464F48801F0021016081802A1BA2
:10769000214607F0E9FF4B48801FFEF7C5F98046F9
:1076A000B8F1010F01DA4FF001084648801F0021B0
:1076B000016000E0A8E08180424643A10AF0D2FACE
:1076C000701CC6B2052EFFF67CAF3E481138FEF79F
:1076D000ABF9012805DA3EA23FA13A4811380AF079
:1076E000C1FA6E2237495139684607F0BDFF7E2244
:1076F000344961391CA807F0B7FF1CA80FC8FEF772
:107700004AF800230B2235A1184605F0B5FE2D4995
:107710000DF2511007F0EFFFD0B92A49113950A8E6
:1077200007F0E9FFA0B927490A310DF25B1007F015
:10773000E2FF68B9234919310DF5B57007F0DBFF99
:1077400030B92049891F0DF24B1007F0D4FF48B122
:1077500001201C49613981F87C0001227C31B9206B
:10776000FDF71BFF1748613890F87A0031283DD1AA
:107770003AE00000004C00400008024084770020FE
:1077800070690020706172772D72737400000000C0
:10779000E4620020706172772D7273742C4F4B2C51
:1077A0002A000000706172772D7273742C66616913
:1077B0006C2C2A00706172772D3100000C6900205A
:1077C0002C000000CF650020256400002C2A00005A
:1077D0003030303031000000257300007061727766
:1077E0002D312C4F4B2C2A00FFF71CFCFE490DF5C8
:1077F000B57007F080FF38B1FB487A3890F87A000E
:10780000302801D1FFF774FCF8A1FA4807F050FFC7
:1078100010B14FF0010901E04FF00009F6A1F54861
:1078200007F046FF08B1012000E0002009EA000946
:10783000B9F1000F7DD000264EE036B9EBA1ED483E
:1078400007F036FF0446A41D44E0641CAFF290012B
:10785000204607F02DFF051E3BD0012E06D0022E3C
:1078600010D0032E1AD0042E31D123E01421DE488B
:107870007A3807F012FF2A1B2146DB487A3807F0D6
:10788000F3FE25E0D8487A38002141618161818387
:107890002A1B2146143007F0E7FE19E01421D248D4
:1078A0005C3807F0FAFE2A1B2146CF485C3807F007
:1078B000DBFE0DE0CC487A380021C1630164A0F8FA
:1078C00044102A1B21463C3007F0CEFE00E000BFEA
:1078D00000BF2C46701CC6B2052EAEDBC2487A38FB
:1078E000D4F80110C0F832106E2200F11001684681
:1078F00007F0BAFE7E22BC497A391CA807F0B4FE14
:107900001CA80FC8FDF747FF00230B22BBA1184698
:1079100005F0B2FDB4497A393CA807F0ECFED8B9BD
:10792000B149663941A807F0E6FEA8B9AE495C390D
:1079300000E01BE00DF5877007F0DDFE60B9AA4995
:107940003E394BA807F0D7FE30B9A74948390DF5A5
:10795000917007F0D0FE48B10120A3497A3981F82F
:107960007C0001227C31B920FDF717FEA6A1A148B9
:1079700007F09EFE18B3A6A19E4807F099FE041ECC
:1079800018D0A6480078C0F3801030B100230B2235
:10799000A3A1184605F070FD0CE0A448007820F083
:1079A00040004030A149087000230B229CA11846DA
:1079B00005F062FD9EA18F4807F07AFE04469FA164
:1079C0008C4807F075FE041E5FD064219D4807F0C7
:1079D00064FEE41D0D2221469A4807F045FE9948B1
:1079E0004079303897490979303901EB810100EB52
:1079F00041000C2801DD012100E000219148C079FF
:107A00003038904A9279303A02EB820200EB420021
:107A10001F2801DD012000E0002008438949497A40
:107A20003039884A127A303A02EB820201EB420185
:107A3000172901DD012100E0002108438149C97AAD
:107A40003039804A927A303A02EB820201EB4201ED
:107A50003B2901DD012100E0002108437949497BF0
:107A60003039784A127B303A02EB820201EB420154
:107A70003B2901DD012100E00021084330B1002352
:107A80000D2271A1184605F0F7FC1DE16D48407B01
:107A900030386C49097B303901EB810100EB410141
:107AA0006848C07A3038674A927A303A02EB8202EC
:107AB00000EB4200DFF88CC1CDE900019CF809C061
:107AC000ACF1300CDFF87C9199F80890A9F13009FD
:107AD00009EB89090CEB4903DFF868C19CF807C082
:107AE000ACF1300CDFF85C9199F80690A9F13009FF
:107AF00009EB89090CEB4902DFF848C19CF805C085
:107B0000ACF1300CDFF83C9199F80490A9F1300900
:107B100009EB89090CEB4901DFF828C19CF803C087
:107B2000ACF1300CDFF81C9199F80290A9F1300902
:107B300009EB89090CEB4900FEF7A3FE4148407BA5
:107B400030384049097B303901EB810100EB4100BD
:107B5000C1B23C48C07A30383A4A927A303A02EBA5
:107B6000820200EB4200C0B2DFF8D8C0CDE90001CC
:107B70009CF809C0ACF1300CDFF8C89099F8089077
:107B8000A9F1300909EB89090CEB490C0CF0FF0352
:107B9000DFF8B0C09CF807C0ACF1300CDFF8A4905F
:107BA00099F80690A9F1300909EB89090CEB490C09
:107BB0000CF0FF02DFF88CC09CF805C0ACF1300C73
:107BC000DFF8809099F80490A9F1300909EB890950
:107BD0000CEB490C0CF0FF01DFF868C09CF803C007
:107BE000ACF1300C38E00000E8650020706172777D
:107BF0002D3200008477002022000000706172772F
:107C00002D322C4F4B2C2A00706172772D330000DF
:107C1000706172772D332C310000000071620020FA
:107C2000706172772D332C4F4B2C2A000263002099
:107C3000706172772D332C30000000007061727714
:107C40002D3400000C690020706172772D342C6691
:107C500061696C2C2A000000DFF8149299F80290F8
:107C6000A9F1300909EB89090CEB490C0CF0FF0074
:107C700007F00CFC02227E49AA20FDF78EFC7D480D
:107C8000006800F4807020B1FDF701FF8146FEF727
:107C9000B5FF7848006800F4007030B1FDF7EEFEE3
:107CA000A0F101094846FEF7EEFE00230B2272A167
:107CB000184605F0E1FB0120724981F87C000122A1
:107CC0000021B920FDF769FC6FA1714807F0F0FCB5
:107CD000041E1DD0AFF21851204607F0E9FC0446FF
:107CE000641CA51C2978207807F0E8F8287807F0AC
:107CF0001DF9074637B900230B2266A1184605F087
:107D0000BBFB05E000230D2265A1184605F0B4FB7E
:107D100067A15F4807F0CCFC041E2DD064215448B5
:107D200007F0BBFC1CA8FDF7D0FC7E221CA955481F
:107D300007F09AFC53485B30FDF776FE81465148C8
:107D40005030FDF771FE82464E487A30A0F10F01A7
:107D50005346A0F11902CDE90109009156A144480A
:107D600009F080FF424807F0BFFC814600234A46E5
:107D70003F49184605F080FB55A1454807F098FC9F
:107D800018B364213A4807F088FC5CA95FA8FEF7A5
:107D900004FE3C49323101F10A00A0F11E02A0F1BB
:107DA0002803CDE90032CDE90201143B48A24AA1E3
:107DB0002F4809F057FF2E4807F096FC8146002314
:107DC0004A462B49184605F057FB48A1304807F0B2
:107DD0006FFC00B36421264807F05FFC5CA95FA834
:107DE000FEF7DBFD022261A9AA20FDF7ADFB5FA82B
:107DF0005CA961AB3DA2CDE900103EA11C4809F091
:107E000031FF1B4807F070FC814600234A461849A1
:107E1000184605F031FB3BA11D4807F049FC041E44
:107E20001FD06421124807F038FC07F015F8074608
:107E30007F2F10D03A4635A10D4809F013FF0C48AA
:107E400007F052FC814600234A460949184605F0CE
:107E500013FB06E007E000230E2230A1184605F0D0
:107E60000BFBFFF7E6FA002062B0BDE8F0870000E8
:107E70000C69002008280040706172772D342C4F67
:107E80004B2C2A006E650020706172772D35000042
:107E900084770020706172772D352C4F4B2C2A008F
:107EA000706172772D352C6661696C2C2A00000098
:107EB000706172722D310000706172722D312C254B
:107EC000732C25642C25732C25732C25642C2A00F7
:107ED000706172722D32000025732C25732C25736E
:107EE0002C25732C25732C25732C2A00706172723B
:107EF0002D34000025732C257325732C25732C2A13
:107F000000000000706172722D733F004164647262
:107F10006573733A25632C2A000000004164647283
:107F20006573732C6661696C2C2A000010B588B0EB
:107F3000044601210805F9F707F801210C20F8F79C
:107F4000E1FF6A48FAF74AFF4FF48050029002209E
:107F50008DF80C008DF80D0000208DF80E0001202A
:107F60008DF80F0002A96248F8F7F0FC0420029097
:107F700002208DF80C008DF80D0000208DF80E0009
:107F800001208DF80F0002A95A48F8F7DFFC0822FB
:107F90000C215748F8F763FD082202215548F8F7ED
:107FA0005EFD04940020ADF81400ADF81600ADF8A5
:107FB0001800ADF81C000C20ADF81A0004A94B48BD
:107FC000FAF74FFF01214948FAF7D0FF012240F2AA
:107FD00025514648FBF780F831208DF80400032036
:107FE0008DF8050000208DF8060001208DF80700AF
:107FF00001A8F8F7B8F840213C48FBF79FF808B013
:1080000010BD10B53C48B0F864006FF30E003A495B
:10801000A1F864000846B0F8640020F40040A1F81C
:1080200064006421344807F038FBC821334807F066
:1080300034FB10BD10B540F225512C48FBF787F8F2
:10804000C8B12A48FAF7C1FFC4B22B48B0F864009F
:10805000C0F30E0063280EDA2749B1F86410C1F3AB
:108060000E00411C244AB2F8642061F30E0222493A
:10807000A1F864200C5440F224411C48FBF767F837
:1080800001280DD11C48B0F8640020F4004000F530
:1080900000401949A1F864001448FAF796FFC4B2E9
:1080A00010BD0FB438B505A800901448009A049983
:1080B00009F0ECFD00200090104807F015FB85B298
:1080C00000240DE000BF40210848FBF72AF80028F3
:1080D000F9D00A48015D0548FAF773FF601C84B2C5
:1080E000AC42EFDB38BC5DF814FB000000500040F0
:1080F00000080240000C0240706B0020D66B00208C
:108100001CB501210220F8F7FDFE01208DF80400C6
:108110008DF806008DF8070002208DF805004FF459
:10812000407000906946A248F8F710FC4FF4407187
:108130009F48F8F785FC1CBD10B59E48006820F4E8
:1081400040209C4908600846006840F48020086090
:1081500049159748F8F774FC0120FCF760F94FF4D3
:1081600080719348F8F76CFC0620FCF758F94FF43F
:1081700000718F48F8F766FC0620FCF750F94FF4C1
:1081800080718B48F8F75EFC0220FCF748F910BDBF
:1081900010B58848006820F44020864908600846E9
:1081A000006840F48020086089158148F8F74AFC8F
:1081B0004FF400717E48F8F745FC0520FCF72FF9D5
:1081C0004FF480717A48F8F73BFC0120FCF727F95F
:1081D0004FF400717648F8F733FC0520FCF71FF9DF
:1081E00010BD10B500247348006820F44020714988
:1081F000086049156E48F8F723FC0120FCF70FF9D9
:108200004FF480716A48F8F71BFC0120FCF707F96E
:1082100009E00120FCF703F9641CFA2C03D9FFF7ED
:10822000B7FF012010BD4FF400716148F8F7F0FB73
:108230000028EED14FF480715D48F8F703FC002070
:10824000F0E710B54FF480715948F8F7FBFB594837
:10825000006820F44020574908600846006840F450
:108260008020086049155248F8F7ECFB0220FCF723
:10827000D6F84FF480714E48F8F7E2FB0220FCF785
:10828000CEF84FF480714A48F8F7DCFB10BD10B50A
:108290004FF480714648F8F7D5FB4648006820F453
:1082A0004020444908600846006840F48020086087
:1082B00049153F48F8F7C4FB0220FCF7B0F84FF42B
:1082C00080713B48F8F7BCFB0220FCF7A8F84FF49C
:1082D00080713748F8F7B6FB10BD70B504463548D5
:1082E000006820F44020334908600846006840F4E4
:1082F0008020086089152E48F8F7A4FB002523E0AC
:10830000E00928B14FF400712948F8F799FB04E01F
:108310004FF400712648F8F795FB6006040E022022
:10832000FCF77DF84FF480712148F8F789FB0220B3
:10833000FCF775F84FF480711D48F8F783FB0220B5
:10834000FCF76DF8681CC5B2082DD9DB70BD70B59F
:10835000054600241748006820F4402015490860AD
:1083600000261BE04FF480711148F8F76BFB0220E8
:10837000FCF755F84FF480710D48F8F761FB600683
:10838000040E4FF400710A48F8F742FB08B1601C74
:10839000C4B20120FCF743F8701CC6B2082EE1DB22
:1083A00015B9FFF774FF01E0FFF74BFF204670BDE2
:1083B000000402400008024070B586B004460D4635
:1083C0001646FCA32246FDA1684609F04BFC01229B
:1083D000FCA1FD4802F0BEFD13222146FB4802F03D
:1083E000E4FDFA48C16803F095F905AB3246294629
:1083F000F64802F0EBFFF54803F02FF90022F1A157
:10840000104602F0A7FD06B070BD70B58AB0002519
:10841000142105A807F041F9002003900490019071
:1084200002906946F9F7A8F801A903A8FEF7B5FA82
:10843000E74B01AAE7A105A809F014FC0122E1A17C
:10844000E14802F087FD022205A9E04802F0ADFDF7
:108450000446042C05D0DE48503890F87C000128F2
:108460007ED1DA4803F0F9F8132205A9D74802F0C3
:108470009CFDD648C16803F04DF9D94B0D22D9A116
:10848000D24802F0A3FFD248113007F02DF906467A
:10849000D34B3246CE491131CC4802F097FFD04B36
:1084A0000222D4A1C94802F091FFCD4B0722D2A1EC
:1084B000C64802F08BFFC648503807F015F906464B
:1084C000C74B3246C2495039C04802F07FFFC44B07
:1084D0000222C8A1BD4802F079FFC14B0922C8A100
:1084E000BA4802F073FFBA483C3807F0FDF8064678
:1084F000BB4B3246B6493C39B44802F067FFB84B33
:108500000222BCA1B14802F061FFB54B0A22BFA113
:10851000AE4802F05BFFAE48323807F0E5F8064699
:10852000AF4B3246AA493239A84802F04FFFAC4B54
:108530000222B0A1A54802F049FFA94B0922B6A129
:10854000A24802F043FFA248143807F0CDF80646CF
:10855000A34B32469E4914399C4802F037FF00E095
:1085600085E09F4B0222A3A1984802F02FFF9C4B6D
:108570000A22ACA1954802F029FF95481E3807F061
:10858000B3F80646964B324691491E398F4802F0A1
:108590001DFF934B022297A18C4802F017FF904BCE
:1085A0001122A3A1894802F011FF894807F09CF825
:1085B00006468B4B32468649844802F007FF884BBB
:1085C00002228CA1814802F001FF854B0D229DA162
:1085D0007E4802F0FBFE7E480B3007F085F8064629
:1085E0007F4B32467A490B31784802F0EFFE7C4BE4
:1085F000022280A1754802F0E9FE794B112295A173
:10860000724802F0E3FE72481B3007F06DF8064630
:10861000734B32466E491B316C4802F0D7FE704BEB
:10862000022274A1694802F0D1FE6D4B0D228EA189
:10863000664802F0CBFE66482A3007F055F8064639
:10864000674B324662492A31604802F0BFFE644BF4
:10865000022268A15D4802F0B9FE614B4FF4C87276
:1086600085495A4802F0B2FE584802F0F6FF13223C
:1086700005A9564802F099FC04463CB3002514E0D5
:10868000681CC5B2514802F0E8FF00224DA1104617
:1086900002F060FC01224BA14B4802F05BFC13226C
:1086A00005A94A4802F081FC04460CB1012000E013
:1086B0000020642D01DA012100E00021084000289B
:1086C000DED1622D02DD05200AB070BD3F48C168D1
:1086D00003F020F8694807F007F80646404B324699
:1086E00066493A4802F072FE3D4B022241A13748EA
:1086F00002F06CFE354802F0B0FF3548503890F873
:108700007C00012807D03248503890F87D009DF851
:10871000021088424DD000202D49503981F87C004C
:1087200001220021B920FCF738FF01220DF10201DE
:10873000BA20FCF732FF132251A1244802F035FC85
:108740002248C16802F0E6FF254B0D2225A11F48F3
:1087500002F03CFE1E48113006F0C6FF0646204BD4
:1087600032461B491131194802F030FE1C4B0222DF
:1087700020A1164802F02AFE194B07221EA1134819
:1087800002F024FE1248503806F0AEFF0646144BA5
:1087900032460F4950390D4802F018FE104B0222A4
:1087A00014A10A4802F012FE0D4B092214A1074839
:1087B0006CE03EE12E747874000000002573257390
:1087C00000000000303A0000E0730020B07100208B
:1087D000BE65002025735F25732E74787400000039
:1087E0000C63002045717569706D656E745F494456
:1087F0003A0000000D0A00005443505F49703A00EF
:108800005443505F506F72743A00000057696669B4
:108810005F535349443A0000576966695F50776473
:108820003A000000576966695F506F72743A000041
:108830004D6561737572655F496E74657276616CC2
:108840003A0000005075625F496E74657276616C23
:108850003A0000004170706F696E746D656E745FF0
:1088600054696D653A0000004D6561737572655F0E
:108870004D6F64653A000000183B0208E06D00206F
:10888000424332352E7478740000000002F09EFDE1
:10889000FA4806F029FF0646F94B3246F749F948EF
:1088A00002F094FDF64B0222AFF2B801F54802F057
:1088B0008DFDF34B0A22AFF2AC01F24802F086FDC7
:1088C000EE480A3006F010FF0646ED4B3246EB4903
:1088D0000A31EC4802F07AFDE94B0222AFF2EC01DA
:1088E000E84802F073FDE64B0922AFF2D401E548F7
:1088F00002F06CFDE148283006F0F6FE0646E04B3B
:108900003246DE492831DF4802F060FDDC4B0222AE
:10891000AFF22011DB4802F059FDD94B0A22AFF229
:10892000FC01D84802F052FDD4481E3006F0DCFEAF
:108930000646D34B3246D1491E31D24802F046FD9D
:10894000CF4B0222AFF25411CE4802F03FFDCC4B88
:108950001122AFF22411CB4802F038FDC7483C3059
:1089600006F0C2FE0646C64B3246C4493C31C548F5
:1089700002F02CFDC24B0222AFF28811C14802F076
:1089800025FDBF4B0D22AFF24411BE4802F01EFD83
:10899000BA48473006F0A8FE0646B94B3246B749FA
:1089A0004731B84802F012FDB54B0222AFF2BC11BC
:1089B000B44802F00BFDB24B1122AFF26811B1487E
:1089C00002F004FDAD48573006F08EFE0646AC4B73
:1089D0003246AA495731AB4802F0F8FCA84B0222B4
:1089E000AFF2F011A74802F0F1FCA54B0D22AFF257
:1089F0008811A44802F0EAFCA048663006F074FE34
:108A000006469F4B32469D4966319E4802F0DEFC89
:108A10009B4B0222AFF224219A4802F0D7FC984BDC
:108A20004FF4C8729849974802F0D0FC954802F07C
:108A300014FE1322AFF2B811924802F0B6FA0446BF
:108A40002CB3002510E0681CC5B28E4802F005FE6C
:108A50000122AFF290218D4802F07CFA132205A981
:108A6000884802F0A2FA04460CB1012000E0002080
:108A7000642D01DA012100E0002108400028E2D144
:108A8000622D04DD82A0FFF70CFB05201CE6BCB9BB
:108A90007C48C16802F03EFE834806F025FE06468B
:108AA000774B32468049774802F090FC744B0222A3
:108AB000AFF2C021734802F089FC724802F0CDFD8C
:108AC0000022AFF20031104602F044FA0020FBE52C
:108AD00010B50122AFF214316C4802F03BFA1322B8
:108AE00072A1684802F061FA6648C16802F012FE9D
:108AF000634B4FF4DC727049624802F067FC6A48CD
:108B000006F0F2FD04465E4B224667495D4802F0DE
:108B10005DFC5B4B0222AFF224315A4802F056FC56
:108B2000584802F09AFD0122AFF26831002002F0AD
:108B300011FA10BD3EB5044600200090019002904D
:108B40005BA32246AFF28C31684609F08BF8012214
:108B5000AFF290314D4802F0FDF9684603F0D1F8CC
:108B60000546484802F079FD15B954A0FFF799FA77
:108B70000022AFF2B031104602F0ECF928463EBDBB
:108B800070B586B004464AA32246AFF2D03101A8A0
:108B900009F068F80122AFF2D4313C4802F0DAF96A
:108BA0000646012249A1374802F0FFF906462EB1D8
:108BB00049A0FFF776FA042006B070BD3148C568B9
:108BC00002F04BFD06460022AFF20841104602F0CB
:108BD000C1F92846F0E72DE9F74FBCB08B461446A3
:108BE00000203B904348007910B93FB0BDE8F08FBA
:108BF00001223BA9B420FCF7C3FC3B98A04201D959
:108C000000203B903CA03B99FFF74BFA28A3AFF222
:108C1000544138A83C9A09F025F83B98201AC821FD
:108C2000B0FBF1F93B98201AB0FBF1F201FB1208FE
:108C3000494636A0FFF735FA414639A0FFF731FA29
:108C4000D82102A806F029FD3A48006807F078FB11
:108C500000F0400018B140F6B83007F04DFB01229B
:108C6000AFF2A041094802F075F98246012238A905
:108C7000044802F09AF9824600266EE082650020E0
:108C80000C630020B0710020183B0208E073002044
:108C90006F70656E20424332352E747874206661A1
:108CA000696C0D0A00000000E06D002074657374AB
:108CB0002E74787400000000AC3C020864656C659A
:108CC000746520737563657373000000303A2F423A
:108CD0004332352E747874006F70656E2062633293
:108CE000357478742073697A65206661696C0D0A41
:108CF000000000001B63002074665F73656E647083
:108D00006F733A256C640D0A000000006C656E7389
:108D10005F71756F7469656E743A256C640D0A0035
:108D20006C656E5F72656D61696E6465723A256C23
:108D3000640D0A00AC620020E14802F08EFC82461D
:108D40000122AFF28051DF4802F004F9824601228D
:108D500038A9DB4802F029F98246BAF1000F01D0A8
:108D6000012000E00020642E01DA012100E0002152
:108D700008400028E0D13B980BEB0001D04802F0FE
:108D8000C9FC0027C3E0D048006807F0D9FA00F01A
:108D9000400000286FD04021CB48006807F0BEFAA1
:108DA000CAA0FFF77EF9C64802F057FC8246802130
:108DB000C548006807F0EEFA41F28833012211023B
:108DC000C148006807F00CFBBD4802F046FC824633
:108DD000C1A0FFF7D5FE04462146C1A0FFF761F907
:108DE00009E0BDA0FFF7CCFE04462146BCA0FFF77A
:108DF00058F9701CC6B20A2C01D2012000E00020F4
:108E0000322E01DA012100E0002108400028E8D1DB
:108E10003B98201AC821B0FBF1F9B9443B98201ABD
:108E2000B0FBF1F201FB12083946B2A0FFF739F9A5
:108E30004946B2A0FFF735F94146B5A0FFF731F931
:108E40000122AFF280619F4802F084F8012238A924
:108E50009B4802F0AAF88246002607E0012238A9C2
:108E6000974802F0A2F88246701CC6B2BAF1000F11
:108E700002D0012001E018E00020642E01DA012177
:108E800000E0002108400028E8D1BAF1000F05D029
:108E900001223BA9B420FCF7E6FBA6E688483B99F3
:108EA00002F038FC9FA0FFF7FCF8C922A1A102A89C
:108EB00008F0D8FE02A806F017FC85B202A84119F6
:108EC0009E4BC8227E4802F0ABF9824602A9294493
:108ED00001F1C8009AA108F0C5FE002602A806F01C
:108EE00003FC02A9019003F008FF20B195A03B9973
:108EF000FFF7D7F879E699A0FFF7D3F83B98C83089
:108F00003B9001223BA9B420FCF7ADFB7F1C4F45F1
:108F1000FFF439AF08F1010295A102A808F0A2FE02
:108F200002A806F0E1FB85B202A84119834B424634
:108F3000634802F075F905EB080085B202A94819EB
:108F40007FA108F08FFE02A98CA0FFF7AAF802A863
:108F500006F0CAFB02A9019003F0CFFE40B18BA03E
:108F6000FFF79FF801223BA9B420FCF77CFB3CE60D
:108F700000203B9001223BA9B420FCF774FB504831
:108F800002F06BFB82460122AFF2C8714D4801F03E
:108F9000E1FF51A0FFF7CEFD00BF26E610B58CB073
:108FA0007F4840797E4909797D4AD2787C4B9B780D
:108FB000CDE90632CDE90810794841780278794840
:108FC0004078784B1B78CDE90230CDE90421754813
:108FD000407974490979CDE900107248C3788278E4
:108FE00071A1794808F03EFE784AA2F11E00A0F176
:108FF0001E01A0F13C03CDE90731CDE909025A3841
:109000005A39B43A783BCDE90332CDE905103C3A00
:109010006D482830A0F10A016B4BCDE901020091A7
:109020006B4A6CA1A0F5077008F01CFE734806F0AF
:109030005BFB841C224640A1714808F013FE0CB073
:1090400010BD2DE9FC4781460C4615464FF42F70A4
:109050000AF01EF8019000200090002780460122AF
:1090600068A1019801F076FF064601AA694665A04D
:1090700002F070FD0646B6B90198C069801E0199DC
:10908000498900FB01F801984089009900FB01F72C
:109090004FEA58002060780828602068800A206025
:1090A0002868800A2860012256A1002001F052FFA2
:1090B0000646019809F0C4FF3046BDE8FC87000071
:1090C000B0710020E0730020AC62002042433235D2
:1090D00020574149540D0A00424332350000000038
:1090E0007365636F6E642D6C656E3A256C640D0A52
:1090F00000000000693D25640D0A00006C656E7378
:109100005F71756F7469656E743D25640D0A0000AA
:109110006C656E5F72656D61696E6465723D256434
:109120000D0A00004243323520726573756D0D0AD9
:10913000000000005075622C25642C000C63002098
:109140002C2A0000626332352073656E64206661EC
:10915000696C3A256C640D0A0000000062633235C8
:109160002073656E64202E2E2E2E2E0D0A00000018
:109170005075622C256C642C0000000072656D61D6
:10918000696E6465723A25730D0A000072656D613F
:10919000696E646572206661696C0D0A00000000EA
:1091A000FB630020EC630020256325632F256325E6
:1091B000632F32302563256320256325633A2563B9
:1091C00025633A2563256300D46F0020157A0020BB
:1091D000CF65002025732C25732C257325732573EB
:1091E0002C25732C25732C25732C25732C25732C7F
:1091F00025732C25732C257300000000E06D0020E2
:109200008C7100203000000010B50446204609F0A3
:109210003FFF10BD10B50446204609F011FF10BDF8
:1092200010B502460020404B802A01D290B213E0D4
:10923000B2F5803F10D240F2B514A1420CD100200B
:1092400001E0441CA0B2802803DA33F810409442B5
:10925000F7D100F18004E0B210BD10B50246002045
:10926000314B802A01DA104609E040F2B514A142E0
:1092700005D1FF2A03DCA2F1800433F8140010BDED
:1092800070B5B0F5803F4DD281B2B1F5805F01DAA3
:10929000264E00E0264E324600BF32F8023B0BB1AC
:1092A000994200DA3CE032F8024B2512E4B21E1972
:1092B0008E4230DD092D2CD2DFE805F005090F13B1
:1092C000171B1F232700CE1A32F8161021E0CE1AE2
:1092D00006F001068E1BB1B21BE0A1F11006B1B27F
:1092E00017E0A1F12006B1B213E0A1F13006B1B24E
:1092F0000FE0A1F11A06B1B20BE001F10806B1B21C
:1093000007E0A1F15006B1B203E0A1F5E356B1B216
:1093100000BF00BF04E0002DBFD102EB4402BCE758
:1093200000BF084670BD00009C3302089C34020850
:109330008E36020870B5044600255CB9FBF7EFFED7
:10934000054635B1FBF7BAFDFF20FBF7B1FDFBF792
:10935000BAFD00BF00BF0DB1012070BD0020FCE7C9
:1093600070B50446002514B1012C0DD10BE0FBF7BC
:10937000D6FE054635B1FBF7A1FDFF20FBF798FDB2
:10938000FBF7A1FD02E001E0012500BF00BF0DB128
:10939000012070BD0020FCE72DE9F04105460E4696
:1093A00017461C464FF0000814B90420BDE8F081B0
:1093B00015B1012D14D110E0E2B239463046FBF769
:1093C0006FFF8046B8F1000F06D0FBF777FDFF2056
:1093D000FBF76EFDFBF777FD05E04FF0000802E0BC
:1093E0004FF0010800BF00BFB8F1000F01D100200D
:1093F000DCE70120DAE72DE9F04105460E46174685
:109400001C464FF0000814B90420BDE8F08115B1E6
:10941000012D08D106E0E2B239463046FBF77DFF68
:10942000804603E002E04FF0010800BF00BFB8F142
:10943000000F01D10020E8E70120E6E72DE9F04127
:1094400006460F4615463EBB37B1012F1CD0022FF2
:1094500011D0032F1DD113E040212D48F7F7F2FA68
:10946000FBF745FD08B9002400E00124402128480D
:10947000F7F7E6FA0FE04FF40070288000240AE0C6
:1094800008202880002406E0FBF70EFE2860002458
:1094900001E0042400BF15E0012E12D137B1012FE5
:1094A0000AD0022F04D0032F08D103E0002407E0E4
:1094B000002405E0002403E0002401E0042400BFB0
:1094C00000E001242046BDE8F0811CB501A9002080
:1094D000F7F7B8FF69460020F8F74EF89DF803004B
:1094E000143040069DF8011040EA41509DF80210EA
:1094F00040EA01409DF8041040EAC1209DF80510A3
:1095000040EA41109DF8061040EA61001CBD0000D1
:1095100000080240014648780A7842EA0020704775
:109520000146C8788A7842EA00204A7842EA002058
:109530000A7842EA0020704700F8011B091200F87F
:10954000011B704700F8011B090A00F8011B090AFA
:1095500000F8011B090A00F8011B7047014609B118
:10956000002070470020FCE7014609B10020704749
:109570000020FCE72DE9F0410646356815F8014B5F
:109580002046FFF7EBFF60B115F8017B3846FFF787
:10959000EBFF18B94FF0FF30BDE8F08107EB042076
:1095A00084B24CB140F2B5112046FFF756FE044696
:1095B00014B94FF0FF30EFE7A04635604046EBE7C7
:1095C0002DE9F04107460C46164640F2B5113846E3
:1095D000FFF726FE0546FF2D0BDD022E02D20020EE
:1095E000BDE8F081281204F8010B04F8015B0220A9
:1095F000F6E705B10EB90020F2E704F8015B01209F
:10960000EEE730B502460B46002400211CE0FA4884
:1096100000EB01100068A8B1F74800EB01100068EA
:109620001568A8420FD1F44800EB01104068956816
:10963000A84208D1F04800EB011080685569A842A3
:1096400001D103E00124491C0229E0D300BF022913
:1096500006D11CB9022B01D0122030BD0020FCE73E
:1096600033B9E54800EB01108089B0F5807F01D166
:109670001020F2E70020F0E7002100E0491C022959
:1096800005D2DD4800EB011000680028F6D1022960
:1096900001D0012070470020FCE710B502460B46C0
:1096A000002116E0D44800EB011000681468A042C5
:1096B0000ED1D14800EB011040689468A04207D158
:1096C000CD4800EB011080685469A04200D102E04F
:1096D000491C0229E6D300BF022922D1002100E063
:1096E000491C022905D2C44800EB0110006800287B
:1096F000F6D1022901D1002010BDBF4C04EB0114AA
:1097000010682060BC4C04EB011490686060BA4C97
:1097100004EB01145069A0600020B74C04EB011465
:10972000A081012B06DBB44800EB0110808908B151
:109730000020E1E713B14FF4807004E0AE4800EB85
:1097400001108089401CAC4C04EB0114A081481C22
:10975000D2E710B50246531E1A46022B17D2A64B6B
:1097600003EB02139989B1F5807F00D10021002914
:1097700001DD4B1E99B2A04B03EB0213998121B975
:1097800000239D4C04EB02142360002000E0022023
:1097900010BD014600200BE0974A02EB0012126850
:1097A0008A4204D10022944B03EB00131A60401C40
:1097B0000228F1D3704770B504460025E078E8B17F
:1097C0006078012304F13801626BFFF714FEA0B941
:1097D0000020E070A16A606B401A216A88420DD2B5
:1097E000A07802280AD1236A616BCA186078012325
:1097F00004F13801FFF7FFFD00E00125284670BDA8
:1098000070B504460D460026606BA84210D0204675
:10981000FFF7D1FF06465EB9607801232A4604F1BE
:109820003801FFF7B9FD10B14FF0FF350126656330
:10983000304670BD70B504462046FFF7BCFF0546B4
:10984000002D37D1207803282DD1207901282AD165
:10985000410204F1380005F020FF4AF6552104F2D8
:109860003620FFF769FE654904F13800FFF76AFE0C
:10987000634904F50770FFF765FE04F50870616938
:10988000FFF760FE04F509702169FFF75BFE606A6F
:10989000401C60636078012304F13801626BFFF7BC
:1098A000AAFD00202071607800221146FFF7C6FD56
:1098B00000B10125284670BD0246891ED069801E70
:1098C000884201D8002070475389106B03FB0100C8
:1098D000F9E72DE9F04781460C46D9F80050022CF3
:1098E00002D3E869A04202D84FF001085EE04FF0D1
:1098F000FF382878012804D002282CD0032851D121
:109900003CE0264606EB5606A86A00EB56212846A0
:10991000FFF776FF00B148E03046761CC0F308013F
:1099200005F13800475CA86A00EB56212846FFF78E
:1099300067FF00B139E0C6F3080105F13800405C6B
:1099400047EA002704F0010008B1380901E0C7F335
:109950000B00804629E0A86A00EB14212846FFF797
:109960004FFF00B121E040F2FF1101EA440205F18E
:1099700038015018FFF7CEFD804616E0A86A00EBCC
:10998000D4112846FFF73CFF00B10EE040F2FF1172
:1099900001EA840205F138015018FFF7C1FD20F0FB
:1099A000704802E04FF0010800BF00BF4046BDE82C
:1099B000F0872DE9F04704460D4616464FF00209A0
:1099C000022D70D3E069A8426DD92078012804D017
:1099D000022850D003280DD166E02F4607EB570729
:1099E000A06A00EB57212046FFF70AFF8146B9F134
:1099F000000F07D07CE000006477002052526141E4
:109A00007272416138467F1CC0F3080104F13800CE
:109A100001EB000805F0010028B1F1B298F8000050
:109A200061F31F1000E0304688F800000120E0706C
:109A3000A06A00EB57212046FFF7E2FE8146B9F10C
:109A4000000F00D054E0C7F3080104F1380001EB27
:109A5000000805F0010010B1C6F3071006E098F801
:109A6000000000F0F000C6F30321084388F800006E
:109A70000120E0703CE0A06A00EB15212046FFF7D2
:109A8000BFFE8146B9F1000F00D031E0B1B240F223
:109A9000FF1202EA450304F138029818FFF74CFD63
:109AA0000120E07024E024E0A06A00EBD5112046FC
:109AB000FFF7A6FE8146B9F1000F00D018E040F292
:109AC000FF1101EA850204F138015018FFF728FD63
:109AD00066F31B00064640F2FF1101EA850204F11D
:109AE000380150183146FFF72DFD0120E07000BF0E
:109AF00000BF4846BDE8F0872DE9F04781460E4695
:109B000017464FF00008D9F80040022E02D3E06952
:109B1000B04202D80220BDE8F08767B100BF4FF025
:109B2000FF3239462046FFF744FF8046B8F1000F68
:109B300001D04046EFE700BF31464846FFF7C9FE77
:109B4000054605B922E0012D01D10220E3E7681C9A
:109B500008B90120DFE7002231462046FFF729FF40
:109B60008046B8F1000F01D04046D4E7E069801E7E
:109B70006169814206D26069401C6061207940F0D1
:109B8000010020712E46E069B042D5D800BF002008
:109B9000C1E72DE9F04782468846DAF80040B8F17F
:109BA000000F06D1276917B1E069B84215D801271F
:109BB00013E041465046FFF78CFE0546022D02D2C7
:109BC0000120BDE8F087681C08B92846F9E7E0697C
:109BD000A84201D92846F4E74746606908B9002041
:109BE000EFE70026474518D17E1CE069B04200D857
:109BF000022631465046FFF76CFE0546012D01D086
:109C0000681C08B92846DCE73DB12569022D03D35D
:109C1000E069A84200D92F460026E6B93E4600BFBB
:109C2000761CE069B04204D80226BE4201D9002069
:109C3000C7E731465046FFF74CFE054605B909E037
:109C4000012D01D0681C08B92846BAE7BE42E7D109
:109C50000020B6E700BF4FF0FF3231462046FFF745
:109C6000A8FE8146B9F1000F08D1B8F1000F05D068
:109C7000324641462046FFF79CFE8146B9F1000F6F
:109C80000DD12661E069801E6169814202D8606958
:109C9000401E6061207940F00100207107E0B9F1B9
:109CA000010F02D14FF0FF3000E0012006463046A0
:109CB00087E7F0B503460D461E68D86A021D680A9C
:109CC0007789B0FBF7F400BF02CA09B90020F0BDE4
:109CD0008C4200D202E0641A121DF5E700BF106842
:109CE0002044F4E72DE9F047044689462046FFF773
:109CF00062FD10B10120BDE8F08749462046FFF71C
:109D0000DBFD074667634FF4007104F1380005F08E
:109D1000C4FC60894FF40041B1EB402F01D80846E4
:109D200001E06089400206464FF0000800E0760836
:109D3000B6F5007F05D93046FFF766FAB0F10008A6
:109D4000F5D0B6F5007F16D93146404605F0A5FCA2
:109D5000760A002500E035446089A84207D97A19BF
:109D6000607833464146FFF746FB0028F3D0404673
:109D7000FFF750FA10E004F138080126002500E052
:109D800035446089A84207D97A196078334641463C
:109D9000FFF731FB0028F3D06089A84201D00120F1
:109DA000A9E70020A7E72DE9F04104460D46266803
:109DB000B5F5001F02D205F01F0010B10220BDE86A
:109DC000F0816561A7681FB93078032800DBF76A66
:109DD00047B93089B0EB551F01D80220EFE7F06A90
:109DE000E0611CE070894FEA402811E039462046C6
:109DF000FFF76FFD0746781C08B90120DFE7022F47
:109E000002D3F069B84201D80220D8E7A5EB0805D3
:109E10004545EBD239463046FFF74EFDE061A7617C
:109E2000E06908B90220CAE7E06900EB5520E0616B
:109E3000C5F3080106F13800084420620020BEE79F
:109E40002DE9F041044688462768606900F1200644
:109E5000B6F5001F01D30020E061E06910B90420CD
:109E6000BDE8F081C6F30800002845D1E069401C38
:109E7000E061A06938B93889B0EB561F3CD80020A2
:109E8000E0610420ECE77889401E00EA562098BB88
:109E90002046A169FFF71DFD0546012D01D80220CE
:109EA000DEE7681C08B90120DAE7F869A8421DD886
:109EB000B8F1000F03D10020E0610420D0E7204674
:109EC000A169FFF766FE05460DB90720C8E7012D19
:109ED00001D10220C4E7681C08B90120C0E7294667
:109EE0003846FFF7FFFE08B10120B9E7A561294612
:109EF0003846FFF7E1FCE0616661C6F3080107F14F
:109F00003800084420620020AAE72DE9F041044609
:109F10000E46D4F8008000212046FFF744FF054696
:109F2000EDB9002700BF4046E169FFF769FC05462F
:109F300005B113E0206A0078E52802D0206A007895
:109F400020B9781C0746B04201D107E00027012163
:109F50002046FFF775FF0546002DE4D000BF042D15
:109F600000D107252846BDE8F08170B505460C46AE
:109F700004F11A00FFF7CEFA06462878032805D127
:109F800004F11400FFF7C6FA46EA0046304670BDF9
:109F900070B506460C461546A9B204F11A00FFF743
:109FA000CBFA3078032804D1290C04F11400FFF710
:109FB000C3FA70BD2DE9F04780460C4604F11A0043
:109FC000FFF7A8FA10B10020BDE8F087207800F074
:109FD0003F00401E00EB800101EBC0054FF001097E
:109FE000002621E0FA49895D0819FFF793FA074630
:109FF000B9F1000F11D0FF2D0BD83846FFF740F90B
:10A00000824629466D1C38F81100FFF739F9824560
:10A0100001D00020D8E7B94605E04FF6FF7087422F
:10A0200001D00020D0E7761C0D2EDBD3207800F085
:10A03000400038B1B9F1000F04D038F8150008B16C
:10A040000020C1E70120BFE72DE9F04780460C461C
:10A0500004F11A00FFF75EFA10B10020BDE8F087A6
:10A06000207820F04000401E00EB800101EBC0058D
:10A070004FF00109002619E0D549895D0819FFF75D
:10A0800049FA0746B9F1000F09D0FF2D01D9002088
:10A09000E4E7B94628466D1C28F8107005E04FF635
:10A0A000FF70874201D00020D8E7761C0D2EE3D345
:10A0B000207800F0400048B1B9F1000F06D0FF2D24
:10A0C00001D90020CAE7002028F815000120C5E7C3
:10A0D0002DE9F04707460C461546984684F80D8052
:10A0E0000F20E07200202073002104F11A00FFF716
:10A0F00023FA681E00EB800101EBC0090020064630
:10A10000824600BF4FF6FF70864204D0484609F1F0
:10A11000010937F81060AE4911F80A1008193146E4
:10A12000FFF70AFA0EB94FF6FF760AF101008246F0
:10A130000D28E7D34FF6FF70864202D037F819009A
:10A1400008B945F040052570BDE8F0872DE9FF4FBF
:10A1500083B0074691461E460498016839604168FD
:10A16000796001893981807AB872052E19D9B04693
:10A1700012E039F802BB00240CE0584668F35F0097
:10A1800080464FEA6B0B08F4803010B1914888EAA2
:10A190000008641C102CF0D3B9F800000028E8D1A6
:10A1A0004646072400BF06F00F0000F1300A3609CA
:10A1B000BAF1390F03DD0AF1070000F0FF0A20466B
:10A1C000641E01A901F800A00CB1002EEBD17E2085
:10A1D00001A90855002509E0785DFFF7BFF920B116
:10A1E000601EA84200D106E06D1C6D1CA54202D283
:10A1F000785D2028F0D100BF00BF082C04D2204693
:10A20000641C01A9085C00E0202029466D1C7854DC
:10A21000082DF2D307B0BDE8F08F30B5014600201D
:10A220000B2200BF431003EBC01411F8015B63194C
:10A23000D8B2531E1A1EF5D130BD2DE9F05F044689
:10A2400089460426D4F800A04FF0FF08C34653E027
:10A250005046E169FFF7D4FA064606B14FE0206A9E
:10A2600005780DB904264AE0206AC07A00F03F075D
:10A27000A771E52D0AD02E2D08D027F02000082840
:10A2800001D1012000E00020484502D04FF0FF0836
:10A290002BE00F2F1DD105F0400038B1206A90F857
:10A2A0000DB005F0BF05A8466069206345450CD197
:10A2B000206A407B584508D1216ADAF80C00FFF784
:10A2C000C3FE10B1A8F1010000E0FF2000F0FF087C
:10A2D0000BE0B8F1000F04D1206AFFF79EFF58454C
:10A2E00002D04FF0FF30206309E000212046FFF745
:10A2F000A7FD064606B102E0E0690028A8D100BF2C
:10A300000EB10020E0613046BDE8F09F2DE9F04736
:10A310000446D4F800A000212046FFF744FD06467D
:10A3200016B13046BDE8F0874FF0FF08C1464FF048
:10A33000FF30206300BF5046E169FFF761FA06462F
:10A3400006B162E0206A05780DB904265DE0206A56
:10A35000C07A00F03F07A771E52D04D007F0080090
:10A3600038B10F2F05D04FF0FF084FF0FF302063BA
:10A3700044E00F2F22D12F20005D00F0400030BBC1
:10A3800005F0400038B1206A90F80D9005F0BF0547
:10A39000A8466069206345450CD1206A407B48454A
:10A3A00008D1216ADAF80C00FFF704FE10B1A8F119
:10A3B000010000E0FF2000F0FF081FE0B8F1000FEF
:10A3C0000AD1206AFFF729FF484505D11DE015E0B5
:10A3D0004C370208211001002F20005D00F0010021
:10A3E00038B90B2204F12401206A05F092F900B972
:10A3F0000BE04FF0FF084FF0FF30206300212046B4
:10A40000FFF71EFD0646002E95D000BF304689E7B7
:10A410002DE9FE4F044626682F20005D00F0A000C5
:10A4200010B10620BDE8FE8F4FF0000901E009F1F0
:10A430000109F06830F819000028F8D1D4E90A12AF
:10A44000606A8DE807009DF80B0000F0010028B35A
:10A4500040212F2001554FF001080EE04346694688
:10A4600004F12400F268FFF771FE2046FFF74EFF6B
:10A47000054605B104E008F10108B8F1640FEDD319
:10A4800000BFB8F1640F01D10720CBE7042D01D044
:10A490002846C7E79DF80B102F2001559DF80B00AB
:10A4A00000F0020030B109F10C000D21B0FBF1F019
:10A4B000401C00E00120074639462046FFF725FDF5
:10A4C00005464DBB781E071E26D06069A0EB4711DC
:10A4D0002046FFF768FC0546F5B904F12400FFF7B4
:10A4E0009CFE824600BF3046E169FFF789F90546C8
:10A4F00005B110E0FAB2216A5346F068FFF7E8FDB3
:10A500000120F07000212046FFF79AFC054615B99E
:10A51000781E071EE7D100BFDDB93046E169FFF7BD
:10A520006FF90546ADB92021206A05F0B6F8206A1A
:10A53000616A0160A16A4160A18D018194F82E10C9
:10A5400081722F20005D00F01800216A087301203D
:10A55000F070284666E72DE9F041044626686769F1
:10A56000206B401C08B9002003E02046216BFFF758
:10A570001AFC0546E5B900BF3046E169FFF740F92E
:10A58000054605B110E000BFE520216A08700120F2
:10A59000F0706069B84200D306E000212046FFF762
:10A5A0004FFC0546002DE7D000BF042D00D1022549
:10A5B0002846BDE8F0812DE9F84F07460C4638687B
:10A5C00000900020A075F86908B9BDE8F88F386BD5
:10A5D000401C002837D00025A846A94624E0009852
:10A5E000C268404608F1010832F81060B9F1000F66
:10A5F00007D1B6F5584F04DBB6F5604F01DAB14626
:10A6000012E0C5F1FF0204F11603591946EA0940A8
:10A61000FEF7D6FF8246BAF1000F01D1002509E00E
:10A6200055444FF0000900BF0098C06830F818008A
:10A630000028D4D100BFB9F1000F00D000250021BF
:10A6400004F1160041550020054680461BE04046B7
:10A6500008F101083A6A165C202E00D113E0052E9D
:10A6600000D1E526B8F1090F07D10C2D05D22E2215
:10A6700028466D1C04F109010A5428466D1C04F19A
:10A6800009010E5400BFB8F10B0FE0D3002104F113
:10A6900009004155A07DB0BB35B93F2228466D1C4D
:10A6A00004F116010A5425E00020054680464FF0CB
:10A6B000080B19E004F1090010F808602E2E01D1F2
:10A6C0004FF0100B412E09DB5A2E07DC386A007B55
:10A6D00000EA0B0010B106F1200086B204F116006A
:10A6E000465508F101086D1C04F1090010F8080036
:10A6F0000028DFD1002104F116004155386A007BA3
:10A7000008B900206072386AC07A00F03F002072F9
:10A71000396A01F11C00FEF703FF2060396A01F17C
:10A720001600FEF7F7FEE080396A01F11800FEF727
:10A73000F1FEA08000BF48E72DE9F34F83B08146CA
:10A74000049800680090D9F80000C768002500BF91
:10A750006846FEF70FFF02900298401C18B90620C9
:10A7600005B0BDE8F08F0298B0F5803F05D30298A0
:10A77000020C28466D1C27F81020029884B2202C69
:10A7800003DB2F2C01D05C2C00D111E0802C06DAE9
:10A790002146FEA004F09EFF08B10620E0E7FF2D51
:10A7A00001D30620DCE728466D1C27F81040CFE7D0
:10A7B00000BF202C01DA042611E002E00098401CC2
:10A7C0000090009800782F28F8D0009800785C2836
:10A7D000F4D0002600980078202800D204260099A2
:10A7E00004980160012D04D1681E37F810002E284E
:10A7F0000BD0022D24D1681E37F810002E281FD14F
:10A80000A81E37F810002E281AD1002027F81500AE
:10A8100080460AE0A84501D22E2100E0202109F15E
:10A82000240000F8081008F10108B8F10B0FF1D36B
:10A8300046F0200109F1240000F8081000208FE7FD
:10A8400008E0681E37F81040202C02D02E2C00D0D3
:10A8500002E06D1E002DF4D100BF002027F8150086
:10A860000DB906207CE74FF0000A01E00AF1010A69
:10A8700037F81A002028F9D0BAF1000F03D137F8C1
:10A880001A002E2801D146F0030600E06D1E25B106
:10A89000681E37F810002E28F8D120220B2109F16C
:10A8A000240004F0F3FE4FF00008C3460820019096
:10A8B00000BF50460AF1010A37F8104004B968E0B9
:10A8C000202C03D02E2C04D1AA4502D046F003063A
:10A8D000EFE70198804501D2AA4516D101980B28CF
:10A8E00002D146F0030654E0AA4501D046F0030623
:10A8F000AA4500D94DE0AA464FF008080B20019068
:10A900004FEA8B604FEA106BD3E7802C0EDB46F0EA
:10A91000020640F2B5112046FEF782FC044604F020
:10A92000800018B104F07F009B490C5CFF2C10DD07
:10A930000198401E404504D846F00306DDF8048027
:10A94000B7E72212404608F1010809F124010A5430
:10A9500018E024B1214691A004F0BCFE18B15F2498
:10A9600046F003060EE0412C03DB5A2C01DC4BF0D1
:10A97000020B612C06DB7A2C04DC4BF0010BA4F1FA
:10A98000200084B2404608F1010809F124010C546A
:10A990008FE700BF99F82400E52802D1052089F847
:10A9A00024000198082803D14FEA8B604FEA106B0E
:10A9B0000BF00C000C2803D00BF00300032801D18E
:10A9C00046F0020606F0020048B90BF0010008B19B
:10A9D00046F010060BF0040008B146F008062F20E0
:10A9E00000F809600020BBE62DE9F3410446276822
:10A9F000019800782F2807D0019800785C2803D0B0
:10AA000000BFB869A0600DE002E00198401C019011
:10AA1000019800782F28F8D0019800785C28F4D0AD
:10AA20000020A06001980078202808D280212F20E3
:10AA3000015500212046FFF7B6F9054637E000BF73
:10AA400001A92046FFF778FE054605B12EE0204615
:10AA5000FFF75CFC05462F20065D95B1042D0FD154
:10AA600006F0200040B106F0040000B9E8E78021BC
:10AA70002F200155002503E006F0040000B905254C
:10AA800014E006F0040000B110E0A07900F010001E
:10AA900008B905250AE0A08AC0F3080207F13800CA
:10AAA00011183846FFF761FAA060C9E700BF2846D1
:10AAB000BDE8FC8170B504464FF0FF302668314692
:10AAC000324601B970BD00BF12F8013B202B01D303
:10AAD0003A2BF9D13A2B11D101250E78302E08DB13
:10AAE0000E78392E05DC8E1C964202D10E78A6F126
:10AAF0003005012D01DA28462260E3E7294E30783F
:10AB000000BFDFE72DE9F041044688460020E070F1
:10AB1000401E606341462046FEF772FE10B10420DD
:10AB2000BDE8F08104F23620FEF7F4FC074694F805
:10AB30003850EB2D03D0E92D01D0E82D5AD14AF63B
:10AB40005520874208D1082217A104F18A0004F099
:10AB5000E0FD08B90020E3E704F14300FEF7DAFC6A
:10AB600006464520055D701E3040E8BBB6F5007F07
:10AB700040DBB6F5007F3DDCB5B3681E284098BBCE
:10AB800004F14600FEF7C6FC70B313E02A3A3C3EDF
:10AB90007C223F7F00000000593702082B2C3B3DF0
:10ABA0005B5D00001A6300204641543332202020B0
:10ABB000000000004820005D401E01281AD804F162
:10ABC0004900FEF7A7FC78B104F14B00FEF7A2FCA8
:10ABD000802806DA04F15800FEF7A2FCB0F5803FA9
:10ABE00008D304F14E0000E004E0FEF793FC08B146
:10ABF000002095E74AF65520874201D102208FE7D1
:10AC000003208DE72DE9FF4107460D460021384618
:10AC1000FFF778FF0646022E06D0032E00D21DB99C
:10AC2000304604B0BDE8F08100BF00240AE007F51B
:10AC3000FB7101EB041101F10800FEF771FC4DF806
:10AC40002400641C042CF2D30DB1681E00E0002027
:10AC5000044600BF5DF8240028B15DF82410384692
:10AC6000FFF750FF00E0032006462DB9022E03D364
:10AC7000601C04460428EDD33046D2E72DE9F74F97
:10AC800084B00021059801600498FFF713FF03903A
:10AC90000398002803DA0B2007B0BDE8F08FFE49C7
:10ACA000039851F820400CB90C20F5E70598046092
:10ACB000069800F0FE000690207878B16078FEF7E4
:10ACC00039FB074607F0010040B9069820B107F0AC
:10ACD000040008B10A20DFE70020DDE70020207033
:10ACE000039860706078FEF73BFB074607F00100B1
:10ACF00008B10320D0E7069820B107F0040008B19E
:10AD00000A20C9E700212046FFF77CFF0546042DF5
:10AD100001D10120C0E7022D01D30D20BCE7D4F8FA
:10AD2000349004F14300FEF7F5FBB0F5007F01D04D
:10AD30000D20B1E704F14E00FEF7ECFB064626B904
:10AD400004F15C00FEF7ECFB064626624820005D3D
:10AD5000A070A078012804D0A078022801D00D208E
:10AD60009AE7A07846434520005D6081608918B16C
:10AD70006089411E084008B10D208DE704F14900AB
:10AD8000FEF7C8FB2081207A00F00F0008B10D20EB
:10AD900082E704F14B00FEF7BDFB8246BAF1000FDB
:10ADA00004D104F15800FEF7BBFB824604F14600D3
:10ADB000FEF7B0FB8346BBF1000F01D10D206BE71E
:10ADC0000BEB0600218900EB1110029002988245DE
:10ADD00001D20D2060E70298AAEB00006189B0FB68
:10ADE000F1F8B8F1000F01D10D2055E70025AB486F
:10ADF000804500D803254FF6F570804500D8022520
:10AE000040F6F570804500D801250DB90D2043E7C7
:10AE100008F10200E061C4F8249009EB0B00A06285
:10AE2000029848442063032D13D104F16200FEF719
:10AE300071FB08B10D202FE7208908B10D202BE709
:10AE400004F16400FEF76CFBE062E06980000190B1
:10AE500014E0208908B90D201EE7A06A3044E062A2
:10AE6000022D02D1E069400007E0207F00F00100E0
:10AE7000E16901EB410100EB51000190216A019869
:10AE800000F2FF10B1EB502F01D20D2004E74FF07C
:10AE9000FF306061206180202071032D2DD104F1ED
:10AEA0006800FEF737FB012827D109F10101204690
:10AEB000FEF7A6FC08BB0020207104F23620FEF746
:10AEC00029FB4AF65521884217D104F13800FEF7D4
:10AED00027FB7349884210D104F50770FEF720FB69
:10AEE0007049884209D104F50870FEF719FB6061CA
:10AEF00004F50970FEF714FB206125706A4800888C
:10AF0000401C80B268490880E0800020A061204693
:10AF1000FEF73FFC0020BFE670B504460D4609264B
:10AF20008CB1206878B12068007860B1A088216871
:10AF3000C988884207D121684878FEF7FBF900F0FC
:10AF4000010000B900260EB9206800E0002028604A
:10AF5000304670BDF7B582B016460398019001A83F
:10AF6000FFF7A8FD0546002D02DA0B2005B0F0BD65
:10AF7000494850F8254024B12046FEF70AFC00203D
:10AF80002070029810B1002002990870424902987E
:10AF900041F825000EB90020E8E7002202A903A825
:10AFA000FFF76CFE07463846E0E72DE9F74F90B013
:10AFB000044616461CB9092013B0BDE8F08F06F010
:10AFC0003F06324602A911A8FFF758FE0546002D9C
:10AFD0006CD1029803904FF40070FEF715F9834688
:10AFE000BBF1000F01D11120E6E70298C0F80CB0C8
:10AFF00003A81199FFF7F8FC05468DB99DF83B00B1
:10B0000000F0800008B106250AE026F0010008B132
:10B01000012000E00020014603A8FEF7F2FA0546F1
:10B0200006F01C00002867D06DB1042D08D1FEF792
:10B0300023FB18B103A8FFF7EBF900E01220054647
:10B0400046F008060AE09DF8120000F0110008B171
:10B05000072503E006F0040000B10825002D5CD1AF
:10B0600006F00800002858D0FEF72FFA00900B9940
:10B0700001F10E000099FEF765FA0B9901F1160037
:10B080000099FEF75FFA0B990298FEF76EFF814672
:10B0900020200B99C8720AE014630020F5FFFF0F0F
:10B0A000525261417272416118630020B3E0002284
:10B0B0000B990298FEF76CFF0B9901F11C0000211F
:10B0C000FEF740FA01200299C870B9F1000F24D0B0
:10B0D0000298D0F834A00022494603A8FEF70CFDE0
:10B0E000054645B951460298FEF78AFB0546A9F187
:10B0F00001000299086110E07DB99DF8120000F08E
:10B10000100008B1042508E006F0020028B19DF8FF
:10B11000120000F0010000B10725BDB906F00800DB
:10B1200008B146F040060298406B60620B98A0623E
:10B1300026F0010008B1012000E00020014603A82C
:10B14000FEF7ABFA2061206900B90225002D5FD11E
:10B150000B990298FEF709FFA0600B9901F11C0002
:10B16000FEF7DEF9E0600020E062029820600298BD
:10B17000C088A0802675002060752062A0614FF411
:10B18000007104F1300004F088FA06F02000E0B30A
:10B19000E068D0B3E068A061029840894002019065
:10B1A000A768D4F80C800DE039462046FEF791FBE5
:10B1B0000746012F00D80225781C00B90125019807
:10B1C000A8EB000815B901988045EDD8E761CDB925
:10B1D000C8F30800B0B139460298FEF76DFB82460D
:10B1E000BAF1000F01D102250CE00AEB58202062D1
:10B1F000226A02994878012304F13001FEF7CCF865
:10B2000000B101250DB1206900E001E0FEF7A1FACF
:10B210005846FDF7FFFF0DB1002020602846CBE621
:10B220002DE9FF4F85B0044615469A46DDF818B063
:10B230000020CAF8000003A92046FFF76DFE049025
:10B24000049810B9607D049018B1049809B0BDE865
:10B25000F08F207D00F0010008B90720F6E7A16912
:10B26000E068401A01900198854200D9019DA8E04C
:10B27000208BC0F30800002874D103984089401E39
:10B28000A16900EA5129B9F1000F1FD1A06910B9D5
:10B29000A06802900CE0E06A28B12046A169FEF7A0
:10B2A00008FD029004E02046E169FEF712FB0290DF
:10B2B0000298022802D202206075C7E70298401C5B
:10B2C00010B901206075C1E70298E061E169039857
:10B2D000FEF7F2FA064616B902206075B6E74E444C
:10B2E0004FEA5528B8F1000F29D009EB080003995F
:10B2F0004989884203D903984089A0EB090803993A
:10B300004878434632465946FEF746F810B10120C8
:10B3100060759BE7207D00F0800068B1206A801B8B
:10B32000404509D2216A891B0BEB41204FF4007282
:10B3300004F1300104F098F94FEA482737E0206A19
:10B34000B04220D0207D00F0800080B1226A0399B5
:10B350004878012304F13001FEF74DF818B10120BF
:10B36000607573E710E0207D00F07F002075039981
:10B3700048780123324604F13001FEF70DF810B190
:10B380000120607562E72662208BC0F30800C0F5DB
:10B390000077AF4200D92F46208BC0F3080204F19A
:10B3A000300011183A46584604F05EF900BFED1B14
:10B3B000DAF800003844CAF80000BB44A0693844F9
:10B3C000A061002D7FF454AF00203FE72DE9FF4F2F
:10B3D00083B0044615469B46049800900020CBF8A5
:10B3E000000001A92046FFF797FD0290029810B9CE
:10B3F000607D029018B1029807B0BDE8F08F207D03
:10B4000000F0020008B90720F6E700BFA069284451
:10B41000A169884202D2A069C0F1FF35C3E0208B48
:10B42000C0F3080000287DD101984089401EA16921
:10B4300000EA512ABAF1000F26D1A06938B9A768ED
:10B4400097B900212046FEF7A4FB07460CE0E06A0E
:10B4500028B12046A169FEF72CFC074604E02046EF
:10B46000E169FEF796FB074607B99FE0012F02D17D
:10B4700002206075C0E7781C10B901206075BBE739
:10B48000E761A06800B9A760207D00F0800078B176
:10B49000226A01994878012304F13001FDF7ABFFDE
:10B4A00010B101206075A7E7207D00F07F002075B6
:10B4B000E1690198FEF700FA064616B902206075A8
:10B4C0009AE756444FEA5529B9F1000F2BD00AEB01
:10B4D000090001994989884203D901984089A0EB64
:10B4E0000A09019948784B4632460099FDF783FFD7
:10B4F00010B1012060757FE7206A801B48450ED29D
:10B50000206A801B009A02EB40214FF4007204F184
:10B51000300004F0A9F8207D00F07F0020754FEA8C
:10B5200049282BE013E0206AB0420FD0E168A069FF
:10B5300088420BD2019948780123324604F1300148
:10B54000FDF72AFF10B10120607555E72662208BB8
:10B55000C0F30800C0F50078A84500D9A846218BA3
:10B56000C1F3080204F1300150184246009904F07A
:10B570007BF8207D40F08000207500BFA5EB08051A
:10B58000DBF800004044CBF80000009840440090F5
:10B59000A0694044A061E168A069884201D9A0691E
:10B5A00000E0E068E060002D7FF439AF00BF207D4F
:10B5B00040F04000207500201EE7F8B504466946BB
:10B5C0002046FFF7A9FC0646002E44D1207D00F05E
:10B5D000400000283FD0207D00F0800070B1226A3A
:10B5E00000994878012304F13001FDF704FF08B108
:10B5F0000120F8BD207D00F07F002075FDF765FF7C
:10B600000746616A0098FEF7FBF806461EBBA56A6E
:10B61000E87A40F02000E8722946A2682068FEF728
:10B62000B7FC05F11C00E168FDF78CFF394605F118
:10B630001600FDF787FF002105F11200FDF77CFFE2
:10B6400001200099C8700098FEF7F4F80646207DA6
:10B6500000F0BF0020753046CBE738B505462846D8
:10B66000FFF7ABFF044664B969462846FFF754FC70
:10B67000044634B92869FEF76CF804460CB900207A
:10B680002860204638BD31B56846FFF713FA0446F6
:10B69000002C01DA0B2038BDFD490C700020FAE7C0
:10B6A00031B58EB0002269460EA8FFF7E7FA0446CE
:10B6B00074BB009801904FF40070FDF7A5FD05469E
:10B6C00015B911200FB030BD0098C56001A80E99C2
:10B6D000FFF78AF90446ACB99DF8330000F080000A
:10B6E00018B10099039888610CE09DF80A0000F0F9
:10B6F000100030B109990098FEF737FC0099886175
:10B7000000E005242846FDF785FD042C00D1052422
:10B710002046D7E72DE9F04F89B004460D4607A92A
:10B720002046FFF7F9FB0890089808B9607D08905B
:10B73000089818B1089809B0BDE8F08FE06A0028B1
:10B740007CD0681C002843D1D4F82C9059F8040B05
:10B75000029002200190A76867B300BF0397002002
:10B7600004900198801C019000BF05970498401C2C
:10B77000049039462046FEF7ACF80746012F02D860
:10B7800002206075D7E7781C10B901206075D2E7F8
:10B790000598401C8742E8D0DDE90101884205D8C0
:10B7A000049849F8040B039849F8040B0798C069FA
:10B7B000B842D3D80198E16A0860DDE90101884206
:10B7C00003D80020C9F80000FAE011200890F7E043
:10B7D000E068A84200D2E568A561002DF4D0691E9A
:10B7E0002046FEF766FAE061E1690798FEF764F823
:10B7F0008246BAF1000F02D1022060759BE70798DC
:10B800004089401E691E00EA51208244208BC0F30B
:10B8100008000028D8D0206A5045D5D0207D00F0FF
:10B82000800080B1226A07994878012304F1300131
:10B83000FDF7E1FD18B1012060757CE712E0207D85
:10B8400000F07F002075079948780123524604F1E3
:10B850003001FDF7A1FD10B1012060756BE7C4F860
:10B8600020A0ADE0E068A84204D2207D00F00200F4
:10B8700000B9E568A06906904FF0000BC4F818B055
:10B88000002D6AD0079840894FEA4028069890B169
:10B89000681EB0FBF8F10698401EB0FBF8F081423C
:10B8A00009D30698401EA8F101018843A061A06950
:10B8B0002D1AE66912E0A6687EB900212046FEF73F
:10B8C00068F90646012E02D10220607533E7701C2C
:10B8D00010B9012060752EE7A660E661D6B325E0B9
:10B8E000A5EB0805A0694044A061207D00F002009E
:10B8F00040B100BF31462046FEF74BF9064636B947
:10B90000002515E031462046FDF7E3FF0646701C92
:10B9100010B9012060750EE7012E03D90798C069A0
:10B92000B04202D80220607505E7E6614545D7D8E8
:10B9300000BFA0692844A061C5F3080050B131469A
:10B940000798FDF7B9FF8346BBF1000F03D1022032
:10B950006075F0E601E00BEB552BE168A0698842C9
:10B9600005D9A069E060207D40F040002075208B63
:10B97000C0F3080020B3206A584521D0207D00F094
:10B98000800078B1226A07994878012304F13001D8
:10B99000FDF731FD10B101206075CCE6207D00F08F
:10B9A0007F0020750799487801235A4604F1300139
:10B9B000FDF7F2FC10B101206075BCE6C4F820B0C0
:10B9C0000898B8E673B582B0044614B9092004B0EB
:10B9D00070BD002201A903A8FFF750F90546002D0C
:10B9E0003ED1019820604FF40070FDF70DFC064633
:10B9F0000EB91120EBE70198C66020460399FEF7C7
:10BA0000F3FF05461DBB2F20005D00F0800050B9FC
:10BA1000A07900F0100028B1216A0198FEF7A5FA7C
:10BA2000A06000E0052595B90198C088A08000219C
:10BA30002046FEF7B8F905464DB9A06840B100218F
:10BA40002046FDF72AFE2061206900B9122501E099
:10BA5000002020613046FDF7DDFB042D00D10525D7
:10BA60000DB1002020602846B1E738B5044669468C
:10BA70002046FFF751FA054645B9206918B12069FB
:10BA8000FDF767FE05460DB900202060284638BD49
:10BA90001A630020F8B507460E4669463846FFF798
:10BAA0003BFA044644BB2EB900213846FEF77BF929
:10BAB000044621E04FF40070FDF7A6FB05460DB9E2
:10BAC0001120F8BD0098C56000213846FEF7B5FB8F
:10BAD0000446042C00D100245CB931463846FEF7F8
:10BAE0006AFD00213846FEF7ABF90446042C00D16C
:10BAF00000242846FDF78EFB2046E2E773B58EB0A2
:10BB00000E46002201A90EA8FFF7B8F80546FDB9B8
:10BB10004FF40070FDF778FB044614B9112010B003
:10BB200070BD0198C46001A80E99FEF75DFF05463F
:10BB30005DB99DF8330000F0800008B1062504E0EF
:10BB40001EB1314601A8FEF736FD2046FDF762FB27
:10BB50002846E4E72DE9F74F86B089469246002251
:10BB600005A906A8FFF78AF88046B8F1000F6BD147
:10BB70000598CAF8000005984169C069801E814295
:10BB800004D805984069C9F800005DE000250598D3
:10BB9000007801281BD102260598009000BF31468D
:10BBA0006846FDF796FE0746781C10B94FF001086D
:10BBB0000CE0012F02D14FF0020807E007B96D1C1D
:10BBC000701C06460599C9698842E8D32FE005989C
:10BBD000C6690598D0F828B0002400BF54B959466A
:10BBE0000BF1010B0598FDF70BFE8046B8F1000F35
:10BBF00000D01BE005980078022808D1059938315B
:10BC00000819FDF787FC00B96D1CA41C09E0059913
:10BC100038310819FDF784FC20F0704000B96D1C24
:10BC2000241DC4F30804701E061ED7D100BFB8F14E
:10BC3000000F09D1C9F800500598456105980079B1
:10BC400040F0010005990871404609B0BDE8F08F49
:10BC5000F8B5044669462046FFF75EF9054615B972
:10BC6000607D051E01D02846F8BD207D00F0020051
:10BC700008B90720F8E7E168A06988423FD2A069C7
:10BC800040B900222046A168FDF736FF0546002096
:10BC9000A06016E02046E169FDF71BFE0646002580
:10BCA000701C00B90125012E00D102254DB9009864
:10BCB000C069B04205D931462046E269FDF71CFF54
:10BCC0000546A069E060207D40F04000207595B9F0
:10BCD000207D00F0800070B1226A0099487801232D
:10BCE00004F13001FDF787FB08B1012503E0207D59
:10BCF00000F07F00207515B165752846B4E7284629
:10BD0000B2E771B59BB00025022269461BA8FEF779
:10BD1000B5FF0446002C66D100980E904FF40070D9
:10BD2000FDF772FA064616B911201CB070BD0098D6
:10BD3000C6600EA81B99FEF757FE04462CB99DF865
:10BD4000670000F0200000B1062424B902210EA8EB
:10BD5000FDF757FC0446002C42D19DF8670000F027
:10BD6000800008B1062405E09DF83E0000F00100C7
:10BD700000B1072414BB16990098FEF7F6F80546A3
:10BD80009DF83E0000F01000C0B100988069A84204
:10BD900001D1072412E0009801900395002101A829
:10BDA000FEF701F804464CB9002101A8FEF745FA58
:10BDB000044604B90724042C00D1002484B90EA839
:10BDC000FEF7C9FB044634B92DB1002229460EA85E
:10BDD000FDF792FE04461CB90098FDF72BFD0446C2
:10BDE0003046FDF717FA20469FE72DE9F14193B061
:10BDF0000222694613A8FEF741FF0446002C7DD1BC
:10BE0000009806904FF40070FDF7FEF906461EB943
:10BE1000112014B0BDE8F0810098C66006A81399FF
:10BE2000FEF7E2FD044604B90824042C05D19DF870
:10BE3000470000F0200000B10624042C6AD10098CD
:10BE40000190002101A8FDF7A4FE0546002405B9D4
:10BE50000724012D00D10224681C00B90124FDF73C
:10BE600034FB8046BCBB29460098FDF73BFF0446E7
:10BE70008CBB20220B210098383003F007FC2E20C9
:10BE8000009981F838001021009880F8431041464D
:10BE900000984E30FDF756FB2A460099383100983D
:10BEA000FEF776F82022009938310098583003F0D8
:10BEB000DBFB2E21009880F85910089F3A46009924
:10BEC00058310098FEF764F801200099C87006A860
:10BED000FEF79EFA0446C4B90E9901F116004146D8
:10BEE000FDF730FB2A460E990098FEF751F8102016
:10BEF0000E99C87201200099C87000E00DE01CB9CD
:10BF00000098FDF797FC044604E00022294601A8AA
:10BF1000FDF7F2FD3046FDF77DF9204679E72DE982
:10BF2000F341A4B025A8FEF7C5FD022209A924A863
:10BF3000FEF7A4FE0446002C70D1099817904FF428
:10BF40000070FDF761F907461FB9112026B0BDE862
:10BF5000F0810998C76017A82499FEF745FD0446AB
:10BF60002CB99DF88B0000F0A00000B1062424B984
:10BF7000022117A8FDF745FB0446002C6DD12022B5
:10BF800001A81F9903F070FB342217A90AA803F037
:10BF90006BFB0AA82599FEF727FD04465CB91999A1
:10BFA0000C98884205D11C990F98884201D1042031
:10BFB00000E008200446042C45D10AA8FEF728FA20
:10BFC0000446002C3FD1129D13220DF1110105F101
:10BFD0000D0003F049FB9DF80F00E872E87A00F0CD
:10BFE000100018B9E87A40F02000E87201200999A1
:10BFF000C870E87A00F0100028B30C9919988842AC
:10C0000021D029460998FDF7B0FF8046414609989E
:10C01000FDF752FC064616B9022414E020E0314632
:10C020000998FDF7EDFB0446099800F1580554B94D
:10C0300068782E2807D129460C9A0998FDF7A8FFA1
:10C0400001200999C87044B917A8FEF784FA04467C
:10C050001CB90998FDF7EEFB04463846FDF7DAF8FF
:10C06000204673E72DE9FF4F85B09A4603AA0121C8
:10C070000598FDF7E3F918B1012009B0BDE8F08F8C
:10C08000DDF80C904FF03F08082701E07806070E16
:10C0900037B1B9FBF7F0B0FBF8F0B0F5806FF5D829
:10C0A00007B9FF274FF40071504603F0F6FA0AF57E
:10C0B000DF764FF0000B444669E0069850F82B50AD
:10C0C000642D07D801D1484603E06420B9FBF0F0A5
:10C0D000684305466019484501D8601901D3A9EBAA
:10C0E000040505B959E0214606F10800FDF72AFAD2
:10C0F000294606F10C00FDF725FA07983071B4FBCC
:10C10000F8F0B0FBF7F00490B4FBF8F0B0FBF7F1F7
:10C1100007FB1100C0B20290B4FBF8F008FB10401E
:10C12000401CC0B2019002987070C021049801EACE
:10C13000900001990843B0700498F0706019401E97
:10C14000B0FBF8F0B0FBF7F004906019401EB0FBB4
:10C15000F8F0B0FBF7F107FB1100C0B202906019D4
:10C16000401EB0FBF8F108FB1100401CC0B201906A
:10C1700002987071C021049801EA90000199084367
:10C18000B0710498F07110360BF1010B2C44BBF127
:10C19000040F02D20CB14C458FD300BF4AF6552193
:10C1A0000AF5FF70FDF7C8F90123002251460598F2
:10C1B000FDF721F908B101205FE700205DE72DE9D7
:10C1C000FF4F99B00F46154619A8FEF773FC029071
:10C1D0000298002803DA0B201DB0BDE8F08FFE495D
:10C1E000029851F8200028B10021FB4A029852F829
:10C1F000200001700298C0B216900020159007B977
:10C20000F64F1698FDF7ACF80190019800F0010088
:10C2100008B10320E0E7019800F0040008B10A200B
:10C22000DAE778681390139838B913AA032116989F
:10C23000FDF704F908B101201390139840B1139849
:10C24000B0F5004F04D81398401E1399084008B168
:10C25000012013904FF40079387800F00F00189007
:10C260007878012804DB7878022801DC787800E00F
:10C2700001200590B96889B1B968B1F5004F0DD8B2
:10C2800048464FEAE97109EBD1614911BA68B2FB3E
:10C29000F1F301FB132109B9B96801E04FF4007112
:10C2A0000491F868B0F1807F05D8F868411E084015
:10C2B00008B9F86800E0002006900698B0FBF9F095
:10C2C00006901C98B0FBF9F01490149808B911204E
:10C2D00082E72C462CB9149901FB09F0FCF794FF76
:10C2E00004460CB9112077E7002010900F9000BF92
:10C2F00010AA01211698FDF7A1F828B115B920461A
:10C30000FCF788FF012067E7189800F0080040B9A3
:10C3100010983F2805D93F200F90DDE90F01081A3A
:10C3200010901098802805D215B92046FCF772FFAE
:10C330000E2051E700BF00BF0698802801D9802059
:10C340000690189800F0020030B1189800F0010033
:10C3500010B94FF003080CE0189800F0010028B95C
:10C3600015B92046FCF756FF132035E74FF00208B9
:10C3700000BF00BFFDF7A9F810990844119000BF55
:10C38000069EB8F1030F31D1A6B910984FEA504B71
:10C3900000200390012603E00398401C03907600E0
:10C3A0008F49039831F8100020B1039831F810003C
:10C3B0005845F1D91098B0FBF6FA082000EB8A0036
:10C3C0004844401EB0FBF9F008902020099000205E
:10C3D00007904FF6F570824502D9824882453BD9D5
:10C3E00015B92046FCF716FF0E20F5E6A6B9109801
:10C3F0004FEA103B00200390012603E00398401C05
:10C40000039076007849039831F8100020B1039822
:10C4100031F810005845F1D91098B0FBF6FA40F603
:10C42000F570824503D9042000EB4A0B07E04FF07A
:10C4300001080AEB4A00401C032101EB500B0BEBF7
:10C440000900401EB0FBF9F0089001200990049803
:10C450004001B0FBF9F0079009990F9808440E903D
:10C46000059A08990E9801FB0201079808440D905F
:10C4700013990D980844401E491E20EA01010D98A9
:10C48000A1EB000BB8F1030F06D1099858440990AD
:10C490000E9858440E9013E00598BBFBF0F100FB9A
:10C4A00011B038B1ABF1010B0998401C09900E98FE
:10C4B000401C0E900598BBFBF0F1089808440890CA
:10C4C0000D9800EB06110F98081A1099884205D9AB
:10C4D00015B92046FCF79EFE0E207DE610990998BE
:10C4E0000A1A0599089800FB11210798081AB0FB51
:10C4F000F6FAB8F1030F0FD14FF6F57082450BD85D
:10C50000069818B97008069000B148E015B92046A1
:10C51000FCF780FE0E205FE6B8F1020F31D14FF636
:10C52000F57082451CD9069830B94020B0EB460F13
:10C5300002D37000069032E0189800F0020010B1AB
:10C540004FF003082BE0069820B970000690802871
:10C5500000D824E015B92046FCF75CFE0E203BE62F
:10C5600040F6F57082450CD8069820B97000069008
:10C57000802800D813E015B92046FCF74BFE0E20AA
:10C580002AE6B8F1010F09D140F6F570824505D9C8
:10C5900015B92046FCF73EFE0E201DE600E0EFE652
:10C5A00000BF4946204603F078F810A001682160DA
:10C5B0004168616001892181807AA072494604F155
:10C5C0000B00FCF7B9FF6673099881B204F10E0005
:10C5D000FCF7B2FF05980FE014630020F83702085B
:10C5E000E8370208F5FFFF0FDA370208EBFE904D3F
:10C5F00053444F53352E30002074B8F1030F01D14E
:10C60000002000E0049881B204F11100FCF794FFCF
:10C610001098B0F5803F06D2109881B204F1130053
:10C62000FCF78AFF04E004F120001099FCF78AFF70
:10C63000F82060753F2104F11800FCF77DFFFF2111
:10C6400004F11A00FCF778FF04F11C000F99FCF7C5
:10C6500079FFB8F1030F25D104F143001199FCF7DC
:10C6600071FF04F124000899FCF76CFF022104F12A
:10C670002C00FCF767FF012104F13000FCF75CFFA0
:10C68000062104F13200FCF757FF802084F84000B7
:10C69000292084F84200132291A104F1470002F0FE
:10C6A000E3FF16E004F127001199FCF74BFF08980F
:10C6B00081B204F11600FCF73FFF802084F82400CB
:10C6C000292084F8260013228AA104F12B0002F00D
:10C6D000CBFF4AF6552104F5FF70FCF72DFF01232F
:10C6E00021460F9A1698FCF786FE28B115B9204608
:10C6F000FCF790FD01206FE5B8F1030F32D1012363
:10C700000F9A921D21461698FCF775FE4946204661
:10C7100002F0C3FF7C492046FCF714FF7B4904F577
:10C72000F270FCF70FFFAAF1010104F5F470FCF7B9
:10C7300009FF022104F5F670FCF704FF4AF65521C3
:10C7400004F5FF70FCF7F8FE01230F9AD21D214675
:10C750001698FCF750FE01230F9A521C214616989A
:10C76000FCF749FE149800FB09F1204602F095FF02
:10C770000E980C900020039047E0B8F1030F10D101
:10C780006FF007012046FCF7DDFE4FF0FF31201D62
:10C79000FCF7D8FE6FF0704104F10800FCF7D2FE00
:10C7A0000AE0B8F1010F01D1594801E06FF007002C
:10C7B00001462046FCF7C6FE0898129000BF149967
:10C7C0001298884201D9149800E0129883465B467B
:10C7D00021460C9A1698FCF70EFE28B115B9204692
:10C7E000FCF718FD0120F7E44946204602F055FF0A
:10C7F0000C9858440C901298A0EB0B0012901298D1
:10C800000028DCD10398401C0390059903988842C6
:10C81000B3D3B8F1030F01D1304600E0079812906E
:10C8200000BF14991298884201D9149800E0129818
:10C8300083465B4621460C9A1698FCF7DCFD28B12E
:10C8400015B92046FCF7E6FC0120C5E40C985844D5
:10C850000C901298A0EB0B00129012980028E0D1D7
:10C8600000BFB8F1030F02D10C2017900DE0109813
:10C87000B0F5803F02D30620179006E0B8F1020F12
:10C8800001D1042000E00120179000BF189800F0AB
:10C89000080090B910980A9000200B9023460AA92E
:10C8A000DDE91602FFF7DEFB0090009828B115B90C
:10C8B0002046FCF7AFFC00988EE400221146169843
:10C8C000FCF7BCFD28B115B92046FCF7A3FC0120FC
:10C8D00082E415B92046FCF79DFC00207CE40000B2
:10C8E0004E4F204E414D45202020204641543332AA
:10C8F000202020004E4F204E414D45202020204634
:10C900004154202020202000525261417272416126
:10C91000F8FFFF001CB501210846F4F7F3FA0120E7
:10C920008DF8040000208DF8060001208DF8070026
:10C9300002208DF8050000906946FC48F4F706F8DF
:10C940000221FA48F4F77EF81CBD10B50221F74821
:10C95000F4F776F8C820F7F774FD4FF47A70F7F71C
:10C9600070FD0221F148F4F76DF810BD10B50221F9
:10C97000EF48F4F765F810BD10B50221EC48F4F764
:10C9800061F810BD70B500240020EA49C870087035
:10C990004871FFF7BFFFFFF7E9FF4FF47A70F7F731
:10C9A00050FDFFF7D2FF4FF4FA60F7F74AFDE2A01F
:10C9B00005F048F94FF47A70F7F743FDE2A005F06F
:10C9C00041F94FF4FA70F7F73CFD41F28830F7F780
:10C9D00038FD002518E0F9F77FF8DFA005F032F9FF
:10C9E0004FF4FA70F7F72DFDDDA1DE4802F060FE8E
:10C9F00005463DB9FFF7BAFF4FF4FA70F7F721FD8E
:10CA0000FFF7A3FF601CC4B20DB9012000E00020B5
:10CA10000A2C01DA012100E0002108400028DAD1C7
:10CA2000D1A005F00FF94FF49670F7F70AFDD4A0E6
:10CA300005F008F94FF47A70F7F703FDC8A1C9486B
:10CA400002F036FE0546D0A005F0FCF84FF4FA706F
:10CA5000F7F7F7FCB8A005F0F5F84FF47A70F7F7A0
:10CA6000F0FCBFA1BF4802F023FE0546C6A005F0BA
:10CA7000E9F84FF4FA70F7F7E4FCF9F72DF8C6A0DF
:10CA800005F0E0F84FF4FA70F7F7DBFCB4A1B54815
:10CA900002F00EFE0546002411E0601CC4B2BEA0E8
:10CAA00005F0D0F84FF4FA70F7F7CBFCBDA1AD4814
:10CAB00002F0FEFD05460A2C01DD012070BD0F2CA1
:10CAC00001DA012000E000200DB9012100E0002181
:10CAD00008400028E1D1012096494871F8F7FCFF91
:10CAE000B2A005F0AFF84FF47A70F7F7AAFCB2A144
:10CAF0009C4802F0DDFD0546002413E0F8F7ECFF4A
:10CB0000AAA005F09FF84FF4FA60F7F79AFCAAA1E3
:10CB1000944802F0CDFD0546601CC4B20A2C01DD2C
:10CB20000120CBE70F2C01DA012000E000200DB935
:10CB3000012100E0002108400028DFD101207D49CB
:10CB4000C870F8F7C9FF9FA005F07CF84FF4967005
:10CB5000F7F777FC9EA1834802F0AAFD05464DB188
:10CB6000287A3038E979303901EB810100EB410056
:10CB700070490870F8F7B0FF00209FE770B50025F6
:10CB8000F8F7AAFF94A005F05DF84FF4FA70F7F7F4
:10CB900058FC95A1734802F08BFD04460FE0F8F7AE
:10CBA0009BFF8DA005F04EF84FF4FA70F7F749FCA3
:10CBB0008DA16C4802F07CFD0446681CC5B20CB91E
:10CBC000012000E00020032D01DA012100E0002116
:10CBD00008400028E3D11CB186A0FBF762FA70BDC3
:10CBE0005CB9F8F779FF7CA005F02CF84FF4FA70E7
:10CBF000F7F727FC85A0FBF754FA00BFEFE72DE914
:10CC0000F04106460F460025F8F766FF854AA2F177
:10CC1000140185A005F016F84FF47A70F7F711FCAF
:10CC200089A1504802F044FD044618E0FFF7A6FF32
:10CC30004FF4FA70F7F705FCF8F74EFF794AA2F1C6
:10CC4000140179A004F0FEFF4FF47A70F7F7F9FBB6
:10CC50007DA1444802F02CFD0446681CC5B20CB905
:10CC6000012000E00020052D01DA012100E0002173
:10CC700008400028DAD12CB101202E49087176A095
:10CC8000FBF70FFA2CB900202A49087179A0FBF7AD
:10CC900008FABDE8F0812DE9FC4104460D4600206C
:10CCA000009001900026F8F717FF224678A1684609
:10CCB00004F0D8FF694677A0FBF7F3F92A466946E6
:10CCC0007AA004F0BFFF4FF47A70F7F7BAFB7DA1AA
:10CCD000244802F0EDFC07460AE04FF47A70F7F7BB
:10CCE000B0FB78A11F4802F0E3FC0746701CC6B2F7
:10CCF0000FB90A2EF1DBBDE8FC812DE9F0410646B3
:10CD00000F460025F8F7E8FE314670A004F09AFFC0
:10CD100031466EA0FBF7C5F94FF49670F7F791FB1B
:10CD20006FA1104802F0C4FC0446FEE0000002407F
:10CD3000000402401B63002041542B4350534D53C9
:10CD40003D300D0A0000000041542B5153434C4B21
:10CD50003D300D0A0000000041540D0A00000000A3
:10CD60004F4B0000EC65002041542B5153454C467D
:10CD700052454749535445523D310D0A00000000C9
:10CD8000415445300D0A000041542B514C45444D4F
:10CD90004F44453D310D0A0041542B514343494412
:10CDA0000D0A00002B5143434944000041542B43DA
:10CDB000474154543F0D0A002B43474154543A20F5
:10CDC0003100000041542B434553510D0A0000002F
:10CDD0002B4345535100000041542B5149434C4FC4
:10CDE00053453D300D0A0000434C4F5345204F4BF7
:10CDF00000000000424332355F436C6F7365536F30
:10CE0000636B6574204F4B0D0A00000042433235BE
:10CE10005F436C6F7365536F636B657420320D0AEB
:10CE2000000000008265002041542B51494F5045BD
:10CE30004E3D312C302C22544350222C25732C256E
:10CE4000732C302C310D0A002B51494F50454E3A6E
:10CE500020302C3000000000424332355F437265C1
:10CE6000617465536F6B6365742073756365737369
:10CE70000D0A0000424332355F43726561746553A9
:10CE80006F6B636574206661696C0D0A00000000B9
:10CE900025640000424332355F53656E64646174FB
:10CEA000615F6C656E733A25730D0A0041542B5116
:10CEB0004953454E443D302C25732C222573220DB9
:10CEC0000A00000053454E44204F4B0041542B5163
:10CED0004953454E443D302C25640D0A00000000A6
:10CEE0003E000000681CC5B23146AFF2200004F0DD
:10CEF000A9FE4FF4FA70F7F7A4FAAFF21C019048BC
:10CF000002F0D6FB04465CB9F8F7E6FD3146AFF215
:10CF1000440004F097FE3146AFF25000FBF7C1F831
:10CF2000874A294687A0FBF7BCF80CB9142DD9DB3A
:10CF300014B90120BDE8F0814FF4FA70F7F781FAD7
:10CF4000394685A004F07EFE394683A0FBF7A9F898
:10CF50004FF49670F7F775FA0025AFF2980178480C
:10CF600002F0A6FB04461BE0681CC5B24FF49670A5
:10CF7000F7F767FAAFF2B401714802F099FB044683
:10CF80004CB9F8F7A9FD394673A004F05BFE3946A9
:10CF900071A0FBF786F86A4A294670A0FBF781F872
:10CFA0000CB9142DE0DB0CB10020C3E70120C1E770
:10CFB00010B56FA1624802F07BFB04460CB1F8F794
:10CFC0008BFD10BD2DE9FC5F0026FFF7A3FCFFF7EA
:10CFD000CDFC4FF47A70F7F734FAFFF7B6FC4FF454
:10CFE000FA70F7F72EFAAFF2B02004F02BFE4FF4F0
:10CFF0007A70F7F726FAAFF2B02004F023FE4FF470
:10D00000FA50F7F71EFA002411E0701CC6B2F8F7C8
:10D0100063FDAFF2682004F015FE4FF4FA70F7F7E5
:10D0200010FAAFF26C21464802F042FB04463C2E57
:10D0300001DA012000E000200CB9012100E000210C
:10D0400008400028E1D10CB9BDE8FC9F00240DE0A8
:10D05000F8F742FD48A004F0F5FD4FF4FA70F7F739
:10D06000F0F948A1364802F023FB04463C2E01DAD1
:10D07000012000E000200CB9012100E0002108405F
:10D080000028E5D104B9DFE740A12D4802F010FBEC
:10D090000446641C607830382178303901EB810116
:10D0A00000EB410520793038E178303901EB81011E
:10D0B00000EB4107E0793038A179303901EB81018B
:10D0C00000EB4108A07A3038617A303901EB8101F8
:10D0D00000EB4109607B3038217B303901EB810165
:10D0E00000EB410A207C3038E17B303901EB8101D3
:10D0F00000EB410B142D07DD4B46424639462846CE
:10D10000CDE900ABF9F7BDFB00BF9DE710B5FFF718
:10D1100039FCFFF733FD1E49A1F11400FFF76FFD45
:10D120001CA10420FFF7E9FD1C4802F0DDFA0446CB
:10D130001A49FFF7E2FD12A10220FFF7DEFD10BD44
:10D14000EC65002074696D65313A25642C72783184
:10D150003A25730D0A0000002573000074696D659F
:10D16000323A25642C7278323A25730D0A00000099
:10D170002B5149555243000041542B43434C4B3FE4
:10D180000D0A00002B43434C4B3A000022000000E4
:10D19000826500205075622D00000000E06D0020C7
:10D1A00010B504462046FAF7DDF810BD2DE9F04130
:10D1B00007460D46144698460026FAF73AF9FDA1AF
:10D1C000204602F075FA20B13946FBA0FAF793F930
:10D1D00003E03946F9A0FAF78EF91DB914B9012018
:10D1E000BDE8F0814046F7F72CF90A20F7F729F956
:10D1F0000020F449B1F8C810C1F30E01F14A5054AF
:10D20000DDB1D4B12946104602F052FA08B101202E
:10D2100000E0002040B92146EA4802F049FA08B18E
:10D22000012000E0002008B1012000E000200646B7
:10D230000EB10120D4E70020D2E7D5B12946E1485C
:10D2400002F036FA08B1012000E0002040B9214682
:10D25000DC4802F02DFA08B1012000E0002008B1FE
:10D26000012000E0002006460EB10120B8E70020B2
:10D27000B6E72946D34802F01BFA08B1012000E0C6
:10D28000002040B92146CF4802F012FA08B101202F
:10D2900000E0002008B1012000E0002006460EB1A9
:10D2A00001209DE700209BE710B500240DE04FF41E
:10D2B000FA730022C4A1C5A0FFF778FF00B110BD2A
:10D2C000601C84B26420F7F7BCF8642CEFDB00BF6D
:10D2D000F5E710B5044624B1012C0AD0022C18D170
:10D2E0000FE040F6C413BCA2B7A1BDA0FFF75EFFDC
:10D2F00010BD40F6C413B8A2B3A1BCA0FFF756FFFF
:10D30000F6E740F6C413B4A2AFA1BBA0FFF74EFFEF
:10D31000EEE70020ECE730B59FB004460D462B4603
:10D320002246B8A101A804F09DFC41F288330022F6
:10D33000A5A101A8FFF73AFF1FB030BD10B586B018
:10D3400004460CB1012000E000200246B2A101A871
:10D3500004F088FC4FF4FA7300229BA101A8FFF7A8
:10D3600025FF06B010BD70B59AB005460E461446AE
:10D37000642101A802F091F915B1012D10D107E047
:10D380003346A9A2A9A101A8009404F06BFC08E00F
:10D390003346AAA2A5A101A8009404F063FC00E012
:10D3A00000BF00BF42F210738BA287A101A8FFF754
:10D3B000FDFE1AB070BDF0B5B5B004460D46164678
:10D3C0001F4664211CA802F068F9642103A802F03A
:10D3D00064F92B4622469AA103A8CDE9006704F020
:10D3E00041FC03AB9AA29EA11CA804F03BFC41F2B5
:10D3F0008833002274A11CA8FFF7D8FE10B90020C2
:10D4000035B0F0BD0120FBE730B5B3B004460D46A2
:10D4100064211AA802F041F9642101A802F03DF943
:10D4200023462A4690A101A804F01CFC01AB90A25F
:10D430008BA11AA804F016FC41F28833002262A1E5
:10D440001AA8FFF7B3FE10B9002033B030BD012099
:10D45000FBE710B54FF4FA7300225BA188A0FFF739
:10D46000A5FE08B9002010BD4FF4FA7388A256A19A
:10D4700088A0FFF79BFEF6E72DE9F04186B006464F
:10D480000F4614461D464FF0000836B139464AA0F3
:10D49000FAF731F84FF001081AE0052D06DA2346B5
:10D4A0002A467FA101A804F0DDFB04E0A21C81A1B3
:10D4B00001A804F0D7FBC823002282A101A8FFF72E
:10D4C00075FEC8233BA280A13846FFF76FFE804659
:10D4D000404606B0BDE8F08110B54FF47A70F6F71B
:10D4E000B0FF7BA0FAF7DDFD4FF4FA70F6F7A9FF65
:10D4F00010BD10B54FF4FA73002276A179A0FFF7A2
:10D5000055FE30B173A12F4802F0D2F808B10220C5
:10D5100010BD0020FCE7F0B503460D461646002777
:10D5200029460A2E03D0002008702846F0BD33B9E2
:10D53000302001F8010B002008702846F6E7002B88
:10D5400003DA2D2001F8010B5B4242F210720DE06C
:10D5500093FBF2F404B937B104F1300001F8010B88
:10D5600004FB123301270A2092FBF0F2002AEFDCC1
:10D57000002008702846D9E70FB470B586B006467B
:10D580000CA8019016E10B9800785C280FD10B983D
:10D59000401C0B9000786E280AD0722809D10D210A
:10D5A0003046F5F70EFD0B98401C0B90AEE0AEE058
:10D5B000A0E0A7E0310000002573000025730D0AEC
:10D5C00000000000847700204F4B000041542B5294
:10D5D0004553544F524500004E554C4C000000003E
:10D5E00041542B43574D4F44453D310041542B434B
:10D5F000574D4F44453D320041542B43574D4F4406
:10D60000453D330041542B43574A41503D22257339
:10D61000222C22257322000041542B4349504D55A2
:10D62000583D256400000000544350002225732219
:10D630002C222573222C2573000000005544500035
:10D64000222573222C222573222C25642C2564008C
:10D6500041542B43575341505F4445463D00000021
:10D66000257325730000000025642C25730000003D
:10D6700041542B4349505345525645523D000000FA
:10D6800041542B4349504D4F44453D31000000006B
:10D690003E00000041542B43495053454E44000086
:10D6A00041542B43495053454E443D25642C256C31
:10D6B0006400000041542B43495053454E443D25DE
:10D6C0006C6400003E20000053454E44204F4B0048
:10D6D0002B2B2B002B4349505354415455533A3074
:10D6E0000000000041542B434950535441545553BA
:10D6F000000000000A213046F5F763FC0B98401C3F
:10D700000B9003E00B98401C0B9000BF4BE00B9874
:10D710000078252840D10B98401C0B900078642895
:10D7200018D0732833D1019810C801900BE02178EC
:10D730003046F5F746FC00BF80213046F5F7F1FC96
:10D740000028F9D0641C20780028F0D10B98401CE8
:10D750000B9020E0019820C801900A2202A92846D7
:10D76000FFF7D9FE02AC0BE021783046F5F729FC33
:10D7700000BF80213046F5F7D4FC0028F9D0641CA6
:10D7800020780028F0D10B98401C0B9003E00B98F8
:10D79000401C0B9000BF06E00B9810F8011B0B908B
:10D7A0003046F5F70EFC00BF80213046F5F7B9FC96
:10D7B0000028F9D00B98007800287FF4E4AE06B07A
:10D7C00070BC5DF814FB70B5A0B004460D4616465B
:10D7D0002B4622463EA102A8009604F043FA4FF4DD
:10D7E000FA730022AFF2202102A8FFF7DFFC20B07D
:10D7F00070BD30B59FB004460D462B4622463FA172
:10D8000001A804F02FFA4FF4FA730022AFF2482176
:10D8100001A8FFF7CBFC1FB030BD10B59EB0044689
:10D8200022463CA1684604F01DFA4FF4FA73002228
:10D83000AFF26C216846FFF7B9FC1EB010BD30B5E1
:10D840009FB004460D462B46224637A101A804F09E
:10D8500009FA4FF47A730022AFF2942101A8FFF77E
:10D86000A5FC1FB030BD00B59FB036A101A804F0E3
:10D87000F9F94FF4FA730022AFF2B42101A8FFF7CF
:10D8800095FC1FB000BD70B504460D460026294624
:10D890002046FFF7D4FF4FF47A70F6F7D2FD012649
:10D8A000304670BD10B5C8212A4801F0F6FE29485F
:10D8B000B0F8C80020F400402649A1F8C800084686
:10D8C000B0F8C8006FF30E00A1F8C80010BD00004A
:10D8D00041542B4D515454555345524346473D30C6
:10D8E0002C312C222573222C222573222C222573E5
:10D8F000222C302C302C22220000000041542B4DD1
:10D90000515454434F4E4E3D302C222573222C252A
:10D91000642C300041542B4D5154545355423D30EA
:10D920002C222573222C310041542B4D515454503C
:10D9300055423D302C222573222C222573222C3176
:10D940002C30000041542B4D515454434C45414E12
:10D950003D300000847700202DE9F04106460F4657
:10D96000154600244FF480514548F3F76BF84FF407
:10D970007A70F6F766FD4FF480514148F3F760F88E
:10D980004FF47A70F6F75DFDFFF78EFC01E0601C46
:10D99000C4B24FF4FA7300223AA13BA0FFF706FC91
:10D9A00080F00100642C01DA012100E00021084030
:10D9B0000028ECD1002401E0601CC4B2032305223E
:10D9C00039463046FFF7F7FC80F00100642C01DA9D
:10D9D000012100E0002108400028EDD1002401E0F1
:10D9E000601CC4B20120FFF774FC80F00100642CBD
:10D9F00001DA012100E0002108400028F0D10024D4
:10DA000001E0601CC4B20120FFF798FC80F0010027
:10DA10000A2C01DA012100E0002108400028F0D1A1
:10DA2000002401E0601CC4B201212846FFF7ECFC91
:10DA300080F00100642C01DA012100E0002108409F
:10DA40000028EFD1BDE8F08110B500244FF4E1309B
:10DA5000FFF7A6FB0E4A02F10A01A1F11E00FFF733
:10DA60007BFF0AE0601CC4B24FF47A7002F044FC01
:10DA7000FFF73FFD022800D13D243C2CF2DB10BD16
:10DA8000000002404F4B00004154453000000000B0
:10DA9000A065002010B54FF48051FE48F2F7D0FF8A
:10DAA00010BD10B54FF48051FA48F2F7CBFF10BD0E
:10DAB0002DE9F04F91B006460F4614461D463046FC
:10DAC000394602F099F81090002801DB109901E026
:10DAD00010994942084602F07EF8824605F05EFB46
:10DAE000ED4AEE4BCDE90A0101F08FFFEA4AEC4B1B
:10DAF000CDE90E013046394601F087FF82462246C5
:10DB00002B4601F082FF22462B46CDE90A01E2486E
:10DB1000E24901F07AFF824622462B4601F075FF6A
:10DB200022462B46CDE906010020DE4901F06DFFBB
:10DB300000224FF08043CDE902013046394601F022
:10DB400064FF82460022D84B01F0B8FECDE9000107
:10DB5000DDE9022301F0B2FECDE90401DDE906238F
:10DB600001F0ACFECDE90801DDE90A2301F0A6FED3
:10DB7000CDE90C01DDE90E2301F0A0FE80468946C7
:10DB800000224FF080433046394601F03EFFC74A3D
:10DB9000C74BCDE9020101F038FF824605F0AEFA2D
:10DBA0000022C44BCDE9040101F02FFF0022C24B3B
:10DBB000CDE908013046394601F027FF8246BB4ACD
:10DBC000BB4B01F022FFCDE9020105F097FA0022DC
:10DBD000B84BCDE9040101F018FFCDE90601DDE9FC
:10DBE000082301F06BFE00224FF08043CDE90A01CB
:10DBF00001F00BFF0022AB4BCDE90C0101F077FFE8
:10DC000042464B46CDE90E0101F058FE804689465A
:10DC10000022A44B2046294601F069FF8246A34A10
:10DC2000A34B01F0F2FECDE9020105F067FA0022F4
:10DC3000A24BCDE9040101F0E8FE9C4A9C4BCDE9E2
:10DC400008012046294601F0E0FECDE9040105F077
:10DC500055FA82460022974B01F0D7FECDE9060126
:10DC6000DDE9082301F02AFE00224FF08043CDE9D0
:10DC70000A0101F0CAFE00228A4BCDE90C0101F035
:10DC800036FF42464B46CDE90E0101F017FE8046B5
:10DC90008946864A864B2046294601F0B6FE8246D2
:10DCA0000022874B01F023FFCDE9020105F026FA9F
:10DCB0000022844BCDE9040101F0A7FE0022824B33
:10DCC000CDE908012046294601F011FF774A784B3B
:10DCD000CDE9020101F099FE824605F00FFA00221B
:10DCE0007A4BCDE9040101F090FECDE90601DDE9B2
:10DCF000082301F0E3FD00224FF08043CDE90A0143
:10DD000001F083FE0022674BCDE90C0101F0EFFE2C
:10DD100042464B46CDE90E0101F0D0FD80468946D2
:10DD20004046494611B0BDE8F08F2DE9F04F8FB065
:10DD300004460D4692469B462046294601F05CFF6C
:10DD40000E90002801DB0E9901E00E994942084629
:10DD500001F041FFCDE9080105F020FA4E4A504B91
:10DD6000CDE90A0101F051FE4B4A4D4BCDE90C01C2
:10DD70002046294601F049FE52465B46CDE90601A0
:10DD800001F043FE444A464BCDE90A0120462946AC
:10DD900001F03BFE22462B46CDE9020101F035FEA3
:10DDA00052465B46CDE9060100204FF0804101F06C
:10DDB0002CFE0022464BCDE902012046294601F007
:10DDC0007DFDCDE90001DDE9022301F077FDCDE91C
:10DDD0000401DDE9062301F071FDCDE90801DDE96B
:10DDE0000A2301F06BFD8046DDE90C2301F066FD9E
:10DDF00006460F4600224FF080432046294601F098
:10DE000004FE8046294A2A4B01F0FFFDCDE90001BE
:10DE100005F074F90022274BCDE9020101F0F5FD70
:10DE20000022254BCDE906012046294601F0EDFDF3
:10DE300080461E4A1E4B01F0E8FDCDE9000105F0C9
:10DE40005DF900221B4BCDE9020101F0DEFDCDE9B9
:10DE50000401DDE9062301F031FD00224FF080438B
:10DE6000CDE9080101F0D1FD00220E4BCDE90A01F8
:10DE700001F03DFE32463B46CDE90C0101F01EFDAE
:10DE800006460F460022074B2046294601F02FFE8A
:10DE9000064A1FE0000402409A9999999999C93F4E
:10DEA0009999B93F00000840000059C0182D44540A
:10DEB000FB210940000034400000184000004440AD
:10DEC00000003E4000007440000028400000644014
:10DED00000C07240FE4BCDE9000101F096FD804686
:10DEE00005F00CF90022FB4BCDE9020101F08DFD9C
:10DEF000F94AF74BCDE906012046294601F085FD98
:10DF0000CDE9020105F0FAF880460022F34B01F05A
:10DF10007CFDCDE90401DDE9062301F0CFFC002200
:10DF20004FF08043CDE9080101F06FFD0022EC4B7A
:10DF3000CDE90A0101F0DBFD32463B46CDE90C019B
:10DF400001F0BCFC06460F460022E64B204629465F
:10DF500001F0CDFD8046E04ADD4B01F056FDCDE9F4
:10DF6000000105F0CBF80022DF4BCDE9020101F002
:10DF70004CFD0022DD4BCDE906012046294601F08B
:10DF8000B6FDD54AD24BCDE9000101F03EFD8046F9
:10DF900005F0B4F80022D64BCDE9020101F035FDC1
:10DFA000CDE90401DDE9062301F088FC00224FF0F1
:10DFB0008043CDE9080101F028FD0022C84BCDE9DE
:10DFC0000A0101F094FD32463B46CDE90C0101F017
:10DFD00075FC06460F46304639460FB0BDE8F08F57
:10DFE0000FB42DE9F04F8FB0DDE91A45DDE91C676C
:10DFF000C04AC14B3046394601F007FDCDE9020168
:10E0000005F07CF8BD4ABE4BCDE9040101F0FDFCF2
:10E0100032463B46CDE908013046394601F0F5FC71
:10E0200022462B46CDE902012046294601F0EDFCAF
:10E03000CDE90001DDE9022301F040FCCDE9040156
:10E0400005F0ACF8CDE90601DDE9082301F036FC66
:10E0500080468946A74AA84B2046294601F0D5FCB0
:10E06000CDE9020104F09EFFA64AA74BCDE90401C9
:10E0700001F0CBFC22462B46CDE90801304639465B
:10E0800004F0D0FECDE90601DDE9082301F016FC1D
:10E0900082468B465046594604F084FF42464B4622
:10E0A000CDE9060101F0B1FC984A994BCDE9080190
:10E0B00001F004FCCDE90A015046594605F01EF86E
:10E0C00042464B46CDE9060101F09FFC914A924B36
:10E0D000CDE9080101F0F2FBCDE90C010AA991E8B4
:10E0E0000E101898A0E80E100FB0BDE8F00F5DF804
:10E0F00014FB0FB42DE9F04F91B0DDE91E010022B1
:10E10000864BCDE9040101F07AFCCDE90801DDE997
:10E110001C010022824BCDE9040101F070FCCDE925
:10E120000601DDE90823FFF7C3FC06460F46DDE9DB
:10E130001E010022794BCDE9040101F060FCCDE91C
:10E140000801DDE91C010022754BCDE9040101F055
:10E1500056FCCDE90601DDE90823FFF7E6FD804620
:10E160008946DDE91E0100226E4BCDE9060101F072
:10E17000BEFC594A564BCDE9080101F046FCCDE9F9
:10E180000A01DDE90A0104F0B9FF04460D46224602
:10E190002B466548654901F038FC22462B46CDE9FF
:10E1A000060101F032FC0022614BCDE9080101F0CB
:10E1B00029FC04460D462046294604F0EFFF82461E
:10E1C0008B4652465B462046294601F01EFC02461D
:10E1D0000B46CDE902015748574901F088FC3E4AF9
:10E1E0003B4BCDE9040101F010FC00224D4BCDE981
:10E1F00008013046394601F008FCCDE90601DDE9A9
:10E20000082301F074FC06460F46DDE90A0104F01C
:10E21000C9FE52465B46CDE902014FF080404749B6
:10E2200001F065FCCDE90001DDE9022301F0EDFB21
:10E23000294A274BCDE9040101F0E7FB0022394BC5
:10E24000CDE908014046494601F0DFFBCDE9060172
:10E25000DDE9082301F04BFC80468946DDE91E011B
:10E2600032463B46CDE9080101F028FBCDE90E011D
:10E27000DDE91C0142464B46CDE9080101F01EFBD9
:10E28000CDE90C010CA991E80E101A98A0E80E1027
:10E2900011B0BDE8F00F5DF814FB2DE9F04F89B027
:10E2A0008246274903C901F0A7FC834601F093FC8D
:10E2B000CDE9000122480CC8009801F0A3FB002220
:10E2C000204BCDE9020101F0A0FB804600223BE09B
:10E2D000FB21094000004440182D44540000344004
:10E2E0000000084000003E4000C07240000028408E
:10E2F00000C062404E04C777102E4A40F168E388A0
:10E30000B5F8F43E54E41071732AC93E39B4C876A6
:10E31000BE9F7A3FFA7E6ABC7493783F008041408A
:10E3200000405A40008066400BEF80AF8F6A7B3F11
:10E330000000F03FC155E32D102B5841C154584106
:10E340002863002000005940FE4B01F0D0FB04463A
:10E350000D46FD4903C901F04FFC804601F03BFC2E
:10E36000064622462B4601F0A9FACDE90601F749F7
:10E3700003C901F041FC834601F02DFCCDE9000109
:10E38000F2480CC8009801F03DFB0022F04BCDE9AB
:10E39000020101F03AFB06460022EA4B01F0A7FB1E
:10E3A00004460D46E94903C901F026FC064601F082
:10E3B00012FC804622462B4601F080FACDE904018A
:10E3C00004A80FC88AE80F0009B0BDE8F08F2DE956
:10E3D000F04F8BB08246DC4903C901F00DFC834647
:10E3E00001F0F9FBCDE90201D7480CC8029801F011
:10E3F00009FB0022D64BCDE9040101F006FB0646DD
:10E400000022D04B01F073FB04460D46CE4903C9F0
:10E4100001F0F2FB064601F0DEFB804622462B4669
:10E4200001F04CFACDE90801C84903C901F0E4FB49
:10E43000834601F0D0FBCDE90201C4480CC8029824
:10E4400001F0E0FA0022C24BCDE9040101F0DDFA4F
:10E4500080460022BB4B01F04AFB04460D46BB49F7
:10E4600003C901F0C9FB804601F0B5FB0646224610
:10E470002B4601F023FACDE90601DDE90801CDE9DB
:10E48000000102A8DDE90623FFF733FE02A80FC84A
:10E4900006AD0FC506A80FC88AE80F000BB0BDE88F
:10E4A000F08F2DE9F04F8BB08246A74903C901F0E8
:10E4B000A3FB834601F08FFBCDE90201A2480CC803
:10E4C000029801F09FFA0022A14BCDE9040101F06E
:10E4D0009CFA064600229B4B01F009FB04460D46C0
:10E4E000994903C901F088FB064601F074FB804698
:10E4F00022462B4601F0E2F9CDE90801934903C910
:10E5000001F07AFB834601F066FBCDE902018F48FA
:10E510000CC8029801F076FA00228D4BCDE9040177
:10E5200001F073FA80460022864B01F0E0FA0446BF
:10E530000D46864903C901F05FFB804601F04BFBA5
:10E54000064622462B4601F0B9F9CDE90601DDE980
:10E550000801CDE9000102A8DDE90623FFF7C9FDA6
:10E5600002A80FC806AD0FC5DDE90801CDE900011D
:10E5700002A8DDE90623FFF733FD02A80FC806ADA8
:10E580000FC506A80FC88AE80F000BB0BDE8F08FD2
:10E59000704710B54F216F4801F07FF800206D499A
:10E5A00081F8A00081F8A10001F1A2000021016022
:10E5B0004160018181720B30016041600181817293
:10E5C0000B300180817075388167C167C0F8801099
:10E5D00084300180817000205E4981F8CA0010BD3E
:10E5E0002DE9F04FA1B000265A4890F8A00000286D
:10E5F00074D00020574981F8A00000BFE4E12EB993
:10E6000055A1544801F054F80446DBE1641C52A1C2
:10E61000204601F04DF8051E6AD00A2E42D2DFE8EE
:10E6200006F041050C121920272E343A2A1B2146E8
:10E630004848A23001F018F835E02A1B21461DA8F1
:10E6400001F012F82FE02A1B21464248AD3001F0BC
:10E650000BF828E02A1B21463E48B83001F004F8A8
:10E6600021E02A1B21463B48BB3000F0FDFF1AE0A9
:10E670002A1B21463748C73000F0F6FF13E02A1B5B
:10E6800021461AA800F0F0FF0DE02A1B214617A82A
:10E6900000F0EAFF07E02A1B21462E48CB3000F0AD
:10E6A000E3FF00E000BF00BF2C460120294981F8AC
:10E6B000A1009DF87400412801D1012000E0002054
:10E6C000244991F8CB1009B1012100E00021084054
:10E6D00028B101201F4981F8CA0008E077E19DF8C0
:10E6E0007400562803D100201A4981F8CA0000BFDF
:10E6F000184991F8B510A1F1300001F06CFA074605
:10E700000022164B01F081F9CDE91C01114991F865
:10E71000B410A1F1300001F05EFA07460022104B60
:10E7200001F073F9CDE918010A4991F8B310A1F18C
:10E73000300001F050FA07460022054B01F065F960
:10E7400010E0000000004E402863002030630020ED
:10E75000000059404E7800202C0000000000F03FDF
:10E7600000002440CDE91401F84991F8B210A1F15C
:10E77000300001F030FA07460022F54B01F045F970
:10E78000CDE91001F14991F8B010A1F1300001F08C
:10E7900022FA07460022EF4B01F037F9CDE90C01D0
:10E7A000EA4991F8AF10A1F1300001F014FA0746E0
:10E7B0000022E94B01F029F9CDE90801E34991F87C
:10E7C000AE10A1F1300001F006FA07460022E34B3B
:10E7D00001F01BF982468B46DC4991F8AD10A1F19E
:10E7E000300001F0F8F907460022DD4B01F00DF989
:10E7F00052465B46CDE9040101F060F8CDE906011F
:10E80000DDE9082301F05AF8CDE90A01DDE90C231E
:10E8100001F054F8CDE90E01DDE9102301F04EF8C6
:10E82000CDE91201DDE9142301F048F8CDE9160124
:10E83000DDE9182301F042F8CDE91A01DDE91C23D6
:10E8400001F03CF8C74A03C2C04991F8C410A1F1D5
:10E85000300001F0C0F907460022C34B01F0D5F8A3
:10E86000CDE91C01B94991F8C310A1F1300001F0C4
:10E87000B2F907460022BD4B01F0C7F8CDE91801F7
:10E88000B24991F8C210A1F1300001F0A4F9074695
:10E890000022B74B01F0B9F8CDE91401AB4991F86A
:10E8A000C110A1F1300001F096F907460022A84BF3
:10E8B00001F0ABF8CDE91001A44991F8BF10A1F126
:10E8C000300001F088F907460022A24B01F09DF8C4
:10E8D000CDE90C019D4991F8BE10A1F1300001F085
:10E8E0007AF9074600229C4B01F08FF8CDE9080128
:10E8F000964991F8BD10A1F1300001F06CF907467E
:10E900000022964B01F081F8CDE904018F4991F87E
:10E91000BC10A1F1300001F05EF907460022904BD7
:10E9200001F073F882468B46884991F8BB10A1F13B
:10E93000300001F050F9074600228E4B01F065F8D7
:10E9400052465B46CDE9000100F0B8FFCDE9020177
:10E95000DDE9042300F0B2FFCDE90601DDE908237B
:10E9600000F0ACFFCDE90A01DDE90C2300F0A6FFC1
:10E97000CDE90E01DDE9102300F0A0FFCDE9120181
:10E98000DDE9142300F09AFFCDE91601DDE9182333
:10E9900000F094FFCDE91A01DDE91C2300F08EFFA1
:10E9A000754A03C200226D4B6E4903C901F09FF8FE
:10E9B0006C4A03C20022694B6F4903C901F097F802
:10E9C0006D4A03C2701CC6B2092E7FF718AE002034
:10E9D0001E901F9020905D4890F8CF008DF8780031
:10E9E0005A4890F8D0008DF879002D208DF87A00E3
:10E9F000564890F8CD008DF87B00544890F8CE0032
:10EA00008DF87C002D208DF87D00504890F8CB00CB
:10EA10008DF87E004D4890F8CC008DF87F001EA840
:10EA200000F062FE07463A461EA94848CB3000F087
:10EA30001BFE00201E901F902090444890F8A300D9
:10EA40003038424991F8A210303901EB810100EBD6
:10EA50004100083000F0FF090A2099FBF0F0303047
:10EA60003A4981F8A2000A2099FBF0F100FB1190CD
:10EA70003030C1B2354880F8A31090F8A2008DF86C
:10EA80007800324890F8A3008DF879003A208DF88C
:10EA90007A002E4890F8A4008DF87B002B4890F85F
:10EAA000A5008DF87C003A208DF87D00274890F86D
:10EAB000A6008DF87E00254890F8A7008DF87F000D
:10EAC0002248A230002101604160018181721EA8AC
:10EAD00000F00AFE07463A461EA91C48A23000F084
:10EAE000C3FD00201E901F90209021B0BDE8F08F44
:10EAF00010B50024154890F8A10000287ED000BF72
:10EB00000020124981F8A1001CA003F09BF806E048
:10EB10000E48A230015D1FA003F094F8641C0B485E
:10EB2000A230005D0028F3D11BA003F08BF807484A
:10EB300090F8CA0000287DD00020044981F8CA005E
:10EB4000002416A003F07EF83BE000004E78002081
:10EB500000408F400088C340006AF84080842E4106
:10EB6000D0126341286300200000F03F00002440E1
:10EB70000000594084D79741306300205361766587
:10EB80005F446174612E55544354696D65203D2086
:10EB900000000000256300000D0A00005361766547
:10EBA0005F446174612E6C61746974756465203DA5
:10EBB000200000005448015DAFF2280003F042F845
:10EBC000641C5148005D0028F4D1AFF2340003F01A
:10EBD00039F800244DA003F035F84B48AD3890F8D3
:10EBE000B810AFF2500003F02DF84748AD3890F858
:10EBF000B910AFF2600003F025F800E036E0AFF2A4
:10EC0000680003F01FF800BF45A003F01BF807E001
:10EC10003D480E30015DAFF2840003F013F8641C30
:10EC200039480E30005D0028F2D1AFF2940003F0B5
:10EC300009F800E017E040A003F004F83248AD38CE
:10EC400090F8C710AFF2B40002F0FCFF2E48AD38C8
:10EC500090F8C810AFF2C40002F0F4FFAFF2C800A1
:10EC600002F0F0FF02E039A002F0ECFF10BD70B539
:10EC70008EB0002400202449AD3981F8D60035E05B
:10EC80004FF47A70F5F7DDFB1F48AD3890F8A0001F
:10EC900008B1FFF7A5FC601CC4B21B48AD3890F862
:10ECA000CA00F8B106A8FFF7F8FA06A80FC80AAD1F
:10ECB0000FC53D242C2114481A30CDE906100891C7
:10ECC000DDE90A01CDE904012C210F480B30CDE923
:10ECD00000100291DDE90C532A4623A1284802F0D6
:10ECE000C1FF03E027A1264802F0BCFF232CC7DBAD
:10ECF000FFF74FFC2748F4F771F801200249AD39BE
:10ED000081F8D6000EB070BDFB78002053617665A7
:10ED10005F446174612E4E5F53203D20000000006F
:10ED2000536176655F446174612E6C6F6E676974C0
:10ED3000756465203D200000536176655F44617411
:10ED4000612E455F57203D200000000047505320B2
:10ED500044415441206973206E6F74207573656659
:10ED6000756C6C210D0A0000252E3766256325730E
:10ED70002563252E37662563257325630000000073
:10ED8000FC6F00204E612C4E612C4E612C4E612C8C
:10ED900000000000003801401CB5F748F4F71EF8E9
:10EDA00001210220F2F7AEF8C020009001208DF87A
:10EDB000040002208DF8050000208DF806000120D7
:10EDC0008DF807006946ED48F1F7C0FD4021EB489A
:10EDD000F1F738FE1CBD10B54FF49660F8F724FA31
:10EDE00010BD10B52021E548F1F72CFE4021E34885
:10EDF000F1F728FE1420F5F724FB4021DF48F1F756
:10EE00001FFE10BD1CB500240020009001900124BD
:10EE10001FE0002000900190D9A32246D9A16846A6
:10EE200002F020FFFFF7B8FFFFF7DBFFFFF7D3FF8C
:10EE30006946D6A0F8F765FA0820F5F702FB20210D
:10EE4000CE48F1F7FDFD4FF4FA70F5F7FAFA601CC1
:10EE5000C4B20A2CDDDB1CBD10B54FF0FF31CC482D
:10EE6000006801F09FFBF5F7C6FB0020C949087058
:10EE7000FFF792FFF8F736FAFFF7B3FFFFF7ABFFA4
:10EE8000C5A1C2A0F8F73DFA0820F5F7DAFA20216B
:10EE9000BA48F1F7D5FD4FF4FA70F5F7D2FABC484D
:10EEA000006801F0A3FBBDA1BD4800F001FC041EF9
:10EEB00002D0641E207810BD7F20FCE730B585B0FD
:10EEC00004460D460020029003900490411EB04875
:10EED000006801F067FB212041232246B1A1CDE962
:10EEE000005002A802F0BEFEF5F785FB0020A949FC
:10EEF0000870FFF751FFF8F7F5F9FFF772FFFFF71A
:10EF00006AFF02A9A1A0F8F7FCF90820F5F799FA21
:10EF100020219A48F1F794FD4FF4FA70F5F791FA31
:10EF20009B48006801F062FB05B030BD7CB504462B
:10EF3000002000900190F8F7D5F900200090019092
:10EF40009BA322469BA1684602F08CFEF8F7CAF903
:10EF5000FFF722FFFFF745FFFFF73DFF69468BA054
:10EF6000F8F7CFF90820F5F76CFA20218348F1F77C
:10EF700067FD4FF4FA70F5F764FA90A1884800F045
:10EF800097FB05468EA1864800F092FB06460DB120
:10EF9000012000E000200EB1012100E00021084323
:10EFA00008B100207CBD0120FCE72DE9F0418AB0CA
:10EFB00080460020834981F80E0178A1784800F04E
:10EFC00077FB002875D000200790089009900490E6
:10EFD0000590069001900290039078A1704800F08F
:10EFE00067FB054676A16E4800F062FB044604B953
:10EFF0006C1C05B9651CA54201D9264600E02E46C9
:10F000006EA1701C00F054FB05466DA1701C00F051
:10F010004FFB044604B96C1C05B9651CA54201D917
:10F02000274600E02F46BA1B314607A800F01CFB1C
:10F030003E4662A1701C00F03BFB054660A1701CBF
:10F0400000F036FB044604B96C1C05B9651CA542EA
:10F0500001D9274600E02F46BA1B314604A800F02C
:10F0600003FB3E464DA1304600F022FB0746BA1B8B
:10F07000314601A800F0F8FAB8F10A0F60D2DFE8D3
:10F0800008F05F050E19232D37414B5501A804AB3D
:10F0900007AA4DA100904B4802F0E4FD51E001A801
:10F0A00004AB07AA48A1009046481E3002F0DAFDE2
:10F0B00047E04CE001A804AB07AA43A100904148F7
:10F0C0003C3002F0CFFD3CE001A804AB07AA3EA112
:10F0D00000903C485A3002F0C5FD32E001A804AB74
:10F0E00007AA39A100903748783002F0BBFD28E02C
:10F0F00001A804AB07AA34A100903248963002F070
:10F10000B1FD1EE001A804AB07AA2FA100902D4875
:10F11000B43002F0A7FD14E001A804AB07AA2AA1AD
:10F1200000902848D23002F09DFD0AE001A804AB0F
:10F1300007AA25A100902348F03002F093FD00E0DB
:10F1400000BF00BF01201F4981F80E017BE0B8F12C
:10F150000A0F76D2DFE808F075050A444A51585F75
:10F16000666E1CA1174802F07DFD6BE019A11548E1
:10F170001E3002F077FD65E00038014000040240D7
:10F180004D21000025642573000000002573000058
:10F19000BC6200206D6200203F2100000D0A0000CB
:10F1A0004468002025632563256325630000000073
:10F1B0004430210025632573000000002B0000006F
:10F1C0002D0000002579002025732C25732C257334
:10F1D000000000004E612C4E612C4E6100000000CA
:10F1E000AFF21001594802F03DFD2BE0AFF21C01D7
:10F1F00056481E3002F036FD24E0AFF22801534895
:10F200003C3002F02FFD1DE0AFF238014F485A307C
:10F2100002F028FD16E0AFF244014C48783002F0CD
:10F2200021FD0FE0AFF254014848963002F01AFD7C
:10F2300008E006E0AFF264014448B43002F012FD89
:10F2400000E000BF00BF0AB0BDE8F0811CB500249B
:10F25000002000900190012429E0F8F743F80020F5
:10F2600000900190AFF2B8032246AFF2E801684681
:10F2700002F0F8FCF8F736F8FFF78EFDFFF7B1FD66
:10F28000FFF7A9FD6946AFF2FC00F8F73AF808204D
:10F29000F5F7D7F820212E48F1F7D2FB4FF4FA709A
:10F2A000F5F7CFF82046FFF780FE601CC4B20A2CA9
:10F2B000D3DB1CBD10B51E2124483C3800F0EDF90D
:10F2C0001E2122481E3800F0E8F91E211F4800F0D8
:10F2D000E4F91E211D481E3000F0DFF91E211B48F5
:10F2E0003C3000F0DAF91E2118485A3000F0D5F908
:10F2F0001E211648783000F0D0F91E2113489630B0
:10F3000000F0CBF91E211148B43000F0C6F910BD51
:10F3100010B54FF0FF310F48006801F043F9FFF7D7
:10F320003BFDF5F768F900200B490870FFF7C2FFB5
:10F33000FFF768FD4FF4FA70F5F783F8FFF786FFE3
:10F340000448006801F052F910BD00006179002006
:10F3500000040240BC6200206D620020014601F002
:10F360000F00091101F00F0101EB81025100421859
:10F37000D0B2704730B501460A2491FBF4F4E2B2F2
:10F380000A2491FBF4F504FB1514E3B203EB021419
:10F39000E0B230BD70B505460C46F8F7CDFE05204D
:10F3A000F5F73DF8D020F8F798FFF8F71AFF052099
:10F3B000F5F735F82846F8F790FFF8F712FF052023
:10F3C000F5F72DF82046F8F788FFF8F70AFF052033
:10F3D000F5F725F8F8F7DCFE70BD70B5044600259A
:10F3E000F8F7AAFED020F8F778FFF8F7FAFE052024
:10F3F000F5F715F82046F8F770FFF8F7F2FE05204C
:10F40000F5F70DF8F8F798FED120F8F766FFF8F752
:10F41000E8FE0520F5F703F80020F8F798FF054609
:10F42000F8F7B6FE284670BD10B5F8F769FE402122
:10F430000E20FFF7AFFF0220F5F703F800210F20A1
:10F44000FFF7A8FF0220F4F7FCFF10BD10B506205F
:10F45000FFF7C3FF554948600520FFF7BEFF53493A
:10F4600008720420FFF7B9FF504948720220FFF7E5
:10F47000B4FF4E4908700120FFF7AFFF4B494870B9
:10F480000020FFF7AAFF4949887010BD2DE9F04719
:10F4900007460C4615461E46DDE908894FF0000A6E
:10F4A0003846FFF767FF00F0FF0A51460620FFF7D6
:10F4B00071FF4FF0000A2046FFF75CFF00F0FF0AE3
:10F4C00051460520FFF766FF4FF0000A2846FFF778
:10F4D00051FF00F0FF0A51460420FFF75BFF4FF099
:10F4E000000A3046FFF746FF00F0FF0A51460220AF
:10F4F000FFF750FF4FF0000A4046FFF73BFF00F0D8
:10F50000FF0A51460120FFF745FF4FF0000A484629
:10F51000FFF730FF00F0FF0A51460020FFF73AFFE7
:10F52000BDE8F08710B50620FFF757FF1F49486078
:10F530000879FFF713FF1D4948600520FFF74DFFCD
:10F540001A490872087AFFF709FF1849087204205F
:10F55000FFF743FF15494872487AFFF7FFFE13494A
:10F5600048720220FFF739FF1049087008460078FA
:10F5700000F03F0008700878FFF7F0FE0B490870B4
:10F580000120FFF72AFF094948704878FFF7E6FE97
:10F59000064948700020FFF720FF044988708878EA
:10F5A000FFF7DCFE0149887010BD0000347A0020AE
:10F5B00000BFFEE7062809D2DFE800F008030405D3
:10F5C000060704E003E002E001E000E000BF00BF46
:10F5D00000BFFEE71EF0040F0CBFEFF30880EFF34F
:10F5E0000980816911F8021CD9B901B590E80F10A2
:10F5F000E047BDE800508CE80300194B93E8060093
:10F60000914208BF704719B12CE9F00FC1F838C01A
:10F610001A60906BB0E8F00F80F309886FF0020E6B
:10F620007047104A13689942FAD801B552F821C0C0
:10F630000FC8E047BDE80050CCF80000704700005C
:10F6400001B501F077F9BDE80140EFF3098CD4E78B
:10F6500001B501F0CBFBBDE80140EFF3098CCCE72D
:10F660005C6300206838020840EA01039B0703D06E
:10F6700009E008C9121F08C0042AFAD203E011F8F1
:10F68000013B00F8013B521EF9D27047D2B201E0B3
:10F6900000F8012B491EFBD270470022F6E710B597
:10F6A00013460A4604461946FFF7F0FF204610BDF0
:10F6B00030B505462A460B4612F8010B13F8014BEC
:10F6C00008B1A042F8D01CB1002802D06D1CF1E7AF
:10F6D000284630BDCAB2401E10F8011F8A4202D02F
:10F6E0000029F9D100207047421C10F8011B0029A5
:10F6F000FBD1801A704710B5002200E0521C835CD9
:10F700008C5CA34201D1002BF8D1D8B2E1B2401AEF
:10F7100010BD30B504460020034600E05B1C934258
:10F7200003D2E05CCD5C401BF8D030BDF0B480EA81
:10F730000102D40F4200B2EB410F02D2024608464A
:10F7400011464A0042D0C30DDDB2C1F3C752AD1A13
:10F75000202D35DAC1F3160141F4000204B1524202
:10F76000C5F1200602FA06F12A411044B3EBD05F3E
:10F7700023D0C4B1012DA0EBC35009DCF0BC4FF085
:10F78000004202EAC352DBB200F5000000F003BB06
:10F79000400000F1807000EBC350A0F1807040EA9F
:10F7A000D170490009E0490841EAC071A0EBC3509B
:10F7B00000F50000400800EBC350F0BC00F0E2BAD6
:10F7C0006142012202EB4101001BF6E7F0BC7047E9
:10F7D00081F00041AAE780F00040A7E780EA01023B
:10F7E00010B502F00043400022D04A001FD0010EA5
:10F7F00001EB1261C0F35600C2F3560240F4000060
:10F8000042F40002A0FB022000047F39140400D05F
:10F81000401C50EA124001D44000491EC2B20C06FE
:10F8200004EBD010401C4008802A02D003E00020E6
:10F8300010BD20F00100002900DA0020184310BD9F
:10F8400030B480EA010202F0004530F0004221F0BD
:10F85000004013D090B1C30DD40DC2F31601C0F314
:10F860001600E41A41F4000140F400027D34914294
:10F8700001D3641C00E04900002C02DA30BC0020F7
:10F8800070474FF400000023914201D3891A0343CB
:10F8900040084FEA4101F7D151B1914202D14FF0F6
:10F8A000004105E002D24FF0010101E06FF00101DB
:10F8B00003EBC450284430BC00F064BA2DE9FE4F7D
:10F8C000804681EA0300C00F0C46009021F0004101
:10F8D00023F00045B8EB0200A94105D2404621467D
:10F8E00090461C460B46024623F00040104347D08A
:10F8F000270DC7F30A00C3F30A510290401A019082
:10F9000040286BDAC3F3130040F4801B0098924642
:10F9100020B10023D2EB030A63EB0B0B019859468D
:10F92000C0F14002504600F0FCF906460D46504634
:10F930005946019A00F014FA10EB080061410024C6
:10F9400087EA115284EAE7731A4340D0009A62B3FF
:10F95000019A012A4FEA075215DC001B61EB0201F4
:10F960004FF0004202EA0752CDE90042001C41F587
:10F97000801132462B4600F04BFA03B0BDE8F08F01
:10F9800040462146F9E7001B61EB0201001C41F5EE
:10F99000801300185B412018A2F5001747EB030104
:10F9A00040EAD570B6196D4111E06D084FEA360690
:10F9B00045EAC0754FEA0752001B61EB0201001CCB
:10F9C00041F5801149084FEA300000195141324693
:10F9D0002B4603B0BDE8F04F00F00BBA00980122AF
:10F9E00040000023D0EB020263EBE0730098214655
:10F9F0004FEAE074B8EB000061EB0401E9E783F043
:10FA000000435BE781F0004158E72DE9FE4F81EAB2
:10FA1000030404F0004421F0004100944FF0000B77
:10FA200023F0004350EA01045ED052EA03045BD0A5
:10FA3000C3F30A54C1F30A552C44A4F2F3340194DD
:10FA4000A0FB0254C1F3130141F48011C3F313036B
:10FA500043F4801301FB024400FB034E840A970A1F
:10FA600044EA815447EA8357A4FB076802958D0A4C
:10FA700005FB07854FEA932C04FB0C542705029DD8
:10FA80004FEA065847EA1637B5EB08056EEB070C48
:10FA9000870E920E47EA811742EA8312A7FB020102
:10FAA000B6EB0B0164EB00042B0D43EA0C335E183C
:10FAB00044EB1C50DA465146E7FB0201C5F3130440
:10FAC0004FEA0B3343EA14534FEA0432019C43EAF2
:10FAD0000603A4F10C040294009CCDE900B400F0EC
:10FAE00097F903B0BDE8F08F00200146F9E72DE952
:10FAF000F04D81EA030404F0004B21F00045144668
:10FB00004FF0000A23F0004150EA050220D054EAE9
:10FB100001021DD0C5F30A570246C5F31303C1F312
:10FB20001300C1F30A5640F4801543F48013A7EB89
:10FB30000608101BD64608F2FD3873EB050002D309
:10FB400008F1010801E092185B41B8F1000F03DAF7
:10FB500000200146BDE8F08D00204FF480110646DC
:10FB600084460EE0171B73EB050705D3121B63EBEE
:10FB7000050306434CEA010C49084FEA300092188D
:10FB80005B4150EA0107EDD152EA030012D082EA4C
:10FB9000040083EA0501084305D0101BAB4106D2DF
:10FBA0000122002306E000224FF0004302E06FF044
:10FBB000010253101AEB06004CEB085110EB0A003F
:10FBC00041EB0B01BDE8F04D00F013B99623002284
:10FBD000114600F0E0B80EB5C10F80EAE0700844AD
:10FBE000CA07002140F233438DE80E000A460B4657
:10FBF00000F00EF903B000BD70B5C1F30A5201F078
:10FC000000450024C1F3130140F2FF3341F4801199
:10FC10009A4201DA002070BD40F233439A42A2F2C8
:10FC2000334203DC524200F08BF800E090402C435A
:10FC3000F1D0404270BD00F0004230F000400AD0E8
:10FC4000C10D01F56071C0F3160042EA0151C2080E
:10FC500040071143704700200146704701F0004300
:10FC600030B421F0004150EA010206D00A0DA2F59D
:10FC70006072C1F31301002A02DC30BC002070471F
:10FC8000440F44EAC104C100E01830BC00EBC2508C
:10FC900000F078B830B50B46014600202022012440
:10FCA00009E021FA02F59D4205D303FA02F5491B4A
:10FCB00004FA02F52844151EA2F10102F1DC30BD60
:10FCC0002DE9F05F0546002092469B468846064691
:10FCD000814640241BE0284641464746224600F024
:10FCE0002FF853465A46C01A914110D31146184670
:10FCF000224600F016F82D1A67EB01084F462246FF
:10FD00000120002100F00DF817EB00094E41201EE4
:10FD1000A4F10104DFDC484631462A464346BDE8EB
:10FD2000F09F202A04DB203A00FA02F100207047FD
:10FD30009140C2F1200320FA03F319439040704729
:10FD4000202A04DB203A21FA02F00021704721FA30
:10FD500002F3D040C2F12002914008431946704797
:10FD6000202A06DBCB17203A41FA02F043EAE0737F
:10FD700006E041FA02F3D040C2F12002914008436C
:10FD8000194670470029A8BF7047401C490008BFAA
:10FD900020F00100704710B4B0FA80FC00FA0CF0BB
:10FDA00050EA010404BF10BC704749B1CCF12004F3
:10FDB00021FA04F411FA0CF118BF01212143084380
:10FDC000A3EB0C01CB1D4FEA00614FEA102042BFAC
:10FDD000002010BC704700EBC35010440029A4BFA2
:10FDE00010BC7047401C490008BF20F0010010BC47
:10FDF000704710B5141E73F1000408DA401C41F17D
:10FE0000000192185B411A4301D120F0010010BD9E
:10FE10002DE9F04D92469B4611B1B1FA81F202E014
:10FE2000B0FA80F220329046FFF77BFF04460F467F
:10FE300040EA0A0041EA0B0153465A46084313D0F0
:10FE4000114653EA010019D0C8F140025046FFF7AD
:10FE500077FF05460E46504659464246FFF761FF7A
:10FE6000084305D0012004E020463946BDE8F08D66
:10FE70000020054346EAE0762C4337430A986305A1
:10FE8000E40AA0EB08000022FD0A44EA47540A30C5
:10FE900002D500200146E9E7010510196941DDE9B5
:10FEA000084500196941BDE8F04DA2E72DE9F04D84
:10FEB00000231A461B1A8A4103DB00200146BDE8D5
:10FEC000F08DC1F30A52C1F3130141F480154FF0D4
:10FED000000BD10702D100186D41521E00270446C5
:10FEE00040F2FF11384601EB620A3E468046024668
:10FEF00000204FF48011FFF723FFC2197141BB1896
:10FF000046EB0100B4EB030C75EB000C04D3E41AD0
:10FF100065EB000517460E46241908F101006D41F6
:10FF200080463428E3DDF91946EB0600091BA84199
:10FF300003D24FF0FF32134601E0002213461BEBC1
:10FF4000070046EB0A51BDE8F04DFFF752BFC1F381
:10FF50000A52C1F3130140F2FF3341F480119A4277
:10FF600002DA00200146704740F233439A42A2F27F
:10FF7000334202DC5242FFF7E3BEFFF7D2BE00007D
:10FF800030B5041E71F1000404DB4FF00044404220
:10FF900064EB0101141E73F1000405DB1C464FF0F5
:10FFA0000043524263EB0403994208BF904230BDC4
:10FFB000064C074D06E0E06840F0010394E80700B6
:10FFC00098471034AC42F6D3F0F7B0F8143F02086B
:10FFD000343F020870B521F0004303430CD0C1F355
:10FFE0000A550024D5EB040564EB0403D617AD1ABB
:10FFF000B34102DB0020014670BD201841EB0251E5
:020000040802F0
:1000000070BD0EB540F2334102910021CDE90011DF
:100010000A460B46FFF7FCFE03B000BD70B58C1816
:1000200010F8015B15F0070301D110F8013B2A110C
:1000300006D110F8012B03E010F8016B01F8016BF9
:100040005B1EF9D12B0705D40023521E0DD401F8F5
:10005000013BFAE710F8013BCB1A921C03E013F8BE
:10006000015B01F8015B521EF9D5A142D8D30020F3
:1000700070BD10B5930712D400F10C03D0071ED148
:1000800053E8000F084203D1BFF32F8F002005E093
:1000900020EA010243E8002404B1F1E710BDC06882
:1000A00000EA01038B42014618BF002112F0010251
:1000B00008BF014653EA020018BF084610BD53E8C6
:1000C000000F00EA01028A4203D0BFF32F8F002005
:1000D00005E020EA010243E8002404B1EFE710BD87
:1000E00010B500F1280151E8002F12B9BFF32F8F8E
:1000F00004E0531E41E8003404B1F4E772B12C303F
:100100000121006850B1821CD2E84F3FC2E8441F71
:1001100004B1F9E71A0602D00830F2E7002010BD5A
:1001200070B5024652F8305F4DB1CC7800235DB116
:100130002E46ED78A5420DD275683346F7E70023C9
:10014000C1E90133C1620DE00024C1E9014300F1BE
:100150002C0403E0C1E9016306F108042160002BCF
:1001600018BF1A1D1160283050E8001F4A1C40E8D3
:10017000002303B1F8E770BDD1E90123002A0EBFC7
:10018000C36293608B68191D002B08BF00F130011A
:100190000A60704701480068704700BF10E000E047
:1001A00007480178012905D106494FF080620A60AD
:1001B000002101700448016841F0010101607047AD
:1001C000407A002004ED00E010E000E04FF0FF3046
:1001D0007047000040B10B490968B1FBF0F0411EC7
:1001E0000020B0EB116F02D04FF0FF307047064A8D
:1001F000FF231370054A06231360516004490870F9
:1002000090607047C462002023ED00E010E000E041
:10021000407A0020B0B500F10C01C289D1E85F3FFF
:100220009A4202D8BFF32F8F04E05C1CC1E8554FFF
:1002300005B1F3E7C28999B20020914238BF01208D
:10024000B0BD10B5930712D400F12803D0071ED11A
:1002500053E8000F084203D1BFF32F8F002005E0C1
:1002600020EA010243E8002404B1F1E710BD806AEE
:1002700000EA01038B42014618BF002112F001027F
:1002800008BF014653EA020018BF084610BD53E8F4
:10029000000F00EA01028A4203D0BFF32F8F002033
:1002A00005E020EA010243E8002404B1EFE710BDB5
:1002B000B0B5104A0023443215462C683CB125697C
:1002C000A94209D3491B04F10C052346F5E7002494
:1002D000C0E90234016106E0C0E902340161A060B6
:1002E0002569691A2161002B18BF03F10C02106007
:1002F000B0BD00BF48630020EFF3058129B9EFF3DB
:10030000108111B9EFF3118111B16FF00500704741
:10031000DFF804C000DF704729100208EFF3058200
:100320002AB9EFF3108212B9EFF311820AB100F08B
:1003300085BEDFF808C000DF704700BF3D1002082F
:10034000EFF3058129B9EFF3108111B9EFF31181B2
:1003500039B120B10178F32904BFC068704700208B
:100360007047DFF808C000DF704700BF6B1002085D
:10037000EFF3058129B9EFF3108111B9EFF3118182
:1003800009B100207047DFF808C000DF704700BFE8
:100390007D100208B0B5EFF305822AB9EFF31082A1
:1003A00012B9EFF31182AAB16FF0030480B10029F2
:1003B0000ED40278F32A0BD100F10C0252E8003F70
:1003C00043EA010442E8004505B1F7E700F0F8FA16
:1003D0002046B0BDDFF804C000DFB0BDE910020860
:1003E00010B5EFF305842CB9EFF3108414B9EFF3D3
:1003F00011848CB16FF0030460B100290AD44BB9A9
:100400000378F32B06D1FFF734FE0446002808BF1B
:100410006FF00204204610BDDFF804C000DF10BDFD
:1004200069110208EFF3058028B9EFF3108010B9C5
:10043000EFF3118010B10348C0687047DFF808C0BF
:1004400000DF704748630020C511020880B500F046
:10045000F8F8EFF3058028B9EFF3108010B9EFF347
:10046000118010B16FF0050080BDDFF808C000DF1B
:1004700080BD00BFD1110208EFF3058028B9EFF36A
:10048000108010B9EFF3118010B16FF005007047C4
:10049000DFF804C000DF704721130208F8B51446E6
:1004A0000E460546EFF3058028B9EFF3108010B92A
:1004B000EFF31180F0B16FF003000DB303BBFEB199
:1004C0002978FA291CD12846FFF70AFE78B16A6A12
:1004D000074600F10C013046FFF7C6F80CB1F8787A
:1004E00020703846FD6000F06BFA0020F8BD6FF018
:1004F0000200F8BD2846DFF80CC03146224600DF76
:10050000F8BD00BFA9130208EFF305832BB9EFF381
:10051000108313B9EFF311830BB100207047DFF89C
:1005200008C000DF704700BF891402082DE9F041C0
:1005300090460D460646EFF3058028B9EFF310808C
:1005400010B9EFF3118018B36FF00307EEB1E3B900
:10055000DDB13078FA2818D106F10C0000F0EBF884
:1005600088B1726A04460C302946FFF77DF80027EF
:10057000F920C4E9015684F80380A7702070204652
:1005800000F01EFA01E06FF002073846BDE8F08186
:100590003046DFF80CC02946424600DFBDE8F08156
:1005A000B9150208EFF305822AB9EFF3108212B9E8
:1005B000EFF3118212B16FF005007047DFF804C04D
:1005C00000DF704779160208EFF3058129B9EFF3D0
:1005D000108111B9EFF3118109B100207047DFF8E4
:1005E00008C000DF704700BF0D170208EFF3058158
:1005F00029B9EFF3108111B9EFF3118111B16FF047
:1006000005007047DFF804C000DF70477517020867
:10061000F8B5876804469FB13D4695F82320696A7E
:10062000BF682046FFF725FD0028F4D0064628467F
:1006300000F02DFB28463146002200F0C5FBEAE71A
:10064000F8BD7047F0B5002390B389B3032A2FD8C3
:10065000034653F8084F0F3121F007012546E61AEB
:100660005C6824F00307F61B8E4205D22C682B46EB
:10067000002CF3D100231BE0D0E900650D44456058
:10068000304450F8046CAE4202D2083845605C68D1
:1006900054B1186824F00304E05041EA0200E11864
:1006A000486019600B4602E041EA020058600833D6
:1006B0001846F0BDB0B50022E8B1E1B100F1080480
:1006C000A1F108020023944206D0254624682B4657
:1006D000002CF8D100220EE051F8045C446825F0AB
:1006E0000305641B446013B11068186002E0002029
:1006F00041F8040C01221046B0BD08B1420702D0F7
:1007000000221046704700221829FAD311F007037F
:10071000F7D110B50A18A2F108038360002342F84C
:10072000083C8268102454600122C0E90014C360B0
:10073000BDE81040E5E710B5002817D0014600F1EC
:10074000140252E8000F10B9BFF32F8F04E00368C2
:1007500042E8003404B1F4E740B1043151E8002F1D
:10076000531C41E8003404B1F8E710BD002010BD6F
:10077000B0B500281ED0C2688A421BD802698A42DE
:1007800018D900F1140213680B60BFF35F8F52E8B1
:10079000003F0C689C42F6D142E8001505B1F2E733
:1007A000043050E8001F4A1E40E8002303B1F8E778
:1007B0000020B0BD6FF00300B0BDB0B5044600200E
:1007C000ACB1A1B19AB193B10020C4E9001004F119
:1007D000080002FB01352CC0481E636120B1991846
:1007E000196001380B46F9E7002018600120B0BD00
:1007F000F8B50446807868B3E56821462846FFF7D7
:10080000BBFC002005F10C06207030462146FFF7A6
:10081000AFFFA868E8B13046FFF78DFFC8B10446C6
:10082000284600F015FA002100220646002700F0B5
:10083000CBFA304600F06CFA81686A6A064604F129
:100840000C00FEF711FFF920A7702070F068E0702F
:1008500025E0F8BDA568A86808B3407883281ED1B4
:10086000284600F0F5F9002100220646002700F096
:10087000ABFA304600F04CFA064680686A6A04F12A
:100880000C01FEF7F1FEF06808B1E1780170277005
:1008900005F10C002146BDE8F840FFF769BF284686
:1008A0002146BDE8F840FFF73BBC2DE9F041044686
:1008B00000274FF00108D4B12546E87864690007A5
:1008C000F9D52F76A8680028F5D0284600F0C0F9A1
:1008D00000210022064600F077FAC5E90367F06AB6
:1008E000686100B1056185F81880F562E3E7BDE84D
:1008F000F081B0B5C278920715D5C068C36A90F888
:1009000021209C688C4208BF8C682CB194F920404F
:1009100055B2AC42C8BFE2B25B69002BF1D190F88E
:100920002010914200D1B0BD80F82020BDE8B04039
:1009300000F0BDB970B5214C04F1560504F15A061A
:10094000B4F85400D5E85F1F11B9BFF32F8F04E04E
:100950004A1EC5E8532F03B1F4E7090429D0D6E8AD
:100960005F1F4A1C904200D80022C6E8532F03B1F3
:10097000F5E788B2E16D51F82000D0B10178F13986
:100980000829DDD8DFE801F006050905050C0F058B
:100990001200D5E7216E8847D2E7616E8847CFE71E
:1009A000A16E8847CCE7E16E8847C9E7216F884789
:1009B000C6E70020BDE8704000F0F2B848630020B0
:1009C00070B50146194800F15603B0F85420D3E839
:1009D0005F4FA24202D8BFF32F8F04E0651CC3E82B
:1009E000565F06B1F3E7A3B2934214D200F1580365
:1009F000D3E85F4F651CAA4200D80025C3E8565FC4
:100A000006B1F5E7C36DA2B243F82210417A39B1BD
:100A10000121817270BD0220BDE87040FEF7CABDA1
:100A200003484FF08051016070BD00BF4863002053
:100A300004ED00E010B58168B1B100F10C01D1E81E
:100A40005F2F12B9BFF32F8F04E0531EC1E8543F4C
:100A500004B1F4E7110407D000F0FAF800210022F5
:100A6000BDE8104000F0B0B910BD000010B5012184
:100A700041700B4990F920301C310A46896841B118
:100A800091F920409C42F8DCC0E9021290600C31E0
:100A900004E00021C0E9021202F10801086010BD63
:100AA00048630020B0B54A1C0DD01A4A00242C32ED
:100AB00015462B68DBB1DD69A9421AD3491B03F146
:100AC00010051C46F5E71349002330310C461A4641
:100AD000236803F11004002BF9D14FF0FF33C361F9
:100AE0000023C0E904329AB102F1100110E00025A0
:100AF00000E00125002CC0E90434C16118BF04F1F5
:100B0000100210602DB1DA69511AD96103F1140194
:100B10000860B0BD48630020C2690169531C0AD057
:100B200021B143694B61CB691A44CA6142693AB940
:100B30000748C162704709B142694A6142691AB106
:100B4000002343611161704701480163704700BF92
:100B50004863002070B5114DEC6A1CB1E0690138A2
:100B6000E06100D070BD042660781338B6EB301F0A
:100B700005D1204600F095F82146FFF7BAFE204641
:100B800000F085F8204600F0B9F8246924B1E06946
:100B90000028E9D000206061EC6270BD486300204D
:100BA000B0B5054613484469017A65B1022905D1FB
:100BB00094F9200095F92010814211DC2846BDE807
:100BC000B04000F09BB8022912D1456A85B194F972
:100BD000200095F9201081420ADD284600F057F8E0
:100BE0002046FFF743FF2846BDE8B04000F0C8B8F4
:100BF000B0BD00BF4863002010B50446002020802F
:100C0000A07881070DD5C00605D41048216B406F30
:100C1000FFF750FD05E00D48216BD0F88400FFF789
:100C2000A7FDA078C00708BF10BD0849D1F888000B
:100C300020B12146BDE81040FFF79ABDD1F88000F1
:100C40002146BDE81040FFF735BD00BF48630020D6
:100C50000146806882688A6002B1D1600021C1606B
:100C6000704710B591F920300246806840B190F984
:100C700020409C42F8DAC1E9020291600C3004E0A5
:100C80000020C1E9020202F10800016010BDC16844
:100C900031B182688A60826802B1D1600021C1608E
:100CA00070470178F12918BF7047C068F9E7B0B5FF
:100CB0000446054625B12878F12802D1ED68F9E708
:100CC000B0BD2046FFF7E3FF28462146BDE8B0400F
:100CD000FFF7C7BF10B50446407833280DD194F80C
:100CE0002320616A2046FFF7ACFA30B10146204666
:100CF0000022BDE8104000F067B810BD0146012099
:100D0000487002481C30FFF7ACBF00BF48630020AA
:100D1000806B2030704700000748416939B1086B8B
:100D20008A6B824204D90068044A904200D170471D
:100D30000120FEF73FBC00BF48630020A52E5AE209
:100D400070B50B4C0B48A26D666E002100F034FEAE
:100D5000094DA8624EB1E26D0848002100F02CFE5A
:100D6000A864002818BF012070BD012070BD00BF1D
:100D7000683E0208B1F50108486300205D0E0208D4
:100D80000249886102214170FFF7C6BF4863002015
:100D900010B50C4C0246237A0020022B11D1636A55
:100DA0007BB160694270FFF77DFE606A81686162B5
:100DB00011B104F11C02CA600021C160FFF7E0FF1D
:100DC000012010BD48630020B0B50446806B154675
:100DD00001622046FFF7A0FE20461DB1BDE8B040ED
:100DE000FFF7DEBEBDE8B040FFF788BFB0B5FFF744
:100DF000D1F9194DE968286D0131E96000B18047EA
:100E0000FFF7A8FE0020FFF7CBFE296C11B3AA69FB
:100E1000A86B90421CBFC5E90E21B0BDE96B11B1B2
:100E20000139E96316D1297A022913D16C6A8CB190
:100E300090F8200094F8201081420BD12046FFF753
:100E400026FFA86BFFF75AFF2046FFF799FF286C93
:100E5000C5E90E40B0BD00BF4863002082B00B481A
:100E60000821D0E91820FFF74FFB094D09496C46CE
:100E7000C5E91301214600224FF0FF33FFF70EFBB7
:100E800010B9DDE900108847E86CF3E7683E020816
:100E900048630020990E020870B5134D6C6C14B3B2
:100EA0002069012601382061ECB12069D8B9E068D9
:100EB00008B1A16881606864E86C04F1180100223F
:100EC0000023FFF733FB18B103202146FEF772FB26
:100ED000E078012804D161692046FFF7E9F900E0D4
:100EE00066706C6CE0E770BD48630020EFF305822C
:100EF0002AB9EFF3108212B9EFF31182CAB16FF081
:100F00000302A0B199B90178F62910D10C30D0E8CC
:100F10005F1F11B9BFF32F8F04E04A1EC0E8532FA3
:100F200003B1F4E70022080408BF6FF00202104684
:100F30007047DFF808C000DF704700BF29180208BB
:100F4000EFF305832BB9EFF3108313B9EFF311839C
:100F50000BB100207047DFF808C000DF704700BF0A
:100F60008118020810B50446EFF3058028B9EFF3A5
:100F7000108010B9EFF3118090B15CB12078F628A1
:100F800008D12046FFF746F938B12046FFF718FD93
:100F9000002010BD6FF0030010BD6FF0020010BD07
:100FA0002046DFF808C000DF10BD00BF01190208AD
:100FB000DFF804C000DFFEE739190208EFF305810E
:100FC00029B9EFF3108111B9EFF3118111B14FF08D
:100FD000FF307047DFF804C000DF7047A119020836
:100FE000EFF305832BB9EFF3108313B9EFF31183FC
:100FF0000BB100207047DFF808C000DF704700BF6A
:10100000B9190208EFF3058129B9EFF3108111B97D
:10101000EFF3118111B16FF005007047DFF804C0E4
:1010200000DF7047891B020830B180B501461320EC
:10103000FFF7AEFEBDE880400020704710B588B1D4
:1010400002466FF0030000290BD41378F32B08D16C
:101050000C3252E8000F20EA010342E8003404B1E8
:10106000F7E710BD6FF0030010BD20B10178F32940
:1010700004BFC068704700207047000010B550B131
:1010800001460468806870B182070FD1CA680021E8
:10109000102A15D221E000241149D1F8900038B16E
:1010A000FFF749FB0AE0C8680028F5D0002114E0EA
:1010B000D1F8800010210122FFF7C4FA58B10121B4
:1010C0000022C0E90142C2608170F321017004492D
:1010D000044A4A6600E000200146084610BD00BFF1
:1010E00048630020110602082DE9F041002831D0A4
:1010F00005466FF00300002934D42A78F32A31D151
:1011000005F10C0050E8002F42EA010440E80043DA
:1011100003B1F7E7A046AC6804B3264696F823204F
:10112000716AA4682846FEF7A4FF0028F4D0074699
:1011300096F82300800738465CBF706A27EA0000F3
:1011400080463046FFF7A3FD304639460022FFF7C0
:101150003BFEE1E76FF00300BDE8F0810020FFF700
:101160001FFD4046BDE8F081F8B580B10C4606464B
:101170006FF00300002909D43178F32906D13046F5
:1011800021461F461546FEF774FF18B1F8BD6FF0F3
:101190000300F8BD87B143203946FFF7F9FD40B1A0
:1011A0000748476930463946FFF75BFD87F823500B
:1011B0007C626FF00100F8BD6FF00200F8BD00BF67
:1011C000486300200148C068704700BF48630020A2
:1011D0002DE9F8434F4F387A30B1012800F096805E
:1011E0004FF0FF30BDE8F88307F108009C21FEF7BF
:1011F00054FADFF82481B8F81000D8E90B41A7F8B9
:101200005400D8E90202FA6538642046FFF775FAFF
:1012100008B1C7F88040D8E90541DFF80091D8E966
:1012200007562046C847D7F88010002818BF214627
:10123000796728463146C847D7F88010002818BF7C
:101240002946B967D8E909412046C847D7F8801030
:10125000002818BF2146D8F83440F9673CB121680E
:10126000D4E902232046FFF7A8FAC7F88440D8F84B
:1012700038403CB12168D4E902232046FFF79DFAAB
:10128000C7F88840D8F83C403CB12168D4E9022333
:101290002046FFF792FAC7F88C40D8F840403CB19E
:1012A0002168D4E902232046FFF787FAC7F8904067
:1012B000D8F844403CB12168D4E902232046FFF726
:1012C0007CFAC7F89440D8F848403CB12168D4E98A
:1012D00002232046FFF771FAC7F89840D8F84C402F
:1012E0003CB12168D4E902232046FFF766FAC7F82B
:1012F0009C40D8F850403CB12168D4E902232046F4
:10130000FFF75BFAC7F8A040012038720020BDE863
:10131000F88300BF48630020683E0208FB0602080D
:10132000B0B51D4C207A01281CD1FFF709FDC8B1CA
:101330001A48FF218175817D026881F0FF01B1FAB1
:1013400081F1C1F12001C2F302228A4228BF511C5F
:10135000FE2202FA01F1124DC17468681149FEF7CC
:1013600039FF10B14FF0FF30B0BDFEF72FFF206105
:10137000FEF716FF04F11C00FFF76AFCFFF700FD03
:101380002878C0070CBF0320022080F314880220B5
:1013900020720020B0BD00BF486300200CED00E0CB
:1013A000683E020851F601082DE9F84300284CD0A8
:1013B0000F466FF00305002949D004460078FA284B
:1013C00045D1204699469046FEF78AFE002841D036
:1013D000064620463146FEF7CFFE626A06F10C0152
:1013E0003846FEF741F9B8F1000F1CBFF07888F8D5
:1013F000000004F10C070025384631463570FFF730
:10140000B7F9A06818B33846FFF795F90025F0B191
:1014100006462046FFF71CFC002101220746FFF785
:10142000D3FC3846FFF774FC8168626A074606F110
:101430000C00FEF719F9F920B5703070F8683146E4
:10144000F0702046FEF76CFE01E06FF003052846C1
:10145000BDE8F883B9F1000F10D083204946FFF7AB
:1014600097FC40B1074841692046FFF7FAFBEFF3CC
:101470000980C0E902786FF00105E8E76FF0020526
:10148000E5E700BF486300202DE9F84F002770B161
:101490000D4661B105F10F0121F003060446B0FAD3
:1014A00080F0B6FA86F10844202803D20027384697
:1014B000BDE8F88F06FB04F872B1D2F808A01368F3
:1014C000D2E90490BAF1000F11D05FEA8A71EDD130
:1014D000D1683429EAD30DE000234FF000093449E4
:1014E0000093D1F8A00078B1FFF725F912E0D16898
:1014F0000029DBD1B9F1000F2FD000274045D6D30A
:1015000019F003002BD0D2E7D1F88000342101225A
:10151000FFF798F882464FF0010BB9F1000F10D198
:10152000BAF1000F0DD0224F4146F86F0022FFF7AD
:1015300089F8814638B148464146FEF7AEF857462D
:101540001AE057461AE0BBF1000F14D0D7F8A000FC
:1015500060B15146FFF70CF90DE00028A6D1BAF1B1
:10156000000FBCD000934FF0000BD6E7D7F88000F7
:101570005146FFF79FF800270BF1020B002F3FF4B5
:1015800096AF0020C7E90950C7E90B000099324621
:10159000C7E90110FA2087F802B0387007F10C0093
:1015A00021464B46FFF709F90148024901677EE7EA
:1015B00048630020F10702082DE9F84338B30E46CE
:1015C0006FF00307002951D005460078FA284DD165
:1015D000A86899469046E8B1407883281AD12846F1
:1015E000FFF736FB0021012204460027FFF7ECFB42
:1015F0002046FFF78DFB044680686A6A3146FEF795
:1016000033F8E06890B380F8008000272EE06FF098
:1016100003072BE005F10C00FFF78DF880B16A6A33
:1016200004460C303146FEF71FF80027F92084F8F5
:101630000380A770207028462146FEF771FD15E053
:10164000B9F1000F10D093204946FFF7A1FB40B13C
:10165000084841692846FFF704FBEFF30980C0E919
:1016600002686FF0010701E06FF002073846BDE83D
:10167000F88300BF4863002070B5044622484569DE
:101680004DB32CB32078F52822D1207E30B30E46FE
:10169000E178CA0702D0E268AA422BD066B3880775
:1016A0000AD5E06895F9201090F920208A4203DAE3
:1016B00080F82010FFF7FBFA53203146FFF768FB54
:1016C00018B120462946FFF7CCFA6FF0010070BD33
:1016D0006FF0030070BD4FF0FF3070BD0020C4E913
:1016E0000350E86A606100B10461012020760020A7
:1016F000EC6270BDFF2802D16FF0020070BD0130B6
:101700002076002070BD00BF4863002070B550B146
:101710008468D0E900657CB1A10710D1C1680020C0
:101720001C2917D270BD002500261149D1F894005C
:1017300038B1FFF700F80AE0C0680028F5D00020B3
:1017400070BDD1F880001C210122FEF77BFF04460A
:1017500058B101206660E570A070F520207004F19A
:1017600008001121FDF799FF00E00024204670BD1C
:101770004863002070B504462A48406970B154B1EE
:101780002178F52907D1217E11B1E268824209D082
:101790006FF0020404E06FF0030401E04FF0FF3447
:1017A000204670BD01392176090601D00024F7E7F3
:1017B000616909B122690A6100F12C0223691546A9
:1017C000002B18BF03F114052960E17889070FD5B4
:1017D00090F8211012684AB193682BB193F9203028
:1017E0004DB2AB42C8BF19461432F3E780F820105F
:1017F000A06888B12046FFF72BFA00210022054699
:101800000026FFF7E1FAC4E90356E86A606100B117
:10181000046101202076EC6200200024FFF7C0F96B
:10182000BEE700BF48630020B0B508B304460078A7
:10183000F6281DD104F10C00D0E85F2F12B9BFF3D8
:101840002F8F04E0531EC0E8553F05B1F4E71004A4
:101850001CBF0020B0BD71B16320FFF799FA20B121
:10186000064841692046FFF7FCF96FF00100B0BD62
:101870006FF00300B0BD6FF00200B0BD4863002000
:1018800070B5054601384FF6FE730C4600219842AC
:1018900098BFAC4201D9084670BD4AB1906816683D
:1018A00070B181070FD1D2680021102AF3D314E060
:1018B00000261149D1F8980038B1FEF73CFF0AE044
:1018C000D0680028F5D00021E5E7D1F8800010218C
:1018D0000122FEF7B7FE60B101210022C58184819B
:1018E000C0E901628170F62101700349034A8A66EA
:1018F00000E000200146CEE748630020350A0208D8
:1019000010B560B10178F62909D1816859B1FFF7A6
:101910009FF9002101220024FFF756FA01E06FF041
:101920000304204610BDFEF775FC0024002808BF04
:101930006FF00204F5E7000070B5184D287A022810
:101940002AD1686A40B36C69E06AFEF7AEFFA0690D
:1019500018B100210022FFF737FAEFF30980A063E6
:10196000686A8168696211B105F11C02CA600026CB
:10197000C660FFF705FA6E61E078C00704D1204623
:10198000BDE87040FFF738B90420E6606070686B0E
:10199000A06000B1C4606C6370BD00BF48630020EC
:1019A00030B10178F12903D1407800F00F00704781
:1019B0004FF0FF30704700002DE9FE4F18B380460E
:1019C0006AB102F1100A96689AE88006D2E90053DB
:1019D000BEB1B00717D1D068442814D317E0012452
:1019E0004FF0180A002300274FF000090025614A34
:1019F0000293D2F88800CDE90015C0B1FEF79BFE36
:101A00001BE0D06818B100242046BDE8FE8F37B136
:101A10000024B9F1000FF7D017F00700F4D1BAF1A4
:101A2000000F24D0AAF101003728ECD821E0D2F829
:101A3000800044210122FEF705FE06464FF0010B0F
:101A400087B97EB184B14B494B4AD1F88400D2F8B2
:101A50005490C8B1FEF76FFE0746002818BF0BF17F
:101A6000100B17E0344635E04248406F0DE04FF070
:101A7000180AB9F1000F1BD00024B9F1480FC3D3E5
:101A800019F0070015D0BFE7486F49460022FEF75E
:101A9000D9FD07460FB134461AE05FEACB7016D085
:101AA0003449D1F8880068B13146FEF761FE0EE096
:101AB0000124002E3FF49BAFCDE9001502934FF0B7
:101AC000000BBDE7D1F880003146FEF7F3FD00249E
:101AD0004BF0020B002C3FF497AF01981821606087
:101AE0000298E07040F2F11084F802B0208004F116
:101AF0000800FDF7D2FD07EB090100204039FD2267
:101B0000C4F82300C4F82700C4F82B0084F82F0081
:101B100084F8222084F821A084F820A0C4E90C795C
:101B2000C4E90E181549009D396013490978490721
:101B30000AD56FF0100101EB99013A1D4FF0CC333B
:101B400011B108C20139FBE7A16B00220D2A03D0B5
:101B500041F822000132F9E7094A4FF08070C1E9EB
:101B60000D28C8630D620348064901662046FFF749
:101B700017F849E748630020683E0208A52E5AE29C
:101B8000B10F0208D50C020870B5C0B10446007848
:101B9000F12814D1607800F00F00012812D003283A
:101BA00014D002281CBF6FF0020070BD24496FF0F2
:101BB00002000A7A022A01D1496A69B970BD6FF040
:101BC000030070BD2046FFF762F805E02046FFF7EE
:101BD0005EF82046FEF7A0FFE06AFEF766FEA06909
:101BE00018B100210022FFF7EFF86078022810D129
:101BF000134DEFF30980A063686A8168696211B1CF
